:020000040800F2
:1000000000070020F10100087D26000835260008C1
:100010005D2600083526000855260008F301000873
:10002000F3010008F3010008F30100080537000898
:10003000F3010008F3010008F3010008F3010008D0
:10004000F3010008F3010008F3010008F3010008C0
:10005000F3010008F3010008F9390008213A00080B
:10006000493A0008713A0008993A0008F30100087B
:10007000F3010008F3010008F3010008F301000890
:10008000F3010008F3010008F3010008F301000880
:10009000F30100081526000825260008C13A0008CB
:1000A000F3010008F3010008F3010008F301000860
:1000B000953B0008F3010008F3010008F301000874
:1000C000F3010008F3010008F3010008F301000840
:1000D000F3010008F3010008F3010008F301000830
:1000E000253B0008F3010008F3010008F3010008B4
:1000F000F3010008F3010008F3010008F301000810
:10010000F3010008F3010008F3010008F3010008FF
:10011000F3010008F3010008F3010008F3010008EF
:10012000F3010008F3010008F3010008F3010008DF
:10013000F3010008F3010008F3010008F3010008CF
:10014000F3010008F3010008F3010008F3010008BF
:10015000F3010008F3010008F3010008F3010008AF
:10016000F3010008F3010008F3010008F30100089F
:10017000F3010008F3010008F3010008F30100088F
:10018000F3010008F3010008F3010008F30100087F
:10019000F3010008F3010008F3010008F30100086F
:1001A000F3010008F3010008F3010008F30100085F
:1001B000F3010008F3010008F3010008F30100084F
:1001C000F3010008F3010008F3010008F30100083F
:1001D000F3010008F3010008F3010008F30100082F
:1001E000550F0008000000000000000000000000A3
:1001F00002E000F000F8FEE772B6374880F30888A6
:10020000364880F3098836483649086040F20000D5
:10021000CCF200004EF63471CEF200010860BFF35C
:100220004F8FBFF36F8F40F20000C0F2F0004EF628
:100230008851CEF200010860BFF34F8FBFF36F8F7C
:100240004FF00000E1EE100A4EF63C71CEF20001D4
:100250000860062080F31488BFF36F8F04F034F930
:1002600004F014FA4FF055301F491B4A91423CBF2D
:1002700041F8040BFAE71D49184A91423CBF41F886
:10028000040BFAE71A491B4A1B4B9A423EBF51F82E
:10029000040B42F8040BF8E700201849184A914271
:1002A0003CBF41F8040BFAE704F012F904F034FA09
:1002B000144C154DAC4203DA54F8041B8847F9E797
:1002C00000F042F8114C124DAC4203DA54F8041B12
:1002D0008847F9E704F0FAB800070020002300205F
:1002E0000000000808ED00E00001002000070020E9
:1002F000B049000800230020A4230020A8230020E8
:1003000014510020E0010008E4010008E4010008A5
:10031000E40100082DE9F04F2DED108AC1F80CD052
:10032000C3689D46BDEC108ABDE8F08F002383F3BF
:1003300011882846A047002003F06AFDFEE703F07D
:10034000F3FC00DFFEE70000F8B500F015FE04F056
:100350005DF8074604F0AEF80646C0BB274B9F4247
:1003600035D001339F4235D0254B27F0FF029A420A
:1003700033D1F8B200F036FC354642F2107400F08A
:1003800037FC08B10024254601F0EAF848B3032001
:1003900000F03AF80024254636B11A4B9F4203D0AC
:1003A00004F080F800242546002004F039F80DB14F
:1003B00000F040F800F050FC02F068F90546ACB9D6
:1003C00000F092FC4FF47A7003F028FDF7E7354611
:1003D0000024D4E704460125D1E705464FF47A749A
:1003E000CDE7B4F57A7F08BF0125D5E702F04EF9D5
:1003F000431BA342E4D900F01DF8DDE7010007B07C
:10040000000008B0263A09B0084B187003280CD831
:10041000DFE800F008050208022000F009BE022013
:1004200000F0FEBD024B00225A607047A823002056
:10043000AC23002010B501F093F830B1234B032218
:100440001A70234B00225A6010BD224B224A1C46D0
:1004500019680131F8D004339342F9D16268A2429D
:10046000F2D31E4B9B6803F1006303F520439A42CD
:10047000EAD203F0E9FF03F0FBFF002000F096FD55
:100480000220FFF7C1FF164B9A6D00229A65996F03
:100490009A67996FD96DDA65D96FDA67D96F196E76
:1004A0001A66D3F88010C3F88020D3F8803072B673
:1004B0004FF0E0233021C3F8084DD4E9003281F336
:1004C00011889D4683F308881047BDE7A8230020C4
:1004D000AC23002000A0000820A00008002300207A
:1004E00000100240094A136849F2690099B21B0CD6
:1004F00000FB01331360064B186844F2506182B26E
:10050000000C01FB0200186080B270471423002029
:100510001023002010B500211022044600F0A2FD97
:10052000034B03CB206061601868A06010BD00BF62
:100530009075FF1FF0B5ADF54F7D6CAC4FF4C472F4
:1005400007460D462046002100F08CFD02F09EF883
:10055000244B4FF47A72B0FBF2F0186093E8070076
:10056000022384E807000DF5E9702382FFF7D2FF2C
:1005700041F204031C49238406A804F033F919232B
:1005800084F832310DF2E32206AB0DF1300C1E4639
:1005900003CE664510605160334602F10802F6D181
:1005A000337813700DAE31460122204600F0A6FDCF
:1005B00000230393AB7E029305F11903019380B2EC
:1005C0000123CDE904600093E97E04A3D3E900236D
:1005D000384602F067FC0DF54F7DF0BD9E6AC421E0
:1005E000818A46EEB4230020F44700082DE9F0414B
:1005F0002C4C237ADAB080460D465BBB27A92846EF
:1006000000F0A2FE0746002842D19DF89D60C82E4A
:100610003ED801464FF4A662204600F023FD4FF479
:100620008073C4F8F8314FF40073C4F80C334FF4FE
:100630004073C4F8203432460DF19E0104F10900E4
:1006400000F0FEFC26449DF89C30777223720BB9B3
:10065000EB7E23728122002106AC27A800F002FD68
:100660000122214627A800F0B5FE00230393AB7EAC
:10067000029305F1190380B201932823CDE90440C8
:100680000093E97E05A3D3E90023404602F00AFC6B
:100690005AB0BDE8F08100BFAFF30080264172720E
:1006A000DF25D7B7FC330020F0B5254E4FF48A750F
:1006B00005FB0065F1B096F8D83085F8DC300024F1
:1006C000D822214685F8E8403AA800F0CBFC06F194
:1006D000090000F0BFFCD5F8E4308DF8F000C2B29C
:1006E00006AF06F109010DF1F100CDE93A3400F051
:1006F000A7FC394601223AA800F0A2FE80B2CDE95B
:10070000047008230127CDE9023706F1D8030193CD
:1007100030230093317A0B4807A3D3E9002302F07A
:10072000C1FBA04206DD01F0B1FFC5F8E00038468C
:1007300071B0F0BD2046FBE778F6339F93CACD8DAC
:10074000FC330020CC3300202DE9F0411D4D1E4E1E
:100750001E4F86B0284602F0D1FB034658B3002452
:10076000CDE90344ADF81440027B8DF8142099685C
:100770004068029403AA03C21B68DFF8548043F068
:100780000043029301F084FF821941F100030094B9
:1007900002A9384601F0DCF8A04205DD284602F047
:1007A000B1FB88F80040D5E798F80030072B05D852
:1007B000013388F8003006B0BDE8F081014802F04E
:1007C000A1FBF8E7CC33002040420F00383900206D
:1007D0003139002070B50D4614461E4602F0BEFAAF
:1007E00050B9022E10D1012C0ED112A3D3E900234F
:1007F000C5E90023012007E0282C10D005D8012CE2
:1008000009D0052C0FD0002070BD302CFBD10BA3DC
:10081000D3E90023ECE70BA3D3E90023E8E70BA31C
:10082000D3E90023E4E70BA3D3E90023E0E700BF0B
:10083000AFF30080401DA12026812A0B78F6339F5C
:1008400093CACD8D9E6AC421818A46EE264172727A
:10085000DF25D7B7F017304A39059E5638B505461B
:100860000E4C0021013500F0C3FBA4F82C55B4F860
:100870002C0500F0A5FB78B1B4F82C0500F0B0FB16
:10088000014648B9B4F82C0500F0B2FBB4F82C3599
:100890000133A4F82C35EAE738BD00BFFC33002053
:1008A00010B50A4B0A4A1A6003F5805393F8582092
:1008B0003AB95C6D2CB1204600F0CCFE204601F028
:1008C00003F8BDE81040034800F0C4BE38390020EA
:1008D00040480008784900202DE9F04F8FB000AF64
:1008E00005460C4602F03AFA00284BD1237E022B33
:1008F0001BD1E38A012B18D101F0C8FE0646FFF791
:10090000F1FD03464FF4C870DFF8D482B3FBF0F278
:1009100006F5167602FB103316FA83F3C8F800309A
:10092000E37E33B9A74B00221A703C37BD46BDE8C1
:10093000F08F07F12401204600F0BAFC0028F4D122
:1009400007F11400FFF7E6FD97F8264007F11401C0
:10095000224607F1270003F013FF0028E2D10F2CF5
:1009600008D8984B1C70D8F80030A3F51673C8F857
:100970000030DAE797F824100029D6D0284602F094
:10098000E5F9D2E7E38A282B33D010D8012B2BD0FE
:10099000052BCAD1BFF34F8F8B498C4BCA6802F429
:1009A000E0621343CB60BFF34F8F00BFFDE7302BF6
:1009B000BBD1874EE17E327A9142B6D1607E31461C
:1009C000002291F8DC50854200F0AD800132042A0B
:1009D00001F58A71F5D1326840F6B831FA328A42AF
:1009E00094BF32603160A0E721462846FFF7A2FDA0
:1009F0009BE721462846FFF7F9FD96E7B2F8EC5051
:100A00007B6005F103094FEA99094FEA8902D11D7C
:100A1000C908A8EBC1039D46EB460021584600F0EB
:100A200021FB04F1EE012A463144584600F008FB50
:100A30007B6813B9012000F0B9FA96F8D20000F0F3
:100A4000BFFA044630B9307200F0DAFA204600F0FE
:100A5000ADFAB0E0D6F8D4203AB996F8D200B6F89C
:100A60002C25824201D8FFF7F9FED6F8D4202A447B
:100A7000944208D296F8D200B6F82C250130824272
:100A800001D8FFF7EBFE70685FFA89F2594600F073
:100A9000F1FA08B9C54679E0726896F8D2002A449E
:100AA0007260D6F8D42005EB0209C6F8D49000F0A5
:100AB00087FA814509D396F8D220D6F8D4000132BE
:100AC000001B86F8D220C6F8D400FF2D0FD80024D2
:100AD000347200F095FA204600F068FA00F040FD0C
:100AE0003C4B188108B9FFF7A5FCC5461DE7BB685C
:100AF00096F8D9000AFB0362FB68D2F8E41082F88A
:100B0000E83001F58061C2F8E030C2F8E410FFF788
:100B1000CBFDFFF719FE96F8D920013202F003024F
:100B200086F8D920B6E74FF48A7A0AFB02F505F178
:100B3000EA013144204600F0B7FCF86000287FF459
:100B4000F4AE3544012285F8E82001F09FFDD5F888
:100B5000E020D6ED007ADFED206A801A192838BF30
:100B6000192040F6B832904228BF1046B8EE677A96
:100B700007EE900AF8EEE77A67EEA67ADFED176ADD
:100B8000E7EE267AFCEEE77AC6ED007A96F8D930E1
:100B90007168BB600AFB03F4321992F8E8505DB14A
:100BA000D2F8E4308B42E8463FF428AF002182F8C7
:100BB000E810C2F8E010C5467368064A9B0A013384
:100BC0001381B2E6C533002000ED00E00400FA0511
:100BD000FC330020B4230020CDCCCC3D6666663FBC
:100BE000C8330020014B1870704700BFC02300209D
:100BF00038B54FF00054144B22689A4221D1607DE1
:100C0000F0B1124B124918701248237D03724FF451
:100C10008073C0F8F8314FF40073C0F80C3300252E
:100C20004FF44073C0F82034C0F8E450C9220930B2
:100C300000F006FAE0222946204600F013FA0120CF
:100C400038BD0020FCE700BF9AAD44C5C02300209A
:100C500016000020FC33002037B500F081FC194D50
:100C60001949288102236B7100220123174801F0E2
:100C7000E9F800230193164B164900931648174BC9
:100C80004FF4805202F03AF8154B197811B112481E
:100C900002F05CF801F0FAFC0446FFF723FC4FF485
:100CA000C873B0FBF3F202FB130304F5167010FADD
:100CB00083F00C4B186003F0FDFB08B10F232B8170
:100CC00003B030BDB423002040420F00383900206B
:100CD000D5070008C4230020CC330020D908000821
:100CE000C0230020C83300202DE9F04F2DED028BEA
:100CF00090A7D7E900670FF24429D9E90089884C09
:100D000095B00DAD9FED848BFFF71EFDDFF834B27B
:100D100000230C93ADF83C300D936B6000230DF174
:100D200025028DED008B4FF0010A09A958468DF878
:100D300025308DF824A001F011FC9DF8242000231B
:100D4000002A40F0AF80204602F008F8054600284F
:100D500047D1DFF8F4B101F099FCDBF8003098429C
:100D60003FD301F093FC0790FFF7BCFB079A4FF4C9
:100D7000C873B0FBF3F101FB130302F5167010FA10
:100D800083F0CBF80000DFF8C4B19BF800100791A6
:100D9000002914BF2B46534610A88DF83030FFF7BA
:100DA000B9FB0799C1F11002D2B2062A10AB28BFD5
:100DB000062219440DF13100079200F041F9079A1B
:100DC0000CAB0393182302930132564BD2B2CDE9F8
:100DD00000A304923B463246204602F005F88BF809
:100DE000005001F053FC504A504D1368C31AB3F53C
:100DF0007A7F32D3106001F04BFC02460B4620464E
:100E000002F08AF8204601F0A9FF30B32B7ADFF810
:100E100040A1002B14BF032302238AF8053001F000
:100E200035FC0DF1400B4FF47A730122B0FBF3F067
:100E30005946CAF80000504600F012FA18230293EF
:100E40003B4B019380B240F25513CDE903B00093C0
:100E500042464B46204601F0C7FF2B7AB3B101F062
:100E600015FC4FF0000A83464FF48A7295F8D900BA
:100E7000504400F0030002FB005393F8E8100029EF
:100E800034D00AF1010ABAF1040FEFD1C82002F000
:100E9000C5FF2B7A002B7FF434AF15B0BDEC028B6D
:100EA000BDE8F08F4FF0904110A84A6982F020020F
:100EB0004A611946102200F0D5F80DF126030AAA5E
:100EC0000CA9584600F06AFE95E8030011AB83E8D0
:100ED00003009DF83C308DF84C300C9B109310A90A
:100EE000DDE90A23204602F0EBF917E7D3F8E0101A
:100EF00049B12B68FA2B38BFFA23ABEB010105335C
:100F0000B1EB430FBDD3FFF7CFFB4FF48A7200283C
:100F1000B7D1BBE7AFF30080000000000000000085
:100F2000CC330020C43300202C390020FC330020B7
:100F300030390020401DA12026812A0BF1C6A7C10F
:100F4000D068080F38390020C8330020C53300208E
:100F5000B423002008B5054800F0C4FEBDE80840F1
:100F6000034A0449002003F0EFBB00BF38390020DA
:100F7000404E0020A108000870B503F0EBF8094EC0
:100F8000094D3080002428683388834208D903F053
:100F9000DDF82B6804440133B4F5204F2B60F2D305
:100FA00070BD00BF344E0020084E002003F084B90D
:100FB00000F10060920000F5204003F007B9000046
:100FC000054B1A68054B1B889B1A834202D91044B3
:100FD00003F0BCB800207047084E0020344E0020BB
:100FE000024B1B68184403F0B7B800BF084E00203E
:100FF000024B1B68184403F0C1B800BF084E002024
:10100000064991F8243033B10023086A81F824306E
:101010000822FFF7CDBF0120704700BF0C4E002013
:10102000022802BF4FF0904320229A6170470000CF
:10103000022802BF4FF090434FF400129A617047AC
:1010400010B50023934203D0CC5CC4540133F9E7BC
:1010500010BD000003460246D01A12F9011B0029F8
:10106000FAD1704702440346934202D003F8011BB1
:10107000FAE770472DE9F8431F4D144695F82420F0
:101080000746884652BBDFF870909CB395F8243031
:101090002BB92022FF2148462F62FFF7E3FF95F886
:1010A0002400C0F10802A24228BF2246D6B241461F
:1010B000920005EB8000FFF7C3FF95F82430A41BD6
:1010C0001E44F6B2082E17449044E4B285F824601A
:1010D000DBD1FFF795FF0028D7D108E02B6A03EB9F
:1010E00082038342CFD0FFF78BFF0028CBD10020B3
:1010F000BDE8F8830120FBE70C4E00202DE9F34703
:101100000D46044600219046284640F27912FFF72A
:10111000A9FF234620220021284602F073F8231D50
:1011200002222021284602F06DF8631D03222221AD
:10113000284602F067F8A31D03222521284602F065
:1011400061F804F1080310222821284602F05AF819
:1011500004F1100308223821284602F053F804F164
:10116000110308224021284602F04CF804F1120332
:1011700008224821284602F045F804F114032022F1
:101180005021284602F03EF804F118034022702155
:10119000284602F037F804F120030822B02128463F
:1011A00002F030F804F121030822B821284602F0A9
:1011B00029F804F12207C0263B463146082228467A
:1011C000083602F01FF8B6F5A07F07F10107F3D14A
:1011D00094F832308DF8073031460DF107030822BC
:1011E000284602F00FF8002604F1330A9DF8073074
:1011F0004FEAC6099E4209F5A47720D394F832310C
:10120000502B28BF50238DF80730B8F1000F08D1BC
:1012100039460DF107030722284601F0F3FF09F2D2
:101220004F17002604F233149DF807309E4207EB57
:10123000C6010DD30731C80802B0BDE8F0870AEB3C
:10124000060308223946284601F0DCFF0136CDE7C7
:10125000A3190822284601F0D5FF0136E4E7000073
:1012600013B504460846002101602346C0F8031068
:101270002022019001F0C6FF0198231D02222021A7
:1012800001F0C0FF0198631D0322222101F0BAFF83
:101290000198A31D0322252101F0B4FF019804F158
:1012A00008031022282101F0ADFF072002B010BD75
:1012B000F7B5047F05460E462CB1838A122B02D95E
:1012C000012003B0F0BD00231946072200962846EE
:1012D00001F05CFE731C00930122002307212846C5
:1012E00001F054FED4B9B31C009305222346082113
:1012F000284601F04BFE0D24B378102BE0D837467A
:10130000B278BB1B934210D32B7FA88A0734E40822
:10131000B3B9844294BF00200120D2E7AB8ADB003E
:10132000083BDB08B3700824E6E7FB1C009321466A
:1013300000230822284601F029FE08340137DFE7A0
:10134000201A18BF0120BCE7F7B5047F05460E46FA
:101350002CB1838ACA2B02D9012003B0F0BD00232F
:10136000194600960822284601F010FE731CD4B9D5
:101370000822009311462346284601F007FE102458
:101380007378C82BE8D8012372785F1C013B934225
:1013900010D32B7FA88A0734E408B3B9844294BFE2
:1013A00000200120D9E7AB8ADB00083BDB08737023
:1013B0000824E5E7F3190093214600230822284674
:1013C00001F0E4FD08343B46DEE7201A18BF012097
:1013D000C3E70000F7B50D4604460021164628462F
:1013E0008122FFF73FFE234608220021284601F014
:1013F00009FF94F901206378002AB8BF7F238DF894
:1014000007309EB90DF1070307220821284601F095
:10141000F9FE0F27002602349DF807309E4207EBA5
:10142000C60105D30731C80803B0F0BD0827F1E7AE
:10143000A3190822284601F0E5FE0136ECE700007A
:10144000F7B50E460546002114463046CE22FFF77A
:1014500009FE2B4628220021304601F0D3FE2B7ACC
:10146000C82B28BFC8238DF807308CB90DF10703AE
:1014700008222821304601F0C5FE30242F469DF871
:1014800007207B1B934205D3E01DC00803B0F0BDCD
:101490002824F3E707F1090321460822304601F02A
:1014A000B1FE08340137EAE7F7B5047F05460E467A
:1014B00034B1838AB3F5827F02D9012003B0F0BD35
:1014C0000096012310220021284601F05FFDDCB9BF
:1014D000B31C0093092223461021284601F056FD33
:1014E00019247388B3F5807FE7D837467288BB1B11
:1014F000934210D32B7FA88A0734E408B3B98442FF
:1015000094BF00200120D9E7AB8ADB00103BDB0849
:1015100073801024E5E73B1D009321460023082239
:10152000284601F033FD08340137DFE7201A18BFE1
:101530000120C3E730B5094D0A4491420DD011F89E
:10154000013B5840082340F30004013B2C4013F0BA
:10155000FF0384EA5000F6D1EFE730BD2083B8EDF9
:10156000F7B5364A106851686B4603C36A4634497A
:101570003448082303F014F9044690BB0A25324A84
:10158000106851686B4603C36A4630492D480823EA
:1015900003F006F90446002847D00369B3F5583F25
:1015A00043D8B0F86620B2F5826F3ED1284A024493
:1015B00002F15C018B4238D35C3B224900209E1A29
:1015C000FFF7B8FF3246074604F164010020FFF739
:1015D000B1FFA3689F4228D1E368984208BF002565
:1015E00023E00369B3F5583F26D8428BB2F5826FEA
:1015F00020D1174A024402F110018B4218D3103B4C
:10160000104900209D1AFFF795FF2A46064604F16F
:1016100018010020FFF78EFFA3689E4202D1E36805
:10162000984201D00D25AAE70025284603B0F0BD59
:101630001025A4E70C25A2E70B25A0E71048000819
:10164000DC5F030000A0000819480008905F030059
:101650000860FFF710B5037C044613B9006803F077
:1016600087F8204610BD00000023BFF35B8FC360E6
:10167000BFF35B8FBFF35B8F8360BFF35B8F7047FC
:10168000BFF35B8F0068BFF35B8F704770B5054693
:101690000C30FFF7F5FF05F1080604463046FFF76A
:1016A000EFFFA04206D930466D68FFF7E9FF2544F9
:1016B000281A70BD3046FFF7E3FF201AF9E7000053
:1016C00070B50546406898B105F10800FFF7D8FFEE
:1016D00005F10C0604463046FFF7D2FF844230463F
:1016E00094BF6D680025FFF7CBFF013C2C44201A06
:1016F00070BD000038B50C460546FFF7C7FFA04295
:1017000010D305F10800FFF7BBFF04446868B4FB81
:10171000F0F100FB1144BFF35B8F0120AC60BFF31D
:101720005B8F38BD0020FCE72DE9F04114460746E9
:101730000D46FFF7C5FF844228BF0446D4B1B84622
:1017400058F80C6B4046FFF79BFF3044286040463A
:101750007E68FFF795FF331A9C4203D86C60012026
:10176000BDE8F0816B60A41B3B68AB602044E8607F
:101770000220F5E72046F3E738B50C460546FFF7AB
:101780009FFFA04210D305F10C00FFF779FF04443E
:101790006868B4FBF0F100FB1144BFF35B8F0120DC
:1017A000EC60BFF35B8F38BD0020FCE72DE9FF4103
:1017B000884669460746FFF7B7FF6C4606B204EB5A
:1017C000C6060025B44209D06268206808EB05010E
:1017D000FFF736FC636808341D44F3E729463846B2
:1017E000FFF7CAFF284604B0BDE8F081F8B505460A
:1017F0000C300F46FFF744FF05F10806044630465B
:10180000FFF73EFFA042304688BF6C68FFF738FF05
:10181000201A386020B130462C68FFF731FF204491
:10182000F8BD000073B5144606460D46FFF72EFFBF
:10183000844228BF04460190DCB101A93046FFF77D
:10184000D5FF019B33B93268C5E90233C5E90024ED
:1018500001200CE09C4238BF019428600198686028
:101860008442F5D93368AB60241AEC60022002B0E0
:1018700070BD2046FBE700002DE9FF410F46694699
:10188000FFF7D0FF6C4600B204EBC0050026AC4267
:1018900009D0D4F8048054F8081BB8194246FFF761
:1018A000CFFB4644F3E7304604B0BDE8F0810000CA
:1018B00038B50546FFF7E0FF044601462846FFF726
:1018C00019FF204638BD000008B102F051BF704733
:1018D0007047000010B41346026814680022A44642
:1018E0005DF8044B6047000000F5805090F86904F3
:1018F0007047000000F5805090F8620470470000C7
:1019000000F5805090F9680470470000502070473F
:10191000302383F3118800F58052D2F8AC34D2F82A
:10192000A8041844D2F8A4341844D2F88C341844CB
:10193000D2F89C341844D2F898341844002383F326
:101940001188704700F58050C0F86414012070477A
:101950002DE9FF470C4600F58051054691F86204D9
:10196000BDF8308098B1D1F888040130C1F88804FE
:101970002068860006D4207B08280BD9667B0EB130
:101980000F2807D9D1F88C340133C1F88C344FF0CB
:10199000FF30AAE0302080F31188E86BD0F8C470E3
:1019A00017F4001713D0D1F890040130C1F8900457
:1019B000D1F89414002940F09B80CDF80080214696
:1019C000284600F0ADFE002383F311888DE0D0F8A7
:1019D000C460686BC6F301464FF0480919FB06095D
:1019E00020680028B4BF40F0804C4FEA804CC9F812
:1019F00000C02068400044BF4CF00050C9F800000F
:101A000094F80CC0300640EA0C40C9F8040094F881
:101A10000DC04FEA461ABCF1000F27D040F4401029
:101A2000C9F80400D1F8C0040130C1F8C00405EBC6
:101A30000A0101F58351087F40F020000877207BE0
:101A4000CDE9022300F0BEFEDDE902230330801061
:101A5000F9B2814207F1010710DA04EB810C09EBBE
:101A60008101DCF804C0C1F808C0F1E705EB0A0108
:101A700001F58351087F6CF34510DFE7E96B012026
:101A8000B040C1F8CC0006F1830105EB4111C1E97A
:101A9000002305EB461101F583512046083104F17E
:101AA0000C0750F804CB41F804CBB842F9D10088B8
:101AB0000880AA4441F278014AF801600AF5805A88
:101AC00008F003019AF87C0041F0100120F01F009B
:101AD00001438AF87C10002181F31188CDF8008041
:101AE0002146284600F01CFE012004B0BDE8F08726
:101AF000002068E738B5C26B936923F00103936156
:101B0000044600F0C3FD0546E36B9B69DB0706D581
:101B100000F0BCFD431BFA2BF6D9002004E004F5CD
:101B20008054012084F8620438BD000013B500F52C
:101B300080540191606DFFF7C3FD1F280AD90199F8
:101B4000606D2022FFF732FEA0F120035842584179
:101B500002B010BD0020FBE708B5302383F31188E5
:101B600000F58050406DFFF77FFD002383F311885F
:101B700008BD0000002202608281426082607047DE
:101B800010B500220023C0E900230023044603818E
:101B90000C30FFF7EFFF204610BD00002DE9F047A5
:101BA0009A4688B0074688469146302383F31188C9
:101BB00007F580546846FFF7E3FF606DFFF766FDA9
:101BC0001F282DD9606D20226946FFF771FE20285D
:101BD00026D194F862341BB303AD444605AB2E46C0
:101BE00003CE9E4220606160354604F10804F6D1C0
:101BF00030682060B388A380DDE90023C9E90023B1
:101C0000BDF80830AAF80030002383F3118853464A
:101C10004A464146384608B0BDE8F04700F044BDAA
:101C2000002080F3118808B0BDE8F0872DE9F84F57
:101C3000064635468846182200210430FFF712FA7E
:101C4000254B45F8403B06F582572C46204620346C
:101C5000FFF796FFA742F9D106F580544FF4805361
:101C600025640025C4E9113501236765E56484F81E
:101C7000503084F8583006F5845706F5A4594FF0D3
:101C8000000A4FF0000B47E908ABA7F11800FFF777
:101C900071FF203747F8285C4F45F4D184F86884F9
:101CA000A4F86A54A4F86C54A4F86E5484F87054E0
:101CB000A4F87254A4F87454A4F8765484F87854B0
:101CC000B8F1000F02D0054800F0DAFC044BF363D2
:101CD0003046BDE8F88F00BF40480008244800089F
:101CE0000064004010B5044B197804464A1C1A7071
:101CF000FFF79CFF204610BD3D4E00202DE9F84324
:101D000015460C4600295CD0022001F06FFE2E49DA
:101D1000B0FBF4F78C428CBF0A2111214B1EB7FB9C
:101D2000F1F601FB1671DAB221B1022B1946F5D892
:101D3000002032E0731EB3F5806FF9D2C2EBC20807
:101D400008F103014FEAE10EC1F3C701A2EB010C58
:101D50000EF101094FF47A735FFA8CF70EFB033E24
:101D600059FA8CFCBEFBFCFCBCF5617F17DC1FFA4A
:101D70008CF34A1C57FA82F27243B0FBF2F08442B1
:101D8000D6D14A1E0F2AD3D87A1E072AD0D80120CE
:101D90002B806E8028716971AF71BDE8F88308F1FE
:101DA000FF314FEAE10CC1F3C701521A0CF1010EE9
:101DB000D7B20CFB03335EFA82F2B3FBF2F39BB2B1
:101DC000D7E70846E9E700BF3F420F0030B50D4BAB
:101DD0000D4D05201C786C438C420ED159785180F2
:101DE00099785171D9789171197911715B7903EBF7
:101DF00083035B001380012030BD013803F106032B
:101E0000E8D1F9E78448000840420F000B4B10B5B9
:101E10004FF45472044600211846FFF723F9084B8B
:101E2000A3624033E362D8332363F0336363E36B2D
:101E300060620022C3F8C02010BD00BF00A40040B3
:101E400070A400402DE9F04700F580551F4695F835
:101E50006834012B88B004468946904604D9002690
:101E6000304608B0BDE8F087994A52F8231009B906
:101E700042F823009748C4F81C90017884F8207039
:101E800099B9302383F31188934B9A6D42F0007215
:101E90009A659A6B42F000729A639A6B22F0007214
:101EA0009A630123037081F3118895F861647EB908
:101EB000302383F311880321152001F0ABFE0321A9
:101EC000162001F0A7FE012385F8613486F31188FE
:101ED000302383F31188E26B936923F0100393613D
:101EE00000F0D4FB8246E36B9E6916F0080609D029
:101EF00000F0CCFBA0EB0A03FA2BF4D9002686F302
:101F00001188ADE79A6942F001029A6100F0BEFBC8
:101F10008246E36B9A69D00706D400F0B7FBA0EBCA
:101F20000A03FA2BF5D9E9E79A6942F002029A61AD
:101F3000E36B4FF0000AC3F854A08AF31188686D70
:101F4000FFF792FB202200216846FFF78BF802A8DA
:101F5000FFF710FE04F58353CDF818A06A4633440A
:101F60000DF1180E9446BCE80300F4451860596062
:101F7000624603F10803F5D1DCF800001860203652
:101F80009CF804201A71B6F5806FDBD1002304F5AC
:101F9000A35285F8603485F863340A3249462046F6
:101FA000FFF7ACFE064690B9E26B936923F001039C
:101FB000936100F06BFB0546E36B9B69D9077FF5E6
:101FC0004EAF00F063FB431BFA2BF5D947E795F8BA
:101FD0006E34C5F87C94591E95F86F34E26B013B62
:101FE0001B0243EA416395F8701401390B43B5F8BD
:101FF0006C14013943EA0143D361B8F1000F36D0C4
:1020000004F5A352123241462046FFF7DFFE90B995
:10201000E26B936923F00103936100F037FB0546FF
:10202000E36B9B69DA077FF51AAF00F02FFB431BC8
:10203000FA2BF5D913E795F87724C5F88084511E5B
:1020400095F87824E36B013A120142EA012295F8EF
:10205000761401390A43B5F87414013942EA014291
:1020600042F40002DA60E36B4FF420629A64204687
:10207000FFF7CCFE002385F86934E36B6FF0404234
:102080001A65E36B154A5A65E36B44229A65E36B64
:102090000722C3F8DC20E36B03229742DA653FF4A2
:1020A000DFAEE26B936923F00103936100F0EEFA77
:1020B0000746E36B9B69DB0705D500F0E7FAC31B16
:1020C000FA2BF6D9CBE6012385F86234C8E600BFC7
:1020D000384E00203C4E0020001002409B000800BB
:1020E0002DE9F04F00F5A5578BB00546904699466F
:1020F0004FF0000B41F2780A1037EB6BD3F8D43075
:1021000023FA0BF3DC0753D505EB4B1151444FEA8F
:102110004B120B7918074BD405F58056D6F894343A
:102120000133C6F89434C7E900890B79990648BF92
:10213000D6F8C43405EB020148BF0133514448BF0F
:10214000C6F8C4340B7943F008030B71DB0724D5C0
:1021500096F863340BB302A8019205F58354FFF798
:102160000FFD019A0834144405AB04F1080C2068F3
:1021700061681A4603C2083464451346F7D12068E3
:102180001060A2889A800123ADF810302B68CDE949
:1021900002891B6C02A928469847D6F8B834D6F8AD
:1021A00064040133C6F8B83410B103681B6998475A
:1021B0000BF1010BBBF1200F9FD10BB0BDE8F08FED
:1021C0002DE9F04F8DB004460F4600F061FA8246CB
:1021D0008946002F56D1E36BD3F89020920141BF7E
:1021E00004F58051D1F8A8240132C1F8A824D3F80D
:1021F0009020160703D100200DB0BDE8F08FD3F872
:102200009050E66AC5F30125482303FB0566E846BE
:102210004046FFF7AFFC326851004ABF22F06043EE
:10222000C2F38A4343F00043920048BF43F0804327
:102230000093736813F400131FBF04F58052012349
:102240008DF80D30D2F8C8340EBF8DF80D30013343
:10225000C2F8C834F38803F00F038DF80C304FF048
:10226000000B9DF80C0000F0ADFA5FFA8BF398427A
:1022700020D9F2180CA90B44127A03F82C2C0BF17C
:10228000010BEEE7012FB6D1E36BD3F8982095014F
:1022900041BF04F58051D1F8A8240132C1F8A82427
:1022A000D3F898201007A6D0D3F89850266BC5F322
:1022B0000125A9E7EFB9E36BC3F8945004A8FFF731
:1022C0005FFC98E80F0007AD07C52B800023ADF831
:1022D000183023682046CDE904A91B6C04A998474F
:1022E00004F5805458B1D4F8A0340133C4F8A034B4
:1022F00082E7012F04BFE36BC3F89C50DEE7D4F8FC
:10230000A4340133C4F8A434012075E72DE9F04169
:1023100005460F4600F58054012639462846FFF74A
:102320004FFF10B184F86364F7E7D4F8B834D4F8F9
:1023300064040133C4F8B83420B10368BDE8F04147
:102340001B691847BDE8F081F0B5C36B1A6C12F435
:102350007F0F2BD000F580541B6CC4F8BC3441F2C5
:102360007805002347194FF0010C00EB43122A4473
:102370005E01117911F0020F15D0490713D4B95934
:10238000C66BD6F8C8E00CFA01F111EA0E0F0AD0BC
:10239000C6F8D010117941F004011171D4F89C24D1
:1023A0000132C4F89C240133202BDED1F0BD0000A3
:1023B00010B5254C254B226802B338B31A6D1206AE
:1023C0000ED580221A6500F063F950EA01020B462F
:1023D00002D0013861F1000302462068FFF780FE59
:1023E0001A4A136D1B032AD523684FF4002103F505
:1023F00080531165012283F8692420E001221A65C7
:1024000008221A654FF480621A6510BD196DC8075D
:1024100002D4196D890705D50321196510460021DD
:10242000FFF774FF094B1A6D100702D41A6DD1061D
:1024300005D518221A6520680121FFF767FF20687B
:10244000BDE81040FFF780BF384E00200064004018
:1024500008B5302383F31188FFF776FF002383F359
:10246000118808BDC36BD3F8C40080F40010C0F31A
:102470004050704708B5302383F3118800F5805031
:10248000406DFFF703F9002383F3118843090CBF64
:102490000120002008BD000000F5805393F8692456
:1024A00062B1C16B8A6922F001028A61D3F8AC245F
:1024B0000132C3F8AC24002283F86924704700007D
:1024C0002DE9F743302181F31188002500F5835170
:1024D00041F2780E4FF0010800F5805C00EB4514E6
:1024E0007444267977071CD4F6061AD5D0F83C90A8
:1024F0008E69D9F8C87008FA06F63E4211D04F68C6
:1025000001970F689742019F9F410AD2C9F8D06096
:10251000267946F004062671DCF898440134CCF89C
:1025200098440135202D01F12001D7D1002383F3F8
:10253000118803B0BDE8F083F8B51E460023137080
:102540000F4605461446FFF795FF80F001003870EE
:102550001EB12846FFF786FF2070F8BD2DE9F04F29
:1025600085B09946DDE90EA30D46029313780193D9
:1025700091F800B08046164600F08AF82B780446A1
:102580000F4613B93378002B41D022463B464046D4
:10259000FFF796FFFFF75CFFFFF77EFF4B463246E3
:1025A0002946FFF7C9FF2B7833B1BBF1000F03D0E9
:1025B000012005B0BDE8F08F337813B1019B002BEB
:1025C000F6D108F580530393029B544577EB030340
:1025D0001DD2039BD3F86404C8B10368AAEB0401BD
:1025E0001B6898474B46324629464046FFF7A4FFF2
:1025F0002B7813B1BBF1000FDAD1337813B1019B03
:10260000002BD5D100F044F804460F46DCE700204B
:10261000CFE7000008B50020FFF7CAFEBDE808407C
:1026200001F0A4B808B50120FFF7C2FEBDE80840DC
:1026300001F09CB800B59BB0EFF3098168226846B1
:10264000FEF7FEFCEFF30583014B9B6BFEE700BF3B
:1026500000ED00E008B5FFF7EDFF000000B59BB00E
:10266000EFF3098168226846FEF7EAFCEFF3058381
:10267000014B5B6BFEE700BF00ED00E0FEE70000F2
:102680000FB408B5029801F079FBFEE701F05ABEDD
:1026900001F03CBE0139C9B202299EBF00EBC10066
:1026A0000023C0E901337047F8B51B885B07054676
:1026B0000E4615D4044600F11807BC4210D06368DA
:1026C00053B12B682846DB6B9847A368C1B23246EA
:1026D000606898470834F0E7A368002BF1D1F9E768
:1026E0000120F8BD73B56C4684E80600014600225F
:1026F0004E68D5B26EB98E685EB900EBC200021D9D
:1027000094E80300013582E803001D70012002B047
:1027100070BD0132032A01F10801E9D10020F6E77A
:102720002DE9F04F89B00446BDF848700E460546C5
:1027300000F118084FF0000907F004074FF0000AF5
:102740004FF0000BA84538D06B680BB9AB684BB1A4
:1027500057B923682046DB6B9847AB68C1B2324655
:10276000686898470835EDE7B9F1000FFAD1CDE96F
:1027700000ABADF80890334603AA06F1080E1868BE
:1027800059689446ACE80300083373456246F6D1B5
:102790001868CCF800009B88ACF80430FFF778FF8D
:1027A0000423ADF808302368CDE900011B6C6946AD
:1027B000204698474FF00109D4E7012009B0BDE851
:1027C000F08F0000082817D909280CD00A280CD04F
:1027D0000B280CD00C280CD00D280CD00E2814BFC0
:1027E0004020302070470C20704710207047142084
:1027F0007047182070472020704700002DE9F041F5
:10280000456A15B94162BDE8F0814B6823F0604725
:10281000C3F38A464FEAD37EC3F3807816EA2306D1
:1028200038BF3E46AC462B465A68BEEBD27F22F0FC
:1028300060440AD0002A18DAA40CB44217D19D4291
:102840000FD10D60DEE71346EEE7A74207D102F095
:102850008044C2F3807242450BD054B1EFE708D2F6
:10286000EDE7CCF800100B60CDE7B44201D0B442E4
:10287000E5D81A689C46002AE5D11960C3E7000034
:102880002DE9F047089D01F007044FEAD5082244DE
:1028900005F0070500EBD1004FF47F49944201D1C8
:1028A000BDE8F08704F0070705F0070A57453E46E4
:1028B00038BF5646C6F10806111B8E4228BF0E4689
:1028C000E10808EBD50E415C13F80EC0B94029FAB7
:1028D00006F721FA0AF1FFB28CEA010147FA0AF77A
:1028E00039408CEA010C03F80EC034443544D5E776
:1028F00080EA0120082341F2210201B240000029B0
:1029000080B203F1FF33B8BF504013F0FF03F4D19E
:102910007047000038B50C468D18A54200D138BD6F
:1029200014F8011BFFF7E4FFF7E7000042684AB123
:10293000136843604389818901339BB29942438183
:1029400038BF83811046704770B588B02022044696
:102950000D4668460021FEF785FB20460495FFF7EB
:10296000E5FF024658B16B46054608AE1C4603CC4F
:10297000B44228606960234605F10805F6D1104687
:1029800008B070BD082817D909280CD00A280CD027
:102990000B280CD00C280CD00D280CD00E2814BFFE
:1029A0004020302070470C207047102070471420C2
:1029B000704718207047202070470000082817D95A
:1029C0000C280CD910280CD914280CD918280CD98B
:1029D00020280CD930288CBF0F200E2070470920EA
:1029E00070470A2070470B2070470C2070470D205D
:1029F000704700002DE9F843078C072F04461ED9C5
:102A0000D0E9029800254FF6FF73C5F12006A5F125
:102A1000200029FA05F108FA06F628FA00F03143F9
:102A20000143C9B21846FFF763FF0835402D03463E
:102A3000EBD1E1693A46BDE8F843FFF76BBF4FF6CB
:102A4000FF70BDE8F883000010B54B6823B9CA8A4F
:102A500063F30902CA8210BD04691A681C6003612D
:102A6000C38A013BC3824A60EFE700002DE9F84FBB
:102A70001D46CB8A0F46C3F30901052981469246BC
:102A80000B4630D00020AAB207F11A049EB2042EE1
:102A90001FFA80F80FD8904503F1010306D3FB8A93
:102AA0000A4462F30903FB8201201AE01AF800606D
:102AB000E6540130EAE79045F1D2A1F1050B1C2361
:102AC0007C68BBFBF3F203FB12BB1FFA8BF6002CF6
:102AD00045D14846FFF72AFF044638B978606FF0C1
:102AE0000200BDE8F88F4FF00008E6E70026066018
:102AF0007860ADB24FF0000B454510D90AEB0803E2
:102B0000221D13F8011B9155B1B208F101081B29D0
:102B10001FFA88F82BD0454506F10106F1D8FB8A4B
:102B2000C3F30902154465F30903BCE7013292B20D
:102B30001C462368002BF9D16B1F0B441C21B3FBEF
:102B4000F1F301339BB29A42D3D2BBF1000FD0D143
:102B50004846FFF7EBFE20B9C4F800B0BFE70122FA
:102B6000E7E7C0F800B05E4620600446C1E745458F
:102B7000D5D94846FFF7DAFE08B92060AFE7C0F8BC
:102B800000B0002620600446B6E700002DE9F04FB3
:102B90002DED028B1C4683B05B6901920746884687
:102BA000002B00F0A780238C2BB1E269002A00F0F3
:102BB000A180072B35D807F10C00FFF7B7FE0546BB
:102BC00038B96FF00205284603B0BDEC028BBDE8B2
:102BD000F08F14220021FEF745FA228CE16905F1FD
:102BE0000800FEF72DFA208C013080B2FFF7E6FED8
:102BF000FFF7C8FE013880B2208401302874636971
:102C0000228C1B782A4403F01F0363F03F0348F033
:102C100000411372384669602946FFF7EFFD012530
:102C2000D1E702339BB20722C18A0633B3FBF2F32A
:102C3000828A521A9BB292B29342C2D800F10C031C
:102C40004FF0000908EE103A4FF0800A4E464D460C
:102C500018EE100AFFF76AFE83460028B1D014224E
:102C60000021FEF7FFF9002E3AD1019BABF80830A6
:102C700002220BF1080E1FFA82FC0CF10100BCF1DC
:102C8000060F218C80B201D88E422BD3FFF796FE1F
:102C9000FFF778FE62691278013802F01F028E4257
:102CA00008BF4FF0400A42EA49121BFA80F14AEA93
:102CB000020A013048F0004281F808A08BF81000A9
:102CC000CBF8042059463846FFF798FD238C013590
:102CD000B3422DB289F001094FF0000AB8D172E772
:102CE0000022C6E7E169895D0EF802100136B6B22E
:102CF0000132C0E76FF0010565E70000F8B5154641
:102D00000E463022002104461F46FEF7ABF9069B13
:102D10006360B5F5001F079BA76034BF6A094FF6D3
:102D2000FF72A36297B2E66104F1100000239A4299
:102D300006D800230360A782E3822383E360F8BD03
:102D40000660013330462036F1E7000003781BB9F6
:102D50004BB2002BC8BF017070470000007870476D
:102D6000F8B50C46C969074611B9238C002B37D139
:102D7000257E1F2D34D8387828BB228C072A2CD8E2
:102D8000268A36F003032BD14FF6FF70FFF7C2FD02
:102D900020F001003102400441EA0561400C41EAA3
:102DA00040254FF6FF72234629463846FFF7EEFED0
:102DB000002807DD626913780133DBB21F2B88BF5F
:102DC00000231370F8BD218A2D0645EA012505432D
:102DD0002046FFF70FFE0246E5E76FF00300F1E73C
:102DE0006FF00100EEE7000070B58AB004461646A9
:102DF0000021282268461D46FEF734F9BDF8383018
:102E0000ADF810300F9B05939DF840308DF81830C9
:102E1000119B07936946BDF84830ADF82030204635
:102E2000CDE90265FFF79CFF0AB070BD2DE9F041C6
:102E3000D36905460C4616460BB9138C5BBB377E2F
:102E40001F2F28D895F80080B8F1000F26D0304603
:102E5000FFF7D0FD3378210241EAC33141EA08018E
:102E6000338A41EA076141EA03410246334641F0B1
:102E700080012846FFF78AFE00280ADD3378012BFF
:102E800007D1726913780133DBB21F2B88BF00238F
:102E90001370BDE8F0816FF00100FAE76FF00300F6
:102EA000F7E70000F0B58BB004460D461746002149
:102EB000282268461E46FEF7D5F89DF84C305A1E6B
:102EC000534253418DF800309DF84030ADF810303A
:102ED000119B05939DF848308DF81830149B07938B
:102EE0006A46BDF85430ADF8203029462046CDE979
:102EF0000276FFF79BFF0BB0F0BD0000406A00B107
:102F000004307047436A1A68426202691A600361BA
:102F1000C38A013BC38270472DE9F041D0F820807D
:102F2000194E14461D464146002709B9BDE8F081F7
:102F3000D1E90223A21A65EB0303964277EB030360
:102F40001ED2036A8B420DD1FFF77EFD036A1B6818
:102F5000036203690B60C38A0161016A013BC3829A
:102F60008846E2E7FFF770FD0B68C8F80030036998
:102F70000B60C38A0161013BC382D8F80010D4E71B
:102F800088460968D1E700BF80841E002DE9F04F14
:102F90008BB00D46DDF8509014469B4680460028C5
:102FA00000F01981B9F1000F00F01581531E3F2B7D
:102FB00000F21181012A03D1BBF1000F40F00B8117
:102FC0000023CDE90833B8F81430B5EBC30F4FEA4E
:102FD000C30703D300200BB0BDE8F08F2B199F422D
:102FE000D8F80C303ABF7F1BFFB227461BB9D8F880
:102FF0001030002B7AD0272D4ED8C5F12806B742C5
:103000004FF000032CBFF6B23E4600932946D8F895
:10301000080008AB3246FFF733FCA7EB060A35443D
:103020005FFA8AFAB8F8143003F10053053BDB006D
:103030000493D8F80C3003932821039B13B1BAF101
:10304000000F2CD1D8F8100040B1BAF1000F05D014
:10305000009608AB5246691AFFF712FC38B2002FEF
:10306000B8D066070AD00AAB03EBD401624211F86C
:10307000083C02F00702134101F8083C082C3CD937
:10308000102C40F2B580202C40F2B780BBF1000F2D
:1030900000F09C80082334E0BA460026C2E7049B77
:1030A000E02B28BFE02306930B44AB42059314D9D1
:1030B0005A1B03980096924534BF5246D2B2691A01
:1030C00008AB04300792FFF7DBFB079A1644AAEB24
:1030D000020A1544F6B25FFA8AFA049B069A059929
:1030E0009B1A0493039B1B680393A6E70093D8F8ED
:1030F000080008AB3A462946AEE7BBF1000F13D0F3
:103100000123B4EBC30F6CD0082C12D89DF82030EB
:10311000621E23FA02F2D50706D54FF0FF3202FAFB
:1031200004F423438DF820309DF8203089F80030D6
:1031300051E7102C12D8BDF82030621E23FA02F29B
:10314000D10706D54FF0FF3202FA04F42343ADF85D
:103150002030BDF82030A9F800303CE7202C0FD8F3
:103160000899631E21FA03F3DA0705D54FF0FF3201
:1031700002FA04F40C430894089BC9F800302AE7CB
:10318000402C2BD0DDE90865611EC4F12102A4F1B9
:10319000210326FA01F105FA02F225FA03F311439D
:1031A0001943CB0712D50122A4F12003C4F1200159
:1031B00002FA03F322FA01F1A240524243EA010368
:1031C00063EB430332432B43CDE90823DDE90823B6
:1031D000C9E90023FFE66FF00100FCE66FF008008C
:1031E000F9E6082CA0D9102CB3D9202CEED8C3E7CF
:1031F000BBF1000FADD0022383E7BBF1000FBBD0C2
:1032000004237EE730B5012A144638BF0124402C40
:1032100085B028BF40240025012ACDE9025518D8E1
:103220001B788DF8083063070AD004AB03EBD40594
:10323000624215F8083C02F00702934005F8083C8A
:10324000009103462246002102A8FFF719FB05B0B2
:1032500030BD082AE4D9102A03D81B88ADF80830FD
:10326000E1E7202A8DBFD3E900231B680293CDE953
:103270000223D8E710B5CB681BB98B600B618B823A
:1032800010BD04691A681C600361C38A013BC382D4
:10329000CA60F0E703064CBFC0F3C030022070479D
:1032A00008B50246FFF7F6FF022806D15306C2F31F
:1032B0000F2001D100F0030008BDC2F30740FBE777
:1032C0002DE9F04F93B0CDE903230A680446104678
:1032D000FFF7E0FF022814BFC2F306260026002AEB
:1032E0000D46824680F2F78112F0C04940F0F3812A
:1032F000097B002900F0EF81022803D02378B34234
:1033000040F0EC81C2F304630693104602F07F03A1
:103310000593FFF7C5FF059B29444FEA834848EA18
:103320000A4848EA4668CE7800230022CDE90823FF
:10333000F309834648EA0008029367D0059B00938F
:1033400002466768534608A92046B847002800F09F
:10335000C881276A4FB9414604F10C00FFF7F4FA1F
:10336000074690B96FF0020054E03B6998450DD0D4
:103370003F68002FF9D1414604F10C00FFF7E4FA51
:1033800007460028EED0236A3B60276297F817C0F3
:1033900006F01F08CCF3840CACEB08001FFA80FE8B
:1033A0000028B8BF0EF12000A8EB0C031FFA83FE23
:1033B000D7E90221B8BF00B2002B0793BEBF0EF1C0
:1033C00020031BB2079352EA010338D0039BDFF8B6
:1033D00024E39A1A049B4FF0000C63EB010196451D
:1033E0007CEB01032BD36B7B97F81AE0734519D163
:1033F000029B002B78D0012821DC7868F8B9DFF82F
:10340000F0C2944570EB010316D337E0276A27B961
:103410006FF00C0013B0BDE8F08F3B699845B5D054
:103420003F68F4E7B24890427CEB010301D30020EF
:10343000F0E7029B002BFAD0079B0F2B17DCFA7DDD
:10344000B30002F0030203F07C031343FB7539461B
:103450002046FFF7F9FA6B7BBB76029B3BB9FB7DFD
:10346000C3F38402013262F38603FB75D0E76A7B03
:10347000BB7E9A42DBD1029B002B35D0B309022BD5
:1034800032D0039BBB60049BFB60142200210DA87B
:10349000FDF7E8FD039B0A93049B0B932B1D0C93F4
:1034A0002B7BADF83EB0013BDBB2ADF83C30069B68
:1034B0008DF84230059B8DF8433094F82C308DF810
:1034C00040A083F001038DF844308DF84180A3685B
:1034D0000AA920469847FB7DC3F38403013303F018
:1034E0001F039B02FB82A2E7FB7DC6F34012B2EBF7
:1034F000D31F40F0F980C3F38403434540F0FC80C0
:10350000029A2B7BB609002A52D016F0010661D12F
:10351000032B40F2F480039BBB60049BFB60FB8A9F
:1035200066F30903FB822B7BAE1D033BDBB2324605
:10353000394604F10C00FFF799FA00280CDA3946F5
:103540002046FFF781FAFB7DC3F38403013303F0C8
:103550001F039B02FB8205E7DDE90884AB883B8300
:103560004FF6FF73C9F12000A9F1200228FA09F1F2
:1035700004FA00F0014324FA02F211431846C9B2DA
:10358000FFF7B6F909F10809B9F1400F0346E9D18F
:10359000B8822A7B033AD2B23146FFF7BBF9FB7DF2
:1035A000B882DA43C2F3C01262F3C713FB753EE779
:1035B00086B92E1D013BDBB23246394604F10C00C0
:1035C000FFF754FA0028BADB2A7BB88A013AD2B254
:1035D0003146E2E7F98AC1F30901013B0429DAB275
:1035E0005BD8281D002307F11B069A4208D910F862
:1035F00001CB06F801C0013101330529DBB2F4D15A
:1036000003990A9104990B91934207F11B010C91C4
:1036100038BF043379680D9134BF55FA83F3002322
:103620000E93FB8AADF83EB0C3F309031A44069B20
:103630008DF84230059B8DF8433094F82C30ADF86E
:103640003C2083F001038DF8443000238DF840A026
:103650008DF841807B602A7BB88A013A291DFFF7EB
:1036600059F93B8BB882834203D1A3680AA920464B
:10367000984720460AA9FFF7FDFDFB7DBA8AC3F3F0
:103680008403013303F01F039B02FB823B8B9A42AE
:103690000CBF00206FF01000BCE67B68002BAFD0A1
:1036A000052001E01C3033461E68002EFAD1091AAD
:1036B000081D2E1D184401EB090CBCF11B0F5FFA0D
:1036C00089F39DD89A429BD916F8013B00F8013B3B
:1036D00009F10109EFE76FF009009BE66FF00A00BE
:1036E00098E66FF00B0095E66FF00D0092E600BFD4
:1036F00040420F0080841E006FF00E008AE66FF0DB
:103700000F0087E6EFF3098305494A6B22F00102B7
:103710004A63683383F30988002383F31188704771
:1037200000EF00E0302080F3118862B60C4B0D4AA8
:10373000D96821F4E0610904090C0A43DA60D3F87E
:10374000FC20094942F08072C3F8FC200A6842F06C
:1037500001020A602022DA7783F82200704700BF56
:1037600000ED00E00003FA05001000E010B5302382
:1037700083F311880E4B5B6813F4006314D0F1EEF1
:10378000103AEFF30984683C4FF08073E361094B12
:10379000DB6B236684F3098800F0BAFA10B1064B9C
:1037A000A36110BD054BFBE783F31188F9E700BF68
:1037B00000ED00E000EF00E03F03000842030008D6
:1037C000434B4FF4007270B51A605A6912F4C06F1F
:1037D000FBD1404B9A6802F00C02042A20D01A68F0
:1037E00042F480721A601A685205FCD501229A6070
:1037F0009A6802F00C02042AFAD13749374A0A6063
:103800000A6812F00F02FBD1C3F8982063221A60F5
:103810001A689603FCD42E4A4FF48071C2F88010C7
:10382000C468E50306D51A6842F480321A601A6843
:103830009103FCD5C269D20709D5D3F8982042F08C
:103840000102C3F89820D3F898209607FBD5426967
:10385000DA6044F480721A6004F0807111B11A6861
:103860009501FBD5996802691B4E22F0030501F012
:10387000030129439960856935603168694009070A
:10388000FBD1134905680D6046684E608068C1F839
:1038900080006E0417D448698505FCD4996802F04D
:1038A000030021F00301014399609200996851409F
:1038B00011F00C0FFAD1E2055EBF1A6822F4807293
:1038C0001A60002070BD48698005FCD5E6E700BF9E
:1038D000007000400010024000200240000604007A
:1038E00008B500F083F9BDE8084000F05BB90000BE
:1038F00010B5394C3948A36A4FF0FF32A262A36A6F
:103900000023A362A16AE16A61F07F01E162E16ADA
:1039100001F07F01E162E16A216B2263216B236385
:10392000216BA16BA263A16BA363A16BE16BE2634B
:10393000E16BE363E16B216C2264226C2364226CF3
:10394000226E42F001022266D4F8802022F00102A9
:10395000C4F88020D4F88020A26D42F08052A26585
:10396000A26F22F08052A267A26F1D4A4FF400415D
:103970009160D360136253629362D36213635363A3
:103980009363D363136453649364D364136553657F
:10399000116841F480711160D4F8902012F4407FD6
:1039A0001EBF4FF48032C4F89020C4F890300D4A06
:1039B0000023A360C4F88820C4F89C30FFF700FF00
:1039C00010B1094800F0DAF9D4F8903023F003235D
:1039D000C4F8903010BD00BF00100240AC48000891
:1039E0000070004055010051A4480008014B53F8F5
:1039F0002000704718230020074A08B5536903F0D8
:103A00000103536123B1054A13680BB1506898470D
:103A1000BDE80840FFF7AABE000401409450002012
:103A2000074A08B5536903F00203536123B1054AFD
:103A300093680BB1D0689847BDE80840FFF796BE81
:103A40000004014094500020074A08B5536903F070
:103A50000403536123B1054A13690BB150699847B8
:103A6000BDE80840FFF782BE0004014094500020EA
:103A7000074A08B5536903F00803536123B1054AA7
:103A800093690BB1D0699847BDE80840FFF76EBE57
:103A90000004014094500020074A08B5536903F020
:103AA0001003536123B1054A136A0BB1506A98475A
:103AB000BDE80840FFF75ABE0004014094500020C2
:103AC000164B10B55C6904F478725A61A30604D5EC
:103AD000134A936A0BB1D06A9847600604D5104A1E
:103AE000136B0BB1506B9847210604D50C4A936BAE
:103AF0000BB1D06B9847E20504D5094A136C0BB1A2
:103B0000506C9847A30504D5054A936C0BB1D06C53
:103B10009847BDE81040FFF729BE00BF00040140F0
:103B200094500020194B10B55C6904F47C425A6132
:103B3000620504D5164A136D0BB1506D98472305E5
:103B400004D5134A936D0BB1D06D9847E00404D5AA
:103B50000F4A136E0BB1506E9847A10404D50C4A5E
:103B6000936E0BB1D06E9847620404D5084A136F68
:103B70000BB1506F9847230404D5054A936F0BB1DE
:103B8000D06F9847BDE81040FFF7F0BD000401403A
:103B90009450002008B500F0F3FCBDE80840FFF7A2
:103BA000E5BD0000062108B5084600F033F80621FF
:103BB000072000F02FF80621082000F02BF806213E
:103BC000092000F027F806210A2000F023F806213A
:103BD000172000F01FF80621282000F01BF8BDE890
:103BE000084007211C2000F015B800004FF0E0232A
:103BF000002258684FF0FF31930003F1604303F552
:103C0000614301329042C3F88010C3F88011F3D2AF
:103C10007047000000F1604303F561430901C9B238
:103C200083F80013012200F01F039A4043099B0010
:103C300003F1604303F56143C3F880211A607047C4
:103C400000230375826803691B6899689142FBD25F
:103C50005A68036042601060586070470023037523
:103C6000826803691B6899689142FBD85A680360AF
:103C7000426010605860704708B50846302383F3EF
:103C800011880B7D032B05D0042B0DD02BB983F3AA
:103C9000118808BD8B6900221A604FF0FF338361E1
:103CA000FFF7CEFF0023F2E7D1E9003213605A603C
:103CB000F3E70000FFF7C4BF054BD9680875186823
:103CC00002681A60536001220275D860FCF722BBBB
:103CD000484E002030B50C4BDD684B1C87B00446C5
:103CE0000FD02B46094A684600F02AF92046FFF714
:103CF000E3FF009B13B1684600F02CF9A86907B0F8
:103D000030BDFFF7D9FFF9E7484E0020793C0008A5
:103D1000044B1A68DB6890689B68984294BF002047
:103D200001207047484E0020084B10B51C68D86829
:103D300022681A60536001222275DC60FFF78EFF53
:103D400001462046BDE81040FCF7E4BA484E00208A
:103D500038B5074C074908480123002523706560E2
:103D600000F03CFC0223237085F3118838BD00BFAE
:103D700070500020D0480008484E002008B572B6A8
:103D8000044B186500F0ACFA00F05CFB024B032218
:103D90001A70FEE7484E00207050002000F010B965
:103DA0008B60022308618B82084670478368A3F109
:103DB000840243F8142C026943F8442C426943F806
:103DC000402C094A43F8242CC26843F8182C0222DC
:103DD00003F80C2C002203F80B2C044A43F8102C97
:103DE000A3F12000704700BF2D030008484E0020BB
:103DF00008B5FFF7DBFFBDE80840FFF75BBF000039
:103E0000024BDB6898610F20FFF756BF484E002039
:103E1000302383F31188FFF7F3BF000008B5014694
:103E2000302383F311880820FFF754FF002383F326
:103E3000118808BD10B503689C68A2420CD85C6864
:103E40008A600B604C602160596099688A1A9A6098
:103E50004FF0FF33836010BD1B68121BECE70000BE
:103E60000A2938BF0A2170B504460D460A26601992
:103E700000F0AEFB00F09AFB041BA54203D8751CB2
:103E80002E460446F3E70A2E04D9BDE8704001200F
:103E900000F0E4BB70BD0000F8B5144B0D46D961CD
:103EA00003F1100141600A2A1969826038BF0A22B1
:103EB000016048601861A818144600F07BFB0A27CF
:103EC00000F074FB431BA342064606D37C1C281952
:103ED00000F07EFB27463546F2E70A2F04D9BDE8FD
:103EE000F840012000F0BABBF8BD00BF484E0020EA
:103EF000F8B506460D4600F059FB0F4A134653F835
:103F0000107F9F4206D12A4601463046BDE8F84060
:103F1000FFF7C2BFD169BB68441A2C1928BF2C46D1
:103F2000A34202D92946FFF79BFF224631460348A8
:103F3000BDE8F840FFF77EBF484E0020584E0020F5
:103F400010B4C0E9032300235DF8044B4361FFF77D
:103F5000CFBF000010B5194C236998420DD0D0E9AD
:103F60000032816813605A609A680A449A6000239C
:103F700003604FF0FF33A36110BD2346026843F88E
:103F8000102F53600022026022699A4203D1BDE8DB
:103F9000104000F017BB936881680B44936000F0F9
:103FA00005FB2269E1699268441AA242E4D91144EE
:103FB000BDE81040091AFFF753BF00BF484E00206C
:103FC0002DE9F047DFF8BC8008F110072C4ED8F837
:103FD000105000F0EBFAD8F81C40AA68031B9A4274
:103FE0003ED81444D5E900324FF00009C8F81C400F
:103FF00013605A60C5F80090D8F81030B34201D170
:1040000000F0E0FA89F31188D5E903312846984792
:10401000302383F311886B69002BD8D000F0C6FAE7
:104020006A69A0EB04094A4582460DD2022000F0DD
:1040300015FB0022D8F81030B34208D1514628466B
:10404000BDE8F047FFF728BF121A2244F2E712EB4F
:10405000090938BF4A4629463846FFF7EBFEB5E75F
:10406000D8F81030B34208D01444211AC8F81C0004
:10407000A960BDE8F047FFF7F3BEBDE8F08700BFD9
:10408000584E0020484E002038B500F08FFA054AFF
:10409000D2E90845031B181945F10001C2E90801DE
:1040A00038BD00BF484E002000207047FEE70000EA
:1040B000704700004FF0FF3070470000BFF34F8F94
:1040C000024A1369DB03FCD4704700BF00200240A2
:1040D00008B5094B1B7873B9FFF7F0FF074B5A6916
:1040E000002ABFBF064A9A6002F188329A601A68B5
:1040F00022F480621A6008BD88500020002002402F
:104100002301674508B50B4B1B7893B9FFF7D6FF22
:10411000094B5A6942F000425A611A6842F48052CF
:104120001A601A6822F480521A601A6842F4806297
:104130001A6008BD88500020002002407F289ABFE6
:1041400000F58030C0020020704700004FF400608E
:1041500070470000802070477F2808B50BD8FFF714
:10416000EDFF00F500630268013204D104308342A0
:10417000F9D1012008BD0020FCE700007F2810B520
:1041800004461FD8FFF79AFFFFF7A2FF0E4BF3225A
:104190001A6102225A615A6942EAC0025A615A6996
:1041A00042F480325A61FFF789FF4FF40061FFF754
:1041B000C5FF00F043F9FFF7A5FF2046BDE810401A
:1041C000FFF7CABF002010BD002002402DE9F843D0
:1041D00040EA020313F00703144606D0304B40F2C6
:1041E00082321A600020BDE8F88385182D4A954276
:1041F0000CD92B4A40F287311160F3E7031D1B688D
:104200004A68934208D1083C08300831072C14D979
:1042100002680B689A42F1D0FFF75AFFFFF74EFF92
:10422000214E08314FF001084FF00009012CA1F197
:10423000080706D8FFF766FF01E0002CECD101204B
:10424000D1E7C6F81480054651F8083C45F8043B10
:1042500051F8043C4360FFF731FF336943F0010339
:104260003361C6F81490026851F8083C9A420CD0A9
:104270000B4B40F2AF321A600C4B18600C4B1C60B9
:104280000C4B1F60FFF73EFFACE72D6851F8043C74
:104290009D4201F10801EBD1083C0830C6E700BFA0
:1042A00084500020000004080020024078500020C4
:1042B000805000207C500020084908B50B7828B1B8
:1042C0001BB9FFF705FF01230B7008BD002BFCD0C5
:1042D000BDE808400870FFF715BF00BF88500020F8
:1042E00008B50649064800F0ABF8BDE808404FF4B1
:1042F00080414FF0805000F0A3B800BF007F010064
:1043000000010020084600F033BA000038B5EFF392
:1043100011859DB9EFF30584C4F30804302334B14B
:1043200083F31188FFF7B0FE85F3118838BD83F35E
:104330001188FFF7A9FE84F3118838BDBDE8384025
:10434000FFF7A2BE38B5FFF7E1FF114C114AC008D4
:1043500040EA4170A0FB025EC908A0FB040C1CEB04
:10436000050CA1FB04404FF000035B41A1FB0212CE
:104370001CEB040C43EB000011EB0E0142F10002B8
:10438000411842F10000090941EA007038BD00BF40
:10439000CFF753E3A59BC4200244D2B2904200D190
:1043A0007047431C800000F1804000F51450006805
:1043B00041F8040BD8B2F1E7124B10B5D3F8904096
:1043C000240409D4D3F89040C3F89040D3F8904027
:1043D00044F40044C3F890400B4C2368024443F477
:1043E00080732360D2B2904200D110BD431C800084
:1043F00000F1804000F5145051F8044B0460D8B22D
:10440000F1E700BF001002400070004007B5012234
:1044100001A90020FFF7C0FF019803B05DF804FB7D
:1044200013B50446FFF7F2FFA04205D0012201A90F
:1044300000200194FFF7C0FF02B010BD70470000DC
:104440007047000070470000074B45F255521A6054
:1044500003225A6040F2FF729A604CF6CC421A6016
:10446000024B01221A70704700300040905000202B
:10447000034B1B781BB1034B4AF6AA221A60704704
:104480009050002000300040054B1A6832B902F10C
:10449000804202F50432D2F894201A60704700BFBF
:1044A0008C500020024B4FF40002C3F89420704758
:1044B0000010024008B5FFF7E7FF024B1868C0F391
:1044C000407008BD8C50002070470000FEE70000DF
:1044D0000A4B0B480B4A90420BD30B4BDA1C121AB7
:1044E000C11E22F003028B4238BF00220021FCF7DC
:1044F000B9BD53F8041B40F8041BECE7544A00080C
:104500001451002014510020145100200023054AAA
:1045100019460133102BC2E9001102F10802F8D14B
:10452000704700BF9450002008B5124B9A6D42F0BE
:1045300001029A659A6F42F001029A670E4A9B6FD8
:10454000936843F0010393600620FFF74FFA0B4B8B
:10455000B0FBF3F04FF080434FF0FF320138986228
:10456000DA6200229A615A63DA605A6001225A6163
:104570001A6008BD00100240002004E040420F0015
:104580004FF0804208B51169D3680B40D9B2C943D6
:104590009B07116107D5302383F31188FFF7FEFBDA
:1045A000002383F3118808BDFFF7BEBF4FF080439F
:1045B000586A70474FF08043002258631A61022204
:1045C000DA6070474FF080430022DA6070470000E5
:1045D0004FF0804358637047FEE7000070B51B4BF7
:1045E00001630025044686B0586085620E46FFF7D9
:1045F00099F804F11003C4E904334FF0FF33C4E920
:104600000635C4E90044A560E562FFF7CFFF2B46FD
:104610000246C4E9082304F134010D4A25658023CC
:104620002046FFF7BDFB0123E0600A4A03750092B4
:1046300072680192B268CDE90223074B6846CDE962
:104640000435FFF7D5FB06B070BD00BF70500020E9
:10465000DC480008E1480008D9450008024AD36A4E
:104660001843D062704700BF484E00204B6843603B
:104670008B688360CB68C3600B6943614B690362DD
:104680008B6943620B6803607047000008B5204BDC
:10469000DA6A42F07F02DA62DA6A22F07F02DA62D4
:1046A000DA6ADA6C42F07F02DA64DA6E42F07F0294
:1046B000DA66184ADB6E11464FF09040FFF7D6FFDE
:1046C00002F11C0100F58060FFF7D0FF02F1380114
:1046D00000F58060FFF7CAFF02F1540100F5806029
:1046E000FFF7C4FF02F1700100F58060FFF7BEFF25
:1046F00002F18C0100F58060FFF7B8FF02F1A8011C
:1047000000F58060FFF7B2FFBDE80840FFF7F0B8A2
:1047100000100240E848000808B500F009F8FFF76B
:1047200017FBBDE80840FFF7AFBE00007047000070
:1047300008B5FFF7D5F8FFF7E9FEFFF7F7FFBDE88B
:104740000840FFF731BF00000B460146184600F055
:1047500001B8000010B5054C13462CB10A460146BD
:104760000220AFF3008010BD2046FCE700000000EF
:10477000024B01461868FFF7C5BD00BF402300206B
:1047800010B501390244904201D1002005E00378C0
:1047900011F8014FA34201D0181B10BD0130F2E700
:1047A0002DE9F041A3B1C91A17780144044603F179
:1047B000FF3C8C42204601D9002009E00578BD422B
:1047C00004F10104F5D10CEB0405D618A54201D182
:1047D000BDE8F08115F8018D16F801EDF045F5D032
:1047E000E7E70000034611F8012B03F8012B002A2C
:1047F000F9D170476F72672E6172647570696C6F62
:10480000742E4E75636C656F2D473439310000008E
:1048100040A2E4F1646891060041A3E5F265699263
:10482000070000004261642043414E4966616365B0
:1048300020696E6465782E00000000000000000012
:10484000451E0008D51800085D2500084519000818
:10485000511900089D1B0008F51A00080D190008E1
:1048600011190008E9180008D1180008591B0008A0
:10487000F5180008E526000895260008011900082B
:104880002D1B000801040E05054B02020E05054B09
:1048900004010E05054B05010B04044B080106033A
:1048A00003460000636C6B73776300000003000035
:1048B00000000000000100000000010103000000F2
:1048C00023283101040704000100000063300000C8
:1048D000CC480008A04E0020705000206D61696E29
:1048E0000069646C650000000004002800000000FE
:1048F000AAAAAAAA00000024DFFF0000000000000E
:104900000000000000000A0000000000AAAAAAAAF5
:1049100000000000FFFF0000000000009900000000
:104920000000000000000000AAAAAAAA00000000DF
:10493000FFFF000000000000000000000000000079
:1049400000000000AAAAAAAA00000000FFFF0000C1
:104950000000000000000000000000000000000057
:10496000AAAAAAAA00000000FFFF000000000000A1
:10497000000000000000000000000000AAAAAAAA8F
:1049800000000000FFFF0000000000000000000029
:104990000000000000000000AAAAAAAA000000006F
:1049A000FFFF000000000000000000000000000009
:1049B0001004000000000000006003000000000080
:1049C000FE2A0100D2040000006889096D8BB9023B
:1049D00000B4C4040068890900688909006889096D
:1049E00000688909006889090068890900000000D9
:1049F0004423002000000000000000000000000030
:104A000000000000000000000000000000000000A6
:104A10000000000000000000000000000000000096
:104A20000000000000000000000000000000000086
:104A30000000000000000000000000000000000076
:104A40000000000000000000000000000000000066
:104A500000000000FFFFFFFFFFFFFFFFFFFFFFFF62
:104A6000FFFFFFFFFFFFFFFFFFFFFFFFFFFFFFFF56
:104A7000FFFFFFFFFFFFFFFFFFFFFFFFFFFFFFFF46
:104A8000FFFFFFFFFFFFFFFFFFFFFFFFFFFFFFFF36
:104A9000FFFFFFFFFFFFFFFFFFFFFFFFFFFFFFFF26
:10A0000000070020D1AF0008051F0108611E0108EC
:10A01000CD1E0108611E0108991E0108D3AF00087A
:10A02000D3AF0008D3AF0008D3AF0008556C0108C8
:10A03000D3AF0008D3AF0008D3AF0008D3AF0008F8
:10A04000D3AF0008D3AF0008D3AF0008D3AF0008E8
:10A05000D3AF0008D3AF000831830108598301084A
:10A0600081830108A9830108D183010819770108B8
:10A070002D770108417701085577010869770108B4
:10A080007D7701089177010889740108D3AF000832
:10A09000D3AF00085512010865120108F9830108C1
:10A0A000D3AF0008D3AF0008D3AF0008D3AF000888
:10A0B000E1840108D3AF0008D3AF0008DD790108BF
:10A0C000F97A0108D3AF0008D3AF0008D3AF000876
:10A0D000D3AF0008CD840108D3AF0008D3AF000888
:10A0E0005D840108D3AF0008D3AF0008D3AF0008E8
:10A0F000D3AF0008D3AF0008D3AF0008D3AF000838
:10A10000D3AF0008D3AF0008D3AF0008D3AF000827
:10A11000D3AF0008D3AF0008D3AF0008D3AF000817
:10A12000B9770108CD770108E1770108F5770108D3
:10A1300009780108D3AF0008D3AF0008D3AF0008F7
:10A14000D3AF0008D3AF0008D3AF0008D3AF0008E7
:10A15000D3AF0008D3AF0008D3AF0008D3AF0008D7
:10A16000D3AF0008D3AF0008D3AF0008D3AF0008C7
:10A17000D3AF0008D3AF0008D3AF0008D3AF0008B7
:10A18000D3AF0008D3AF0008D3AF0008D3AF0008A7
:10A19000D3AF0008D3AF0008D3AF0008D3AF000897
:10A1A000D3AF0008D3AF0008D3AF0008D3AF000887
:10A1B000D3AF0008D3AF0008D3AF0008D3AF000877
:10A1C000A57701081D780108317801084578010854
:10A1D000D3AF0008D3AF0008D3AF0008D3AF000857
:10A1E00015B50008ADF800089D180108B53501083F
:10A1F000C95A010800000000000000000000000033
:10A2000040A2E4F1646891068D0B318B183F21D890
:10A21000BC9B010003BEC59300001004FFFFFFFFBD
:10A22000FFFFFFFF81F0004102E000BF83F0004329
:10A2300030B54FEA41044FEA430594EA050F08BFE1
:10A2400090EA020F1FBF54EA000C55EA020C7FEAA5
:10A25000645C7FEA655C00F0E2804FEA5454D4EB22
:10A260005555B8BF6D420CDD2C4480EA020281EAEC
:10A27000030382EA000083EA010180EA020281EA24
:10A280000303362D88BF30BD11F0004F4FEA013176
:10A290004FF4801C4CEA113102D0404261EB410185
:10A2A00013F0004F4FEA03334CEA133302D052420B
:10A2B00063EB430394EA050F00F0A780A4F10104C7
:10A2C000D5F1200E0DDB02FA0EFC22FA05F2801801
:10A2D00041F1000103FA0EF2801843FA05F35941E7
:10A2E0000EE0A5F120050EF1200E012A03FA0EFC66
:10A2F00028BF4CF0020C43FA05F3C01851EBE37190
:10A3000001F0004507D54FF0000EDCF1000C7EEBAC
:10A3100000006EEB0101B1F5801F1BD3B1F5001FEA
:10A320000CD349085FEA30004FEA3C0C04F1010409
:10A330004FEA445212F5800F80F09A80BCF1004F32
:10A3400008BF5FEA500C50F1000041EB045141EAB4
:10A35000050130BD5FEA4C0C404141EB0101013C7D
:10A3600028BFB1F5801FE9D291F0000F04BF01466C
:10A370000020B1FA81F308BF2033A3F10B03B3F13E
:10A3800020020CDA0C3208DD02F1140CC2F10C02CE
:10A3900001FA0CF021FA02F10CE002F11402D8BF2C
:10A3A000C2F1200C01FA02F120FA0CFCDCBF41EAF8
:10A3B0000C019040E41AA2BF01EB0451294330BDC7
:10A3C0006FEA04041F3C1CDA0C340EDC04F11404A4
:10A3D000C4F1200220FA04F001FA02F340EA03007B
:10A3E00021FA04F345EA030130BDC4F10C04C4F1C1
:10A3F000200220FA02F001FA04F340EA03002946A1
:10A4000030BD21FA04F0294630BD94F0000F83F4EA
:10A41000801306BF81F480110134013D4EE77FEACD
:10A42000645C18BF7FEA655C29D094EA050F08BF19
:10A4300090EA020F05D054EA000C04BF19461046FA
:10A4400030BD91EA030F1EBF0021002030BD5FEA3E
:10A45000545C05D14000494128BF41F0004130BD66
:10A4600014F580043CBF01F5801130BD01F00045BA
:10A4700045F0FE4141F470014FF0000030BD7FEA2D
:10A48000645C1ABF194610467FEA655C1CBF0B4628
:10A49000024650EA013406BF52EA033591EA030F3F
:10A4A00041F4002130BD00BF90F0000F04BF002137
:10A4B000704730B54FF4806404F132044FF000056A
:10A4C0004FF0000150E700BF90F0000F04BF0021E3
:10A4D000704730B54FF4806404F1320410F0004549
:10A4E00048BF40424FF000013EE700BF42004FEA44
:10A4F000E2014FEA31014FEA02701FBF12F07F43C1
:10A5000093F07F4F81F06051704732F07F4208BF77
:10A51000704793F07F4F04BF41F40021704730B57E
:10A520004FF4607401F0004521F000411CE700BFCA
:10A5300050EA010208BF704730B54FF000050AE04D
:10A5400050EA010208BF704730B511F0004502D54E
:10A55000404261EB41014FF4806404F132045FEA50
:10A56000915C3FF4D8AE4FF003025FEADC0C18BFF9
:10A5700003325FEADC0C18BF033202EBDC02C2F1EB
:10A58000200300FA03FC20FA02F001FA03FE40EA7D
:10A590000E0021FA02F11444BDE600BF70B54FF081
:10A5A000FF0C4CF4E06C1CEA11541DBF1CEA13555F
:10A5B00094EA0C0F95EA0C0F00F0DEF82C4481EAC7
:10A5C000030621EA4C5123EA4C5350EA013518BFE7
:10A5D00052EA033541F4801143F4801338D0A0FBD4
:10A5E00002CE4FF00005E1FB02E506F00042E0FB81
:10A5F00003E54FF00006E1FB03569CF0000F18BF87
:10A600004EF0010EA4F1FF04B6F5007F64F540742E
:10A6100004D25FEA4E0E6D4146EB060642EAC621C1
:10A6200041EA55514FEAC52040EA5E504FEACE2E2E
:10A63000B4F1FD0C88BFBCF5E06F1ED8BEF1004F31
:10A6400008BF5FEA500E50F1000041EB045170BDAD
:10A6500006F0004646EA010140EA020081EA0301F1
:10A66000B4EB5C04C2BFD4EB0C0541EA045170BDED
:10A6700041F480114FF0000E013C00F3AB8014F167
:10A68000360FDEBF002001F0004170BDC4F10004B0
:10A69000203C35DA0C341BDC04F11404C4F1200531
:10A6A00000FA05F320FA04F001FA05F240EA02008C
:10A6B00001F0004221F0004110EBD37021FA04F6C2
:10A6C00042EB06015EEA430E08BF20EAD37070BD7C
:10A6D000C4F10C04C4F1200500FA04F320FA05F0DB
:10A6E00001FA04F240EA020001F0004110EBD370DD
:10A6F00041F100015EEA430E08BF20EAD37070BD4D
:10A70000C4F1200500FA05F24EEA020E20FA04F325
:10A7100001FA05F243EA020321FA04F001F00041D4
:10A7200021FA04F220EA020000EBD3705EEA430E45
:10A7300008BF20EAD37070BD94F0000F0FD101F074
:10A740000046400041EB010111F4801F08BF013CAD
:10A75000F7D041EA060195F0000F18BF704703F0EB
:10A760000046520043EB030313F4801F08BF013D72
:10A77000F7D043EA0603704794EA0C0F0CEA13552E
:10A7800018BF95EA0C0F0CD050EA410618BF52EAE8
:10A790004306D1D181EA030101F000414FF00000EE
:10A7A00070BD50EA410606BF1046194652EA4306FC
:10A7B00019D094EA0C0F02D150EA013613D195EA70
:10A7C0000C0F05D152EA03361CBF104619460AD1B8
:10A7D00081EA030101F0004141F0FE4141F47001C2
:10A7E0004FF0000070BD41F0FE4141F4780170BDB2
:10A7F00070B54FF0FF0C4CF4E06C1CEA11541DBF17
:10A800001CEA135594EA0C0F95EA0C0F00F0A7F818
:10A81000A4EB050481EA030E52EA03354FEA013145
:10A8200000F088804FEA03334FF0805545EA131358
:10A8300043EA12634FEA022245EA111545EA106520
:10A840004FEA00260EF000419D4208BF964244F1B7
:10A85000FD0404F5407402D25B084FEA3202B61AD6
:10A8600065EB03055B084FEA32024FF480104FF4AA
:10A87000002CB6EB020E75EB030E22BFB61A75461E
:10A8800040EA0C005B084FEA3202B6EB020E75EBB1
:10A89000030E22BFB61A754640EA5C005B084FEA19
:10A8A0003202B6EB020E75EB030E22BFB61A7546E6
:10A8B00040EA9C005B084FEA3202B6EB020E75EBF1
:10A8C000030E22BFB61A754640EADC0055EA060EB2
:10A8D00018D04FEA051545EA16754FEA06164FEAF5
:10A8E000C30343EA52734FEAC2025FEA1C1CC0D1A1
:10A8F00011F4801F0BD141EA00014FF000004FF02E
:10A90000004CB6E711F4801F04BF01430020B4F1EE
:10A91000FD0C88BFBCF5E06F3FF6AFAEB5EB030CA6
:10A9200004BFB6EB020C5FEA500C50F1000041EBA3
:10A93000045170BD0EF0004E4EEA113114EB5C0470
:10A94000C2BFD4EB0C0541EA045170BD41F4801143
:10A950004FF0000E013C90E645EA060E8DE60CEA4B
:10A96000135594EA0C0F08BF95EA0C0F3FF43BAF68
:10A9700094EA0C0F0AD150EA01347FF434AF95EA1F
:10A980000C0F7FF425AF104619462CE795EA0C0F03
:10A9900006D152EA03353FF4FDAE1046194622E7D0
:10A9A00050EA410618BF52EA43067FF4C5AE50EAAA
:10A9B00041047FF40DAF52EA43057FF4EBAE12E79A
:10A9C0004FF0FF3C06E000BF4FF0010C02E000BF7B
:10A9D0004FF0010C4DF804CD4FEA410C7FEA6C5C5E
:10A9E0004FEA430C18BF7FEA6C5C1BD001B050EA01
:10A9F000410C0CBF52EA430C91EA030F02BF90EAEC
:10AA0000020F0020704710F1000F91EA030F58BFAA
:10AA1000994208BF90422CBFD8176FEAE37040F00C
:10AA2000010070474FEA410C7FEA6C5C02D150EAAA
:10AA3000013C07D14FEA430C7FEA6C5CD6D152EA65
:10AA4000033CD3D05DF8040B704700BF844610462A
:10AA500062468C461946634600E000BF01B5FFF729
:10AA6000B7FF002848BF10F1000F01BD4DF808EDF9
:10AA7000FFF7F4FF0CBF012000205DF808FB00BFCA
:10AA80004DF808EDFFF7EAFF34BF012000205DF824
:10AA900008FB00BF4DF808EDFFF7E0FF94BF012071
:10AAA00000205DF808FB00BF4DF808EDFFF7CEFF72
:10AAB00094BF012000205DF808FB00BF4DF808EDB1
:10AAC000FFF7C4FF34BF012000205DF808FB00BF82
:10AAD0004FEA410C7FEA6C5C02D150EA013C0AD19A
:10AAE0004FEA430C7FEA6C5C02D152EA033C02D18C
:10AAF0004FF0000070474FF0010070474FEA4102ED
:10AB000012F5001215D211D56FF47873B3EB6252BF
:10AB100012D94FEAC12343F0004343EA505311F0E6
:10AB2000004F23FA02F018BF404270474FF0000078
:10AB3000704750EA013005D111F0004008BF6FF0B6
:10AB4000004070474FF00000704700BF4A0011D22C
:10AB500012F5001211D20DD56FF47873B3EB625277
:10AB60000ED44FEAC12343F0004343EA505323FA83
:10AB700002F070474FF00000704750EA013002D1F8
:10AB80004FF0FF3070474FF0000070474FEA41022E
:10AB9000B2F1E04324BFB3F5001CDCF1FE5C0DD93B
:10ABA00001F0004C4FEAC0024CEA5070B2F1004F85
:10ABB00040EB830008BF20F00100704711F0804F88
:10ABC00021D113F13872BCBF01F00040704741F44D
:10ABD00080114FEA5252C2F11802C2F1200C10FA51
:10ABE0000CF320FA02F018BF40F001004FEAC12335
:10ABF0004FEAD32303FA0CFC40EA0C0023FA02F3D9
:10AC00004FEA4303CCE77FEA625307D150EA0133AE
:10AC10001EBF4FF0FE4040F44000704701F000407E
:10AC200040F0FE4040F40000704700BF7BB972B9AD
:10AC30000029BEBF00204FF0004106E008BF0028F9
:10AC40001CBF6FF000414FF0FF3000F0BFB9ADF115
:10AC5000080C6DE904CE002909DB002B1ADB00F09B
:10AC60004DF8DDF804E0DDE9022304B0704740420E
:10AC700061EB4101002B1BDB00F040F8DDF804E044
:10AC8000DDE9022304B0404261EB4101524263EB33
:10AC900043037047524263EB430300F02FF8DDF8A3
:10ACA00004E0DDE9022304B0404261EB410170475A
:10ACB000524263EB430300F021F8DDF804E0DDE9E4
:10ACC000022304B0524263EB4303704753B94AB9BD
:10ACD000002908BF00281CBF4FF0FF314FF0FF30A4
:10ACE00000F074B9ADF1080C6DE904CE00F006F87F
:10ACF000DDF804E0DDE9022304B070472DE9F047F8
:10AD0000089D04468E46002B4DD18A42944669D94F
:10AD1000B2FA82F252B101FA02F3C2F1200120FA32
:10AD200001F10CFA02FC41EA030E94404FEA1C4880
:10AD3000210CBEFBF8F61FFA8CF708FB16E341EA7C
:10AD4000034306FB07F199420AD91CEB030306F102
:10AD5000FF3080F01F81994240F21C81023E634423
:10AD60005B1AA4B2B3FBF8F008FB103344EA0344C7
:10AD700000FB07F7A7420AD91CEB040400F1FF33DC
:10AD800080F00A81A74240F207816444023840EA19
:10AD90000640E41B00261DB1D4400023C5E9004352
:10ADA0003146BDE8F0878B4209D9002D00F0EF80D5
:10ADB0000026C5E9000130463146BDE8F087B3FA08
:10ADC00083F6002E4AD18B4202D3824200F2F980F0
:10ADD000841A61EB030301209E46002DE0D0C5E9F3
:10ADE000004EDDE702B9FFDEB2FA82F2002A40F03F
:10ADF0009280A1EB0C014FEA1C471FFA8CFE012642
:10AE0000200CB1FBF7F307FB131140EA01410EFBE5
:10AE100003F0884208D91CEB010103F1FF3802D28C
:10AE2000884200F2CB804346091AA4B2B1FBF7F086
:10AE300007FB101144EA01440EFB00FEA64508D9A9
:10AE40001CEB040400F1FF3102D2A64500F2BB80E6
:10AE50000846A4EB0E0440EA03409CE7C6F1200735
:10AE6000B34022FA07FC4CEA030C20FA07F401FA7B
:10AE700006F31C43F9404FEA1C4900FA06F3B1FB04
:10AE8000F9F8200C1FFA8CFE09FB181140EA014169
:10AE900008FB0EF0884202FA06F20BD91CEB010106
:10AEA00008F1FF3A80F08880884240F28580A8F15E
:10AEB00002086144091AA4B2B1FBF9F009FB1011B0
:10AEC00044EA014100FB0EFE8E4508D91CEB01014E
:10AED00000F1FF346CD28E456AD90238614440EAF1
:10AEE0000840A0FB0294A1EB0E01A142C846A64671
:10AEF00056D353D05DB1B3EB080261EB0E0101FAFA
:10AF000007F722FA06F3F1401F43C5E90071002656
:10AF10003146BDE8F087C2F12003D8400CFA02FCAC
:10AF200021FA03F3914001434FEA1C471FFA8CFEBC
:10AF3000B3FBF7F007FB10360B0C43EA064300FBAC
:10AF40000EF69E4204FA02F408D91CEB030300F14A
:10AF5000FF382FD29E422DD9023863449B1B89B201
:10AF6000B3FBF7F607FB163341EA034106FB0EF38A
:10AF70008B4208D91CEB010106F1FF3816D28B4237
:10AF800014D9023E6144C91A46EA004638E72E4603
:10AF9000284605E70646E3E61846F8E64B45A9D2FB
:10AFA000B9EB020864EB0C0E0138A3E74646EAE76A
:10AFB000204694E74046D1E7D0467BE7023B614418
:10AFC00032E7304609E76444023842E7704700BF81
:10AFD00002E000F000F8FEE772B6374880F3088818
:10AFE000364880F3098836483649086040F2000048
:10AFF000CCF200004EF63471CEF200010860BFF3CF
:10B000004F8FBFF36F8F40F20000C0F2F0004EF69A
:10B010008851CEF200010860BFF34F8FBFF36F8FEE
:10B020004FF00000E1EE100A4EF63C71CEF2000146
:10B030000860062080F31488BFF36F8F0EF0FEFFC8
:10B040000FF018F94FF055301F491B4A91423CBF91
:10B0500041F8040BFAE71D49184A91423CBF41F8F8
:10B06000040BFAE71A491B4A1B4B9A423EBF51F8A0
:10B07000040B42F8040BF8E700201849184A9142E3
:10B080003CBF41F8040BFAE70EF0DCFF0FF038F993
:10B09000144C154DAC4203DA54F8041B8847F9E709
:10B0A00000F028FA114C124DAC4203DA54F8041B9C
:10B0B0008847F9E70EF0C4BF0007002000230020F6
:10B0C00000A0000808ED00E00001002000070020BB
:10B0D000A83902080023002014250020182500208C
:10B0E000E0720020E0A10008F4A10008F4A100082B
:10B0F000F4A100082DE9F04F2DED108AC1F80CD015
:10B10000C3689D46BDEC108ABDE8F08F002383F331
:10B1100011882846A04700200EF07EF9FEE70EF0C9
:10B1200003F800DFFEE7000010F8012B11F8013BE7
:10B13000012A28BF9A42F7D0D01A7047034613F865
:10B14000012B002AFBD1181A0138704701F0FF01CA
:10B15000102A2BDB10F0070F08D010F8013B013A42
:10B160008B422DD010F0070F42B3F6D1F0B441EA74
:10B17000012141EA014122F007047FF0000700238A
:10B18000F0E80256083C85EA010586EA010685FAE0
:10B1900047F5A3FA87F586FA47F6A5FA87F68EB93A
:10B1A000EED1F0BC01F0FF0102F0070232B110F85D
:10B1B000013B013A83EA010313B1F8D10020704743
:10B1C00001387047002D06BF35460338073815F0A3
:10B1D000010F07D1013015F4807F02BF013015F453
:10B1E000C03F0130F0BC0138704700BF38B50022C5
:10B1F000002304460D46FFF743FC28B920462946A4
:10B20000BDE8384000F00AB8204605F1004100F0E2
:10B2100005F8404261EB410138BD00BFD0B50C4B91
:10B22000002206460F46FFF7B9F9FFF78FFC0446E8
:10B23000FFF73AF9074B0022FFF7B0F902460B4639
:10B2400030463946FEF7F2FFFFF780FC2146D0BDBD
:10B250000000F03D0000F0417047000070B504466A
:10B26000183004F045FC144B1449196004F13C00FB
:10B27000002314269DB206FB05120133127C002A1E
:10B28000F8D10F4B1D800F4B1A6812B10E4806F013
:10B290003DFE186004F58053012104F581501A62C7
:10B2A0009977043006F028F8084B1A680AB1084864
:10B2B000EDE71C60204670BD1436002028E401082C
:10B2C00012360020D43500204CE301081825002058
:10B2D00067E3010838B51A4D04460EF063FE0EF020
:10B2E00075FE286820231A46006C4FF4E13102F005
:10B2F00003F828684FF4807380224FF4E131C06C6A
:10B3000001F0FAFF204600F029F90EF05FFE20461A
:10B3100000F0C0FF04F1180004F0A6FC0EF056FE89
:10B3200005F042F82B68D86A03685B68984710B14B
:10B33000044806F057F8BDE8384006F011BE00BFDB
:10B340003825002088E301080148FFF7C3BF00BF8C
:10B350003C2500202DE9F341144C154EDFF86080A8
:10B36000144F20460EF086FD134A0146121B134867
:10B3700001F02AF80DF0FCFD0446A4B1206AE16951
:10B380000191B04214BF251AA8EB06050EF072FD1C
:10B39000019902462B46384601F016F820460DF07A
:10B3A000F7FD0446E9E702B0BDE8F08100010020A6
:10B3B00000070020B2E3010800070020A8E301080D
:10B3C0000023002010B50F4C03F05CFB2368986A43
:10B3D00003680522DB69002198472368986A03689F
:10B3E00064211B6998472368986A036828215B6871
:10B3F00098472368986A0368BDE810401B690021DC
:10B40000184700BF3825002038B5054606F0A8FDCE
:10B410002B4A1368C31AB3F57A7F044609D9294B1E
:10B4200010601B782BB94FF09042536983F02003D2
:10B43000536104F0E9FC244A136841F28831E31AAD
:10B440008B4206D9016821B1146002891F4800F0BF
:10B45000BBFF6B7ADA070AD51D4A136841F28831BF
:10B46000E31A8B4203D928461460FFF773FF6B7A07
:10B470009B0709D4174A1368E31A132B1DD82846D3
:10B48000BDE8384001F022B806F06AFD43F6982383
:10B490009842EFD91048FFF795FF10480EF094FC42
:10B4A000BFF34F8F0E490F4BCA6802F4E06213439B
:10B4B000CB60BFF34F8F00BFFDE71460DFE700BF35
:10B4C0001C2500200023002024250020C4E30108BF
:10B4D00020250020282500203C250020010007B061
:10B4E00000ED00E00400FA050148FFF78DBF00BF42
:10B4F0003C25002038B5054B1C6823680A461D68AA
:10B50000034B01462046A847002038BD38250020BF
:10B510002C25002010B50A4C2046FFF79FFE094A53
:10B52000094920460EF00EFF06F0B0F9074B084A15
:10B530001860BDE810400749074801F0FDBD00BF95
:10B540003C2500201C3F002059B20008382500206F
:10B55000E9B4000849B300082C25002013B50446BF
:10B5600003F0FAFF02F0CEFF204603F075FF18B19A
:10B57000B4F90030022B0BD004F060FA02F094FC16
:10B5800002230DF106012046ADF8063004F00AFA58
:10B5900002230DF106012046ADF8063004F0F8F95B
:10B5A00002B0BDE8104003F095BE0000BFF34F8F1E
:10B5B0000549064BCA6802F4E0621343CB60BFF34F
:10B5C0004F8F00BFFDE700BF00ED00E00400FA056B
:10B5D00013B51022002104468DF807200EF0EAFE74
:10B5E000054B1B68D86A03680DF107021B6B2146E7
:10B5F000984702B010BD00BF38250020F0B58BB0D1
:10B60000174604460E4606F0ABFC054602F00CFC5D
:10B6100003464FF4C87005F5167504F58054B3FB66
:10B62000F0F202FB103315FA83F3A361FD7E2DB90E
:10B630001B4805F0D7FE25770BB0F0BD384605A9AD
:10B6400001F0C8F907460028F6D101A8FFF7C0FFAE
:10B650009DF8165001A92A460DF117000EF08CFE38
:10B6600020B1104805F0BEFE2777E5E70F2D09D879
:10B67000A3692577A3F51673A36129460A4805F047
:10B68000B1FED9E79DF814100029D5D030460AF054
:10B6900021FE9DF81420A17F044805F0A3FECBE70E
:10B6A000C8E40108F3E4010814E5010836E50108DF
:10B6B00007B5104601A901F03BF858B9074B9DF8B2
:10B6C00004101B68D86AA1F1FF02036851421B688D
:10B6D0005141984703B05DF804FB00BF38250020B6
:10B6E00038B5084615461C460AF0FCFD60B99DF8C1
:10B6F0001030022B07D1012C05D11BA3D3E9002365
:10B70000C5E90023012038BD0B2C0BD884B1601E85
:10B710000A280DD8DFE800F00E0C0C0C160C0C0CEF
:10B720000C1E1A00282C09D040F24C439C4215D024
:10B730000020E8E70EA3D3E90023E1E70EA3D3E955
:10B740000023DDE70EA3D3E90023D9E70EA3D3E955
:10B750000023D5E70EA3D3E90023D1E70EA3D3E955
:10B760000023CDE7AFF30080401DA12026812A0BE6
:10B770009E6AC421818A46EE26417272DF25D7B7C0
:10B78000F017304A39059E56D5A4D139F922B6A70B
:10B79000CDD269EBC51A133B03806A5575F3008758
:10B7A00013B59DF81040CDE9003413460A46014612
:10B7B000806AFFF795FF02B010BD000070B500F57C
:10B7C00080560D46746974B90C2101200EF0CCF935
:10B7D000706108B9002070BD056084600430FAE72C
:10B7E0002646A46824B12368AB42F9D1201DF2E7B4
:10B7F0000C2101200EF0B8F9B0600028EAD00560F5
:10B80000B3689C60B068E9E72DE9F04190B000F5BD
:10B810008151BDF8587004461646043140F2434247
:10B8200001A8984601F0C6FC012F0ED146EA074157
:10B830002046FFF7C3FF054670B9002401A801F0B8
:10B84000D5FC204610B0BDE8F08104F144000AF0B8
:10B8500049FD0028EAD1F0E73822002102A80EF0C5
:10B86000A9FD02238DF808309DF85C308DF820305A
:10B87000189B0993BDF86430ADF82830CDE9046811
:10B88000ADF81870079506F06DFB0D4BC01841F12F
:10B890000001CDE90C0104F1440002A90AF024FDE5
:10B8A000084B0028D5BF9A881A6801321218D4BFF5
:10B8B0009A801A600028D4BF00240124BEE700BF8C
:10B8C00040420F008435002030B58FB014460D463D
:10B8D0003822002168460EF06DFDDDE91223CDE926
:10B8E0000223BDF85030ADF8103004F11903059370
:10B8F000A37E8DF81830159B0793BDF85830ADF82E
:10B90000203006F02FFB0D4BC31841F100016A46B1
:10B91000CDE90A312846E17E0AF02AFD084B0028CD
:10B92000D5BF9A881A6801321218D4BF9A801A605B
:10B930000028D4BF002001200FB030BD40420F00CE
:10B9400084350020F0B591B005460E46104608A992
:10B95000144601F007F938BB9DF82030012B07D1C0
:10B9600004F06CF802F0A0FA03F0B4FC03F0F4FD6C
:10B970001022002106AF0CA80EF01CFD0122394652
:10B980000CA88DF8382001F011F90A23029307A3BF
:10B99000D3E9002380B2CDE90370CDE9002331461D
:10B9A00022462846FFF790FF11B0F0BDCDD269EBDB
:10B9B000C51A133B2DE9F041ADF5487D66AC05464F
:10B9C0000E46174600214FF4C47220460EF0F2FCDA
:10B9D00006F0C6FA2F4B4FF47A72B0FBF2F0186003
:10B9E00093E8070084E8070001F072FA037C2374EF
:10B9F00001F06EFA437C63740323A374264B5A69E7
:10BA000062610DF5DD709A68DB68A261E361FFF7A2
:10BA1000DFFD41F20403EA682384204B002A186802
:10BA20001F4B29DDCDE900320DF2CB211D4BC06A41
:10BA3000502201F0FDFC50210DF2CB200FF090F9C7
:10BA40000DF11C0884F8320141460122204600F025
:10BA500089FE012302930DA3D3E9002380B2CDE92F
:10BA60000380CDE9002331463A462846FFF72CFFF4
:10BA70000DF5487DBDE8F081009350220A4BC06A65
:10BA80000DF2CB2101F0D4FCD5E700BF9E6AC421A2
:10BA9000818A46EE7835002000A200083825002073
:10BAA0005BE5010854E50108943102082DE9F041F5
:10BAB0001546ADF5866D06460F460EF087FA08A9C5
:10BAC000284601F089F80446002840F09F8001468E
:10BAD0004FF4D072A4A80EF06DFC9DF8B880B8F1B8
:10BAE000100F7ED808F1FF330F2B2BD842460DF1F3
:10BAF000B9010DF2D1300EF04FFC424651490DF123
:10BB0000B9000FF005F90246B0B94F480DF11F0119
:10BB100002F0E6FE0446002C63D09DF8B83073B303
:10BB20009DF828305BB39DF81F20013A032A6DD899
:10BB3000DFE802F01C2E384122460DF11F010DF204
:10BB4000D130E5E7BDF82000479447AA0DF11F0169
:10BB500003F0E8F90446002843D0012300930DF2D6
:10BB6000D132112347A902F0F7FDD4E7012B4DD1C3
:10BB70000C9B8DF81C3147A9204603F0F5FE9DF87B
:10BB80001F30013B032B41D8DFE803F01C444A4F30
:10BB9000012B3BD10C9BADF81C3147A9204603F08B
:10BBA0001BFFECE7012B31D10C9B479347A92046A3
:10BBB00003F034FFE3E7022B28D10CA9204603F061
:10BBC000A5FEDCE701238DF8903294F90030DA17F6
:10BBD000CDE9A6325C210DF2D1300FF0C1F88DF81D
:10BBE000D00347AC01222146A4A801F01DF90B2384
:10BBF000029312A3D3E9002380B2CDE90340CDE93B
:10BC0000002339462A463046FFF75EFE0DF5866D65
:10BC1000BDE8F08101238DF89032B4F90030D6E709
:10BC200001238DF890322368D1E702238DF89032FA
:10BC30002368A693CEE700BFAFF30080D5A4D13927
:10BC4000F922B6A778E5010881E501082DE9F04F52
:10BC5000DFF8D0A08BB0804608F1440948460AF0CE
:10BC6000C3FB0546002854D00024007E0694CDE98D
:10BC70000744ADF8244001F023FA2A7E8DF8240011
:10BC800005F1100107A80EF087FB2B6843F0004375
:10BC9000069306F067F9204B0390C218DAF8040007
:10BCA0000E4641F1000308F5805750B30168009437
:10BCB00009690D4606A9A847A04222DCDAF804006B
:10BCC00003689B6A9847D0E90A23CDE9042306F06C
:10BCD00049F9DDE90423801A61EB03010F4B83422C
:10BCE00074EB01030DD37B7F072B10D90C4A7C77B3
:10BCF0009388013393804846039A33460AF082FBC7
:10BD000007E048460AF074FB00237B77A4E7013381
:10BD10007B770BB0BDE8F08F40420F007F841E00A0
:10BD200084350020A43500202DE9F0414FF0005368
:10BD3000DFF8E0801B684345FCB005460C4616461C
:10BD400004D03148DC2200210EF034FB4FF00057C4
:10BD500049A9C7F80080304600F088FE002849D184
:10BD60009DF824313B750BB9F37E3B759DF8252179
:10BD700026480DF593710EF00FFB20460AF0B2FA3B
:10BD80004FF0005307AF58758122002128A80EF00C
:10BD900011FB3946012228A800F0AEFE28230293A9
:10BDA00017A3D3E9002380B2CDE90370CDE90023C6
:10BDB000214632462846FFF787FD154F3326013EC0
:10BDC00016F0FF06284608D0FFF740FF3B68986A48
:10BDD000036801215B689847F1E7FFF7F3FA204613
:10BDE0000AF080FA40F0304040F400200DF0ECFF03
:10BDF000FFF7DCFB7CB0BDE8F08100BFAFF3008053
:10BE000026417272DF25D7B70400002016000020FB
:10BE1000382500209AAD44C5F0B5044689B00846DF
:10BE20000E4615460AF05EFA68B92B7E022B1FD12A
:10BE3000EB8A012B1CD12A463146204609B0BDE8C9
:10BE4000F040FFF7DBBBEB8A0B2B0BD883B1013B38
:10BE50000A2B0DD8DFE803F00E0C0C0C1E0C0C0C9A
:10BE60000C463E00282B0DD040F24C42934241D06C
:10BE700009B0F0BD2A463146204609B0BDE8F04081
:10BE8000FFF798BD2A463146204609B0BDE8F0408C
:10BE9000FFF74ABF07AF1E4805F0A4FA0122394652
:10BEA00006A88DF8182000F037FD0523029316A38D
:10BEB000D3E9002380B2CDE90023CDE903702A46FF
:10BEC00031462046FFF700FD06F04AF804F580549D
:10BED0002062CDE72A463146204609B0BDE8F04051
:10BEE000FFF7E4BD2A463146204609B0BDE8F040E0
:10BEF000FFF728BD2A463146204609B0BDE8F0408C
:10BF0000FFF7D6BBAFF30080F017304A39059E56D5
:10BF10008CE501080A460146806AFFF77DBF0000F4
:10BF200049421B4B112912D8DFE801F00911110D0C
:10BF30001111111111111519151D2125292D9A689D
:10BF400001329A6070479A8901329A817047DA8982
:10BF50000132DA8170475A8B01325A8370471A8B4B
:10BF600001321A8370471A8A01321A8270475A8A3C
:10BF700001325A8270479A8B01329A8370479A8AAB
:10BF800001329A827047DA8A0132DA82704700BF42
:10BF9000843500202DE9F04F374E97B00023CDE9CE
:10BFA0000B330A93ADF8343073680446002B5FD02E
:10BFB000324D01274FF0000A4FF0000B70688DF8EA
:10BFC00014704FF000088DF815800368CDE900ABC0
:10BFD0000DF11502D3F8089005A94346C8479DF80E
:10BFE0001430002B44D0414620220EA80EF0E2F976
:10BFF0007068036806AAD3F814800AA90DF1160325
:10C00000C047002834DD9DF8340001F075F80BA915
:10C0100002468DF8500012A80EF0BEF904F1440853
:10C020000A9B0E930EA9DDE9062340460AF0EAFBBF
:10C0300010F10D0F014603D02046FFF771FFBDE759
:10C040000E980AF0CFFB03900E980AF0C5FB039BF5
:10C05000CDE9000708AA41462046FFF741FB18B189
:10C060002B8A01332B82A9E76B8B01336B83A5E706
:10C0700017B0BDE8F08F00BFA43500208435002044
:10C0800007B500F1440168460AF09EFBBDF80400C4
:10C0900064235843BDF80030B0FBF3F080B203B026
:10C0A0005DF804FBF0B597B0044605F059FF4FF476
:10C0B0007A73B0FBF3F0434B434D1B682860D86A9A
:10C0C00003685B6D98474FF6FF73984228BF184688
:10C0D00028810EA90122284600F0F6FB0EAB80B2A3
:10C0E0000293182240F255130025CDE90032039047
:10C0F0002EA3D3E9002304952046FFF785FB637A3E
:10C1000059074ED501220EA93048314F00F0B4FA3C
:10C110000EAB80B202931F264FF4AB73CDE900360D
:10C12000039024A3D3E9002304952046FFF76CFB7A
:10C13000786803689B6A9847002832D03A788DF86F
:10C14000382002680F924268ADF840208268ADF84E
:10C150004220C268ADF844200269ADF84620426929
:10C16000ADF8482082691392C269ADF85020026A86
:10C17000ADF8522007AF436AADF85430012239467A
:10C180000EA800F023FA40F2571380B2CDE90270F6
:10C190000093049509A3D3E9002301962046FFF7F5
:10C1A00033FB17B0F0BD00BFAFF30080F1C6A7C1ED
:10C1B000D068080FD1F886A9B8E33A76753CA33C5D
:10C1C000AE0C08CE382500207835002084350020BC
:10C1D000A4350020F0B506468DB044300AF082F850
:10C1E0002A4D20B100232B7001200DB0F0BD05F0C9
:10C1F000B7FE2B7804463BB13046FFF741FF0121E3
:10C200000246234805F0EEF801F00EFE4FF4C87325
:10C2100006F58057B0FBF3F202FB130304F516702A
:10C2200010FA83F000238DF818303B7FB8611BB9FA
:10C2300001228DF81820BB7708A8FFF7C9F9397FCC
:10C24000C1F11004E4B2062C28BF062408AB224634
:10C2500019440DF119000EF09FF8013406AB0025CA
:10C26000029318220123E4B2CDE90032049505A31C
:10C27000D3E9002303943046FFF7C6FA3D772846FA
:10C28000B3E700BF401DA12026812A0B0023002018
:10C290009CE5010870B5244D244E4FF4807386B0A0
:10C2A000AB80044605F05CFE4FF47A73B0FBF3F00C
:10C2B00028606288B4F902307F2A98BF33700DF18C
:10C2C0001701002304F108008DF8173003F04CFB30
:10C2D00041F2E84000F000FE054608B104F016FB0C
:10C2E000134B1D60134B00225D601A702DB12B683B
:10C2F00061685B680122284698470F4B009304F160
:10C30000440004F174010D4B01944FF47A620390E0
:10C3100009F0B4FF3178039821B106B0BDE8704050
:10C3200009F0D8BF06B070BD78350020B9350020BF
:10C33000AC350020A4350020A1B7000815BF0008C7
:10C3400030B50628134698BF1D4AC7B098BF155C84
:10C3500007930C464FF07C024FF0000127A888BFDE
:10C3600000250EF027F8079B22465A210DF1BE004A
:10C3700004F0EEFF5A2828BF5A2008AC8DF8BD0003
:10C380002146012227A88DF89C5000F0CFFA002307
:10C39000049380B243F6FF731822CDE90240CDE941
:10C3A0000032084804A3D3E90023FFF72DFA47B071
:10C3B00030BD00BFAFF30080759D040C8EA454D631
:10C3C00058E601083C2500200FB407B504AA072051
:10C3D00052F8041B0192FFF7B3FF03B05DF804EBC2
:10C3E00004B0704737B5044644300AF00BF82046D5
:10C3F000FFF746FE462802D92A4804F0F3FF2046FC
:10C40000FFF750FE94F90850002D38D0002304F1B6
:10C410000800EDB201A98DF8043003F0A5FA2A2D29
:10C42000214C0AD1214D2846FFF7CEFF2368986A98
:10C43000036864215B689847F5E72B2D04D11C48FD
:10C44000FFF7C2FF1B4B98474FF4FA6101A800F0B9
:10C4500097FE2468A06A03684FF47A715B68984776
:10C46000E06A03689B6A984718B1012816D0124801
:10C4700000E01248FFF7A8FF01A800F08DFE104B66
:10C4800000225A7105F06CFD47F23053984207D9EB
:10C490000C4803B0BDE830400DF096BC0A48E9E70F
:10C4A00003B030BDD4E5010838250020F2E50108CD
:10C4B00003E6010838ED00E03EE6010813E6010856
:10C4C00078350020263A09B028E601082DE9F34125
:10C4D000044605F045FD38490B68C31A322B054662
:10C4E0001BD9364B1B78C3B13548027801239340E2
:10C4F00023F4AA4323F055031B041B0C002B0EBF8F
:10C5000001260026202343EA465301324FF090468D
:10C5100002F01F02B36102700D6004F5805605F051
:10C520001FFDB369984202D92046FFF753FE254A02
:10C530001368EB1AB3F57A7F07D3156005F012FD87
:10C5400002460B462046FFF74DFF05F005FD04F5BA
:10C550008155DFF874800746043505F0FDFCC01BEB
:10C56000B0F57A7F17D2D8F80030986A03684FF494
:10C5700080619B68984740F2D772294601A800F075
:10C5800019FE2046FFF762FB2046FFF703FD01A8D6
:10C5900000F02CFEE1E7336A5BB105F0E1FC336AA1
:10C5A000C01AB0F57A7F04D92046FEF70BFFFEF7DC
:10C5B000FDFF02B0BDE8F081B4350020002300206B
:10C5C000B8350020B03500203825002070B50C4665
:10C5D000192605463246002120460DF0EBFE2B467B
:10C5E0002046082200210AF0A7F82B1D2046202211
:10C5F00008210AF0A1F805F108032046102228219D
:10C600000AF09AF805F10A032046102238210AF0B0
:10C6100093F805F10C032046102248210AF08CF80B
:10C6200005F10E032046102258210AF085F805F185
:10C6300010032046102268210AF07EF805F1140349
:10C640002046202278210AF077F805F118032046C9
:10C65000102298210AF070F805F11A0320461022E2
:10C66000A8210AF069F8204605F11C031022B82120
:10C670000AF062F8304670BD70B50C461C260546BF
:10C680003246002120460DF095FE2B462046202202
:10C6900000210AF051F82B1D2046102220210AF01B
:10C6A0004BF805F108032046202230210AF044F817
:10C6B00005F10C032046102250210AF03DF805F147
:10C6C0000E032046102260210AF036F805F110030F
:10C6D0002046102270210AF02FF805F1120320469F
:10C6E000102280210AF028F805F1140320461022B8
:10C6F00090210AF021F805F1160320461022A0210E
:10C700000AF01AF805F1180320461022B0210AF0A9
:10C7100013F805F11A0320461022C0210AF00CF884
:10C720002046AB191022D0210AF006F8304670BD21
:10C7300013B50446007F10B1A38A012B0CD8002347
:10C74000009108221946204609F0B8FE237FA08AEE
:10C7500023B9B0FA80F0400902B010BD013818BF0B
:10C760000120F9E72DE9F3470D46044600219046E4
:10C77000284640F279120DF01DFE234620220021AA
:10C78000284609F0D9FF231D02222021284609F05E
:10C79000D3FF631D03222221284609F0CDFFA31DEC
:10C7A00003222521284609F0C7FF04F108031022BF
:10C7B0002821284609F0C0FF04F11003082238217F
:10C7C000284609F0B9FF04F1110308224021284648
:10C7D00009F0B2FF04F1120308224821284609F0AB
:10C7E000ABFF04F1140320225021284609F0A4FFD6
:10C7F00004F1180340227021284609F09DFF04F13E
:10C8000020030822B021284609F096FF04F12103F5
:10C810000822B821284609F08FFF04F12207C0261C
:10C820003B46314608222846083609F085FFB6F512
:10C83000A07F07F10107F3D194F832308DF807306B
:10C8400031460DF107030822284609F075FF00263E
:10C8500004F1330A9DF807304FEAC6099E4209F5F4
:10C86000A47720D394F83231502B28BF50238DF871
:10C870000730B8F1000F08D139460DF10703072240
:10C88000284609F059FF09F24F17002604F2331425
:10C890009DF807309E4207EBC6010DD30731C8084B
:10C8A00002B0BDE8F0870AEB0603082239462846A5
:10C8B00009F042FF0136CDE7A3190822284609F006
:10C8C0003BFF0136E4E7000013B5044608460021AB
:10C8D00001602346C0F803102022019009F02CFFCC
:10C8E0000198231D0222202109F026FF0198631DD3
:10C8F0000322222109F020FF0198A31D03222521F4
:10C9000009F01AFF019804F108031022282109F008
:10C9100013FF072002B010BD08B5034608460021EA
:10C920000170012209F008FF012008BD2DE9F34143
:10C930000D4604460021164628467B220DF03AFD9E
:10C94000234603220021284609F0F6FE63781F2BB8
:10C9500028BF1F238DF8063005220DF106030321A1
:10C96000284609F0E9FE01239DF80620DF0003F1C7
:10C970000108013B9A421CD894F821305A2B28BF59
:10C980005A238DF807303EB939460DF107030722C7
:10C99000284609F0D1FE0737002622349DF80730DB
:10C9A0009E4207EBC6010DD30731C80802B0BDE8AF
:10C9B000F08104EB080308223946284609F0BCFE42
:10C9C0004346D1E7A3190822284609F0B5FE0136EF
:10C9D000E4E70000F7B5047F05460E462CB1838AD4
:10C9E000122B02D9012003B0F0BD00231946072203
:10C9F0000096284609F062FD731C00930122002373
:10CA00000721284609F05AFDD4B9B31C009305222A
:10CA100023460821284609F051FD0D24B378102B38
:10CA2000E0D83746B278BB1B934210D32B7FA88A3D
:10CA30000734E408B3B9844294BF00200120D2E750
:10CA4000AB8ADB00083BDB08B3700824E6E7FB1C7D
:10CA50000093214600230822284609F02FFD0834C0
:10CA60000137DFE7201A18BF0120BCE7F7B5047FC4
:10CA700005460E462CB1838ACA2B02D9012003B089
:10CA8000F0BD0023194600960822284609F016FD3D
:10CA9000731CD4B90822009311462346284609F096
:10CAA0000DFD10247378C82BE8D8012372785F1C21
:10CAB000013B934210D32B7FA88A0734E408B3B913
:10CAC000844294BF00200120D9E7AB8ADB00083BF9
:10CAD000DB0873700824E5E7F3190093214600236F
:10CAE0000822284609F0EAFC08343B46DEE7201A13
:10CAF00018BF0120C3E70000F7B50D46044600212A
:10CB00001646284681220DF055FC234608220021B6
:10CB1000284609F011FE94F901206378002AB8BF75
:10CB20007F238DF807309EB90DF1070307220821F6
:10CB3000284609F001FE0F27002602349DF8073031
:10CB40009E4207EBC60105D30731C80803B0F0BD0C
:10CB50000827F1E7A3190822284609F0EDFD013660
:10CB6000ECE7000037B50446007F0D4610B1A38AFC
:10CB7000072B15D8002319460095082220460835B2
:10CB800009F09CFC0123009530220821204609F081
:10CB900095FC237FA08A2BB906288CBF002001209A
:10CBA00003B030BD073818BF0120F9E738B50C468F
:10CBB000002121600546C4F80310034630222046B8
:10CBC00009F0BAFD204605F108030122302109F0E1
:10CBD000B3FD072038BD00002DE9F04390F81C801C
:10CBE00085B006460D46B8F1000F06D0838AE02BCB
:10CBF00003D9012005B0BDE8F083002319460D22BA
:10CC00000095304609F05AFC0DF10F030093032202
:10CC100000230D21304609F051FC9DF80F30042B04
:10CC2000E7D82B72013B032B03D8DFE803F0253054
:10CC30003B461024B8F1000F5FD105F19803009333
:10CC4000214643460722304609F038FC073495F860
:10CC500098305C2BCDD82F4695F898207B1B9342BB
:10CC600052D3337FB08A0734E408002B58D1844272
:10CC700094BF00200120BDE705F11003009340227E
:10CC800001231021304609F019FC5024D2E705F1A8
:10CC900010030093202201231021304609F00EFCDE
:10CCA0003024C7E705F11003009308220023102168
:10CCB000304609F003FC1824BCE705F1100300938B
:10CCC000082200231021304609F0F8FB2B7C802B32
:10CCD0008FD8002705F111092B7CFC009F4204F13D
:10CCE0001804A7D209EB070300930822002321466A
:10CCF000304609F0E3FB0137EEE7B38AC4EBC30328
:10CD0000DB0885F89830A2E707F1990300932146E4
:10CD100000230822304609F0D1FB083401379BE795
:10CD2000201A18BF012065E7F7B50C46137809688B
:10CD30008DF8063015460DF106030322064609F06C
:10CD4000FBFC2168033121602B78013B032B0CD8BD
:10CD5000DFE803F0020D161F05F1080340223046FC
:10CD600009F0EAFC23684033236003B0F0BD05F10D
:10CD700008032022304609F0DFFC23682033F3E764
:10CD800005F108030822304609F0D6FC2368083371
:10CD9000EAE72B7A802B28BF80238DF80730082202
:10CDA0000DF10703304609F0C7FC23680833236000
:10CDB000002709359DF807309F42D6D2EB1921682C
:10CDC0000822304609F0B8FC236808332360013795
:10CDD000F0E7000073B50C46137809688DF807304A
:10CDE00015460DF107030222064609F0A5FC21684D
:10CDF000023121602B78012B03D0022B0BD002B023
:10CE000070BD05F108034022304609F095FC236807
:10CE100040332360F3E705F108032022304609F090
:10CE20008BFC23682033F4E773B50D4604460021DC
:10CE30001646284640F273120DF0BCFA052322462E
:10CE400001A928460193FFF76FFF019B04F19002AF
:10CE5000053301A928460193FFF766FF019B04F5FE
:10CE60009072063301A928460193FFF7B3FF019B97
:10CE700004F59872063301A928460193FFF7AAFF2B
:10CE800094F840315C2B28BF5C238DF803304EB9F9
:10CE90000DF1030301990722284609F04DFC019B7F
:10CEA00007330193002604F241149DF803300199E1
:10CEB0009E4203D30731C80802B070BDA3190822EF
:10CEC000284609F039FC019B083301930136ECE751
:10CED00000487047A8E601080121884238BF08468B
:10CEE0000CF042BEFFF7F8BF08B10CF041BE70472E
:10CEF000FFF7FABF10B4026854681A4623465DF87B
:10CF0000044B1847002070470120704700207047ED
:10CF100000207047002070477047000000207047D5
:10CF200000207047704700007047000037B5054685
:10CF30000C468322011D01A800F03CF9611EC9B214
:10CF400002299EBF05EBC1010023C1E9073301A8F7
:10CF500000F04CF903B030BD2DE9F7431E461B88A5
:10CF60005B070546884620D4011D422201A800F037
:10CF700021F92C4605F118094C4513D0E3696BB132
:10CF80002B6828465B6C98473388276AC1B243F008
:10CF90000403E0694246B8470834EDE7236A002BF2
:10CFA000EED1F9E701A800F021F9012003B0BDE8B6
:10CFB000F08300007FB56D4685E806000446011D3C
:10CFC000712203A81E4600F0F5F821460022C86928
:10CFD000D3B288B9086A78B995E8030004EBC202B5
:10CFE0001C32013382E803000124337003A800F0EF
:10CFF000FDF8204604B070BD0132032A01F108019A
:10D00000E5D10024F2E700002DE9F04F2DED028B71
:10D010008BB004468B465322011D01A8BDF85880F1
:10D020009FED258B00F0C6F8254604F1180900276E
:10D0300008F0040AA94536D0EB690BB92B6A63B135
:10D04000BAF1000F0BD1236820465B6C984743462A
:10D05000C1B25A46D5E90706B0470835EAE7002FBE
:10D06000FBD18DED028BADF810705B4605AA0BF17C
:10D07000080C18685968174603C7083363453A46D1
:10D08000F7D1186838609B88BB8004F06BFF0423DD
:10D09000ADF810302368CDE902019B6C02A920464F
:10D0A00098470127D9E701A800F0A0F801200BB0AC
:10D0B000BDEC028BBDE8F08F000000000000000016
:10D0C000082817D90C280CD910280CD914280CD9E9
:10D0D00018280CD920280CD930288CBF0F200E20FE
:10D0E0007047092070470A2070470B2070470C20BA
:10D0F00070470D2070470000082817D909280CD068
:10D100000A280CD00B280CD00C280CD00D280CD0E1
:10D110000E2814BF4020302070470C20704710208C
:10D120007047142070471820704720207047000077
:10D13000436818478368184710B5024C8260C0E9FD
:10D14000004110BD40E70108007B00F0010070477E
:10D15000704700008160828070470000826838B5A7
:10D1600004465AB1037B13F0010507D143F00103D4
:10D1700003739047237B65F30003237338BD0000DE
:10D1800010B5044B1B680446986A03681B699847EE
:10D19000204610BD3825002010B5054B1B680446FD
:10D1A000986A036800211B699847204610BD00BF9C
:10D1B00038250020F8B50C4B01601E680446B06AA3
:10D1C00003681B6C17469847054610B1F36AA3F82D
:10D1D0004270206803689B6898471DB1F36A00227B
:10D1E000A3F842202046F8BD3825002010B504469B
:10D1F00000680368DB689847204610BDC181B1FA1A
:10D2000081F0400970470000C089704770470000F6
:10D2100000207047704700007047000000207047F2
:10D2200000207047704700004FF4B4507047000072
:10D230000020704700207047002070470020704792
:10D2400000207047007B70477047000007B50368F7
:10D250008DF80710DB6801220DF10701984703B034
:10D260005DF804FB08B5036801225B6A9847002853
:10D27000D4BF0020012008BD07B503680DF10701E8
:10D28000DB69984720B19DF8070003B05DF804FB07
:10D290004FF0FF30F9E7000013B50446084601914E
:10D2A000FDF74CFF23680199DB680246204602B077
:10D2B000BDE810401847000004F054BE10B44468A4
:10D2C0002CB903685DF8044BD3F880301847002070
:10D2D0005DF8044B7047000082681AB90368D3F800
:10D2E000903018470020704782681AB90368D3F855
:10D2F000943018470020704730B4456825B9046859
:10D30000E46FA44630BC604730BC704700231A4627
:10D31000FFF7F2BF10B484680CB19C4206D10368D9
:10D320005DF8044BD3F8843092B2184700205DF8C2
:10D33000044B70470023FFF7EDBF000001390129BE
:10D340008CBF0020012070470020704700207047EC
:10D35000002070477047000000230B7070470000EA
:10D3600070470000704700000020704700207047A1
:10D3700000207047704700004368C26893423CBF7A
:10D380008268D15443680133436001207047000034
:10D39000F8B505460C468F180026BC4207D02B680E
:10D3A00014F8011B9B68284698470644F5E7304669
:10D3B000F8BD000000207047002070470020704733
:10D3C0000020704738B590F89C308B4204460D46DB
:10D3D0000CD080F89C1004F0C3FD2368C4F8A000B2
:10D3E0005B682046984708B984F84D5038BD000066
:10D3F0007FB50D461446194600267AB1531E0B4AD6
:10D400006846CDE90026089ACDE9025300F08EF86F
:10D410000198844204D92E5404B070BD1346EEE73F
:10D42000002CF9D02C4404F8016CF5E764E70108FE
:10D4300008B410B585B007AC54F8043B00940394CD
:10D44000FFF7D6FF05B0BDE8104001B070470000FF
:10D4500070B5044602F0D8FC5E224FF4000102F0E1
:10D46000BFFC0D4E0D4B1D6833783BB9E86A0422B2
:10D470002146483004F078FD01233370EB6A2A22FC
:10D4800083F84620EB6A93F89C301BB90448214688
:10D4900004F03CFD70BD00BFBA35002038250020E7
:10D4A00048E7010807B503680DF10701DB699847F4
:10D4B00020B19DF8070003B05DF804FB4FF0FF308A
:10D4C000F9E70000F8B506460F4614460025AC42C1
:10D4D0000AD0336830469B699847431C01D12846DF
:10D4E000F8BD78550135F2E72046F9E70EB403B5EB
:10D4F00003AA036852F8041B5B680192984702B0C4
:10D500005DF804EB03B0704700F010B813B50446A3
:10D5100008460191FDF712FE23680199DB68024677
:10D52000204602B0BDE81040184700002DE9F04F3A
:10D530002DED028B06468DB0904691F80090B9F122
:10D54000000F00F0DE82B9F1250F08D04B1C0393C9
:10D55000336849469B68304698470399EDE791F850
:10D5600001908B1CB9F1250F0393F1D00025AA4639
:10D570002C461F2C3BD8B9F12B0F2DD01CD8B9F15C
:10D58000200F2BD0B9F1230F2ED0A9F13003DBB23D
:10D59000092B36D860064BBF05EB85050AEB8A0AD6
:10D5A00003EB450503EB4A0A4EBF05F0FF050AF001
:10D5B000FF0A44F0200407E0B9F12D0F11D0B9F1B2
:10D5C000300FE2D144F00104039B13F8019B039355
:10D5D000B9F1000FCDD126E044F0020444F0040478
:10D5E000F2E744F00804EFE744F01004ECE77F2C86
:10D5F000CBD9230617D5B9F16C0F14D144F480743C
:10D60000E2E7B9F12E0F05D1620600F17A8244F00B
:10D610004004D9E7B9F16C0F02D144F08004D3E79C
:10D62000B9F1680FD0D0A9F14503022B61D809F1F7
:10D63000200944F010045FFA89F908F1070828F07E
:10D640000708F8E80201FDF7A1FA14F0400F08BF3F
:10D65000062524F0C004B9F1650F08EE100AA4B243
:10D6600050D144F0400427060DD59FED977AF0EE97
:10D67000C87AF4EEC77AF1EE10FAC2BF4FF63F73E4
:10D68000234043F0400414F0800346D03B2DA946CC
:10D6900028BF4FF03B0909F101095FFA89F9072713
:10D6A0001722002106A802930CF084FE4A46394650
:10D6B00006A8B0EE480A04F049FE9DF81830019320
:10D6C00003F00902012A029B83462FD0A0072FD422
:10D6D00014F0040F0CBF00222022019911F00C0756
:10D6E00058D0002A40F0AB82BAF1030F50D8174649
:10D6F00037E0A9F16503022B00F25B8124F01004EE
:10D70000A4B29AE7B9F1660F02D144F08004AAE707
:10D71000002DA8D0013DEDB2A5E70A2D83BF0A2553
:10D7200099462F462F4698BF9946B9E72D22D4E750
:10D730002B22D2E70427AAEB07072107FFB20AD45E
:10D74000336802929B6820213046013F984717F0CA
:10D75000FF07029AF4D122B1336811469B68304624
:10D760009847019B594D13F0080F594B08BF1D46B0
:10D77000013D04F0100415F8011F002900F0B580E8
:10D780000CB12039C9B2336830469B689847F2E73C
:10D790000327D0E7CDF808B0002B36D0019BD94441
:10D7A000DB065FFA89F907D59DF81930312B04BFE4
:10D7B00009F1FF395FFA89F94FFA89F3002B44DD4B
:10D7C000B9F1080F28BF4FF0080914F08003049343
:10D7D0001ABF2BEAEB730133052302B101330DB1FC
:10D7E000691C0B449A45C4BFAAEB0303DFB214F0D3
:10D7F000090F2FD177B3336805929B6820213046FB
:10D80000013F9847FFB2059AF4E76006DDD45D4515
:10D8100004DB1BF1040FA8BF44F080046B1C06A9B5
:10D820000B4435B113F80119302902D1013DEDB295
:10D83000F7E72106C9D505F101095D455FFA89F9C8
:10D8400006DDA5EB0B05EDB2BFE74FF00109BCE724
:10D850000025BAE722B1336811469B6830469847E5
:10D86000220708D43FB1336830219B683046013F1E
:10D870009847FFB2F6E7049B002B47D02BEAEB74E6
:10D88000ABEB040A06AB9A44ABEB09096D42A34526
:10D8900017DBA14515DA9AF80110013CA54219DC05
:10D8A000002900F0D281336830469B689847631C9A
:10D8B00004D133682E219B68304698470AF1010A4B
:10D8C000E5E73021E9E700BF7F96184B94E70108B0
:10D8D00090E70108A34507D19DF81930352B0FD8E3
:10D8E00002D1019BDD060BD559B9002F3FF435AEAF
:10D8F000336820219B683046013F9847FFB2F4E728
:10D90000312133689B6830469847EEE79DF819103F
:10D9100031291EBF019B03F0EF03019333683046AA
:10D920009B689847E5B9336814F0100F14BF452180
:10D9300065219B6830469847BBF1000F29DACBF18F
:10D94000000302932D21336830469B6898473021AD
:10D95000029B092B23DD01310A3BC9B20293F7E791
:10D9600033682E219B68304698470235EDB24FF060
:10D9700002094B460CAA1A44336812F8181C9B681B
:10D9800009F101095FFA89F930469847A945F0D1B4
:10D99000C9E702D1019BDC06D1D42B21D3E7336840
:10D9A00030469B6898470299336830319B68C9B20A
:10D9B000A9E7B9F1630F37D0B9F1730F4FD0B9F1BF
:10D9C000640F63D124F0900714F4807FBFB20DF18F
:10D9D00018097BD008F1070222F00702904651682F
:10D9E00058F8080B002904DA404261EB410147F086
:10D9F00080070A234A4600F07BF9A0EB0900C4B275
:10DA00007B0640F19F8027F00109AC421FFA89F99B
:10DA100080F0D28007F01403102B03D127F01107F8
:10DA20001FFA87F9AB468FE058F8043B8DF81830A1
:10DA300001250DF11809200701D4AA451CD84D4431
:10DA40005746A9453FF451AF336819F8011B9B684D
:10DA500030469847002FF4D0013FFFB2F1E758F865
:10DA6000049B14F0400F14BF29464FF0FF31484685
:10DA70000DF076F90546DEE7336820219B683046D5
:10DA80000AF1FF3A98475FFA8AFAD6E7B9F1690FC7
:10DA900098D0B9F1750F27D124F01004A7B20A234A
:10DAA00017F4807FDBB20DF1180944D008F10708A4
:10DAB00028F00708F8E802014A4600F019F9A0EB3F
:10DAC000090027F08007C4B2BFB299E758F8040BE9
:10DAD0000028B8BF40424FF00A024946B8BF47F09D
:10DAE000800700F0B7F888E724F00607B9F1700F57
:10DAF000BFB214D00AD8B9F1580F13D0B9F16F0FD3
:10DB000017D00DB0BDEC028BBDE8F08FB9F1780FE6
:10DB1000F7D1F90601D547F004071023C0E747F015
:10DB20001007F6E7E20601D547F006074FF4047345
:10DB3000B6E70823B4E758F8040B1A46494600F044
:10DB400089F8BCE7A346B94619F0100F41D00CABD9
:10DB5000234413F8193C302B30D129F016091FFA51
:10DB600089F919F0080744D119F0010F35D0DA45C9
:10DB700045D904EB0A05A5EB0B05EDB2336819F0A6
:10DB8000100F9B683FD030213046984719F0040FA2
:10DB900008D0336819F0020F9B6814BF5821782110
:10DBA000304698473368AC429B6839D230213046C2
:10DBB000013D9847EDB2F5E7A346C5E719F0040F1C
:10DBC00002D10BF1010B01E00BF1020B5FFA8BFBB1
:10DBD000C7E719F0860FC4D0F3E73368DA459B68CE
:10DBE0000FD9202130460BF1010B98475FFA8BFBD0
:10DBF000F3E7DA4505D9AAEB0B07FFB2BEE72546E6
:10DC0000BCE70027BAE719F0860FCBD019F0020F56
:10DC100014BF2B21202119F0800F18BF2D21BFE741
:10DC2000651E06AB53FA85F5336815F801199B6834
:10DC3000013CE4B230469847002CF5D155E6BAF1E4
:10DC4000040F3FF677AD002786E5A3457FF44DAE80
:10DC500042E600BF082A30B505D10346C008FCD112
:10DC600030330B700DE0102A0DD100F00F0202F1DD
:10DC70003003392B88BF02F13703000901F8013B5B
:10DC8000F3D1084630BD03460022DCB223F0010385
:10DC9000023342F10002580840EAC270C31842EB56
:10DCA0005202180940EA0270C01842EB1212030A2D
:10DCB00043EA0263181842EB1222030C43EA0243C0
:10DCC0001B1842EB1242D31842F100001B0943EA31
:10DCD0000073C3EB4315C3EB85053034020904EB35
:10DCE000450453EA101001F8014BCED1C9E70000FA
:10DCF000082B30B50AD10346C00840EA4170C90874
:10DD000050EA0104F7D13033137013E0102B13D114
:10DD100000F00F0404F13003392B4FEA101088BFD4
:10DD200004F1370340EA0170090902F8013B50EAA7
:10DD30000103EDD1104630BD20F00104023441F161
:10DD40000003610841EAC3710C1943EB5303210935
:10DD500041EA03710C1943EB1313210A41EA0361F1
:10DD60000C1943EB1323210C41EA0341091943EB3E
:10DD70001343591843F10003C5B2080940EA037080
:10DD8000C0EB4014C0EB84043035190905EB4405A1
:10DD900050EA131302F8015BCED1CBE770EE600AB4
:10DDA000DFED057AF0EEE00AF4EEE70AF1EE10FAA4
:10DDB0004CBF0120002070470000003410B5B4EEC5
:10DDC000400AF1EE10FA2DED028B0446B0EE608AA7
:10DDD000F0EE418A0FD702F017F8A2B24FF480613B
:10DDE00001F0FEFF38EE288AB6EE000A28EE000A9F
:10DDF000BDEC028B10BDB4EEE00AF1EE10FA07D4D0
:10DE0000B4EE410AF1EE10FAC8BFB0EE410AEFE7F6
:10DE1000B0EE600AECE70000884203DB9042014666
:10DE2000A8BF114608467047094A136849F26900BD
:10DE300099B21B0C00FB01331360064B186844F2C7
:10DE4000506182B2000C01FB0200186080B2704782
:10DE500008230020042300207047000038B505681F
:10DE600004462DB1284604F003F92846FFF73CF894
:10DE7000204638BD13460246014801F019BE00BFD6
:10DE80000E36002013B50422054B019304460146CB
:10DE90000DEB0200FFF7EEFF024B1C8002B010BD3D
:10DEA000FFFF3F000036002007B5502304228DF805
:10DEB0000430412300210DEB02008DF805300623CC
:10DEC0008DF806308DF80710FFF7D4FF0420FFF718
:10DED000D9FF03B05DF804FB00EB0212907B20B980
:10DEE0001BB19289120758BF3F20984008447047E1
:10DEF000430608D4000A08D0054B1B88184214BFFB
:10DF0000012000207047002070470120704700BFAB
:10DF10000436002010B50B4B1A880B4B01301B68E0
:10DF200080B2142404FB0033824207D9DC898C427E
:10DF300003F1140304D0013080B2F5E7002010BDD6
:10DF40000120FCE712360020143600208289836805
:10DF5000D20648BF1B681846704700008289836854
:10DF6000D20648BF1B6818467047000007B5042357
:10DF700000220DEB03010B48019201F079FD9DF8A1
:10DF80000430502B07D19DF80530412B03D19DF86B
:10DF90000630062B01D0FFF787FF012003B05DF8A4
:10DFA00004FB00BF0E36002082894368920705D526
:10DFB0001B68181E18BF01200B6070470120FBE78B
:10DFC00037B58B891446DA070D4605D523684A68AC
:10DFD00013442360012012E09B07FBD50A4B1B680A
:10DFE000142201A902FB0030FFF7DEFF48B10199BE
:10DFF00022686B680A44D3581BB15B1A236003B0D4
:10E0000030BD0020FBE700BF143600202DE9F04FA3
:10E010008BB01F469DF854800691142353430593FB
:10E0200008F10603DBB2054616464FF0000B0793D6
:10E030005FFA8BFA07EB0A1999F80F40002C4CD0C5
:10E04000062C28D1B8F10B0F21D84846FFF77EFFE8
:10E050000446C8B1169B099309AA49463046FFF702
:10E06000AFFF88B11499434652463846FFF734FF54
:10E07000099B0293079B0699CDE90003324623468C
:10E080002846FFF7C3FF18B90BF1010BD0E70020BA
:10E090000BB0BDE8F08F1499434652463846FFF75F
:10E0A0001BFFB0EB953FEFD1C5F30423A342EBD1A7
:10E0B0000B4C059B206809A91844FFF775FF002841
:10E0C000E2D0D9F80430099A1344169A1344069AF8
:10E0D00013602068059B1844DAE72046D8E700BFA4
:10E0E000143600202DE9F04F1F4B5FFA80F8B3F88B
:10E0F00000A0C0F3403348EA03281C4B1E680F46BB
:10E1000087B00546C0F3042B00211FFA81F9CA45E8
:10E1100027D9F3894345344620D1337C062B0FD1D0
:10E120003046FFF71BFFC8B10023CDE90133009350
:10E130004A46034639462846FFF768FF044609E089
:10E140009B450BD105A93046FFF72EFF0028F5D0DF
:10E15000059B3B60204607B0BDE8F08F01311436C7
:10E16000D3E70024F6E700BF123600201436002063
:10E170002DE9F04F98468DB0142353430693484B36
:10E180009DF85890DDF868B004461868069B0E4666
:10E1900018440AA91746FFF707FF00287DD000237F
:10E1A000079309F10603DBB209939DF81CA006EB67
:10E1B0000A15EB7B002B70D0062B3BD12846FFF7CE
:10E1C000C5FE0890002831D0B9F10B0F65D8179B18
:10E1D0000B930BAA29463846FFF7F2FE30B39BF8A3
:10E1E0000030012B59D85A1C0BEB83038BF800200D
:10E1F00041465D6052464B463046FFF76DFE1B9A26
:10E200000899CDE904B2199A0392189A02920B9ACE
:10E210000192099A009203463A462046FFF7A8FF6A
:10E2200000BB9BF80030013B8BF80030079B0133AB
:10E230000793BAE7179A686810440A9A1044A042F4
:10E2400013D14B46524641463046FFF745FE189BD8
:10E250001B9A1860199B1D6000231370104B1868DF
:10E26000069B18440DB0BDE8F08F052BDED1031DD1
:10E270009C4203D000F108039C42D7D11B9B201A7B
:10E280008008187052464B4641463046FFF724FE40
:10E29000189B1860199B1D60E0E70020E2E700BFB3
:10E2A000143600202DE9F04F8BB00025DFF8A4A034
:10E2B000079306460F4690461560254B1B881FFAAC
:10E2C00085FB5B4541D9DAF80000142303FB0B04FE
:10E2D00009A9204694F81090FFF766FE98B3B9F1AB
:10E2E000060F17D12046FFF739FE014658B3149B9D
:10E2F0000593079B0297CDE903830023CDE9003303
:10E300005A463046FFF734FF0446E0B120460BB0D2
:10E31000BDE8F08F0998B04204D1149A00233B6005
:10E320001370F3E7B9F1050F0DD1031D9E4203D021
:10E3300000F108039E4206D1149B301A8008187021
:10E3400000233B60E2E70135B7E70024DEE700BFCA
:10E3500012360020143600202DE9F04798460D882B
:10E36000234B0446C5F30809186809EB890588B0F2
:10E3700000EB850507A92846119E95F810A01746C1
:10E38000FFF712FE20B90025284608B0BDE8F08747
:10E390000021BAF1060FC8F8001013D12846FFF784
:10E3A000DDFD0028EFD0109B0091CDE90383CDE97E
:10E3B00001170B46059601464A462046FFF7D8FE50
:10E3C0000546E1E70798A04202D139603170DBE7EA
:10E3D000BAF1050FD7D1031D9C4203D000F1080309
:10E3E0009C42D0D1241AA408002334703B60CBE7B0
:10E3F000143600200138C0B204289ABF014B185CC3
:10E4000000207047F8E701082DE9F04F2DED028B51
:10E4100083B000240093931DDBB208EE103A05464A
:10E420000E461746A246A0464FF0010BE0B201018E
:10E4300005EB001090F80F90B9F1000F5AD0837BD4
:10E440003F2B02D92E4803F061FD17B1002B08BF06
:10E450003F23C3F1200EA3F1200C2AFA03F208FA9D
:10E460000EFE28FA0CFC42EA0E0242EA0C0212F0FE
:10E47000010FC3F1200CA3F12002E3D10BFA02F249
:10E480002BFA0CFC42EA0C020BFA03F3B9F1060F6B
:10E4900043EA0A0A42EA080813D10B2FD2D8FFF741
:10E4A00055FD814658B16858FCF748FE009B18445A
:10E4B000C3B218EE102A31464846FFF7A5FF0134D3
:10E4C000B4E74846FFF796FF01900028BAD0685895
:10E4D000FCF734FE009B1844C0B2B9F1050F04BF2D
:10E4E0000230C0B21028019BACD8308804300344FD
:10E4F0003380E4E703B0BDEC028BBDE8F08F00BFD2
:10E5000098E701082DE9F04F85B00423DFF89890D3
:10E51000ADF80E3000244FF0140A214B1B881FFA6F
:10E5200084F8434539D9D9F800300AFB08F15D1861
:10E530002F7CB5F80EB0062F23D1B8F1000F02D111
:10E54000184803F0E3FC28460193FFF707FD064651
:10E55000A8B1019B5858FCF7F1FD0022C3B20DF1A0
:10E560000E013046FFF750FF59464046FFF7D2FCF8
:10E570000028E5D1062F02D0AB899B07E0D40134F7
:10E58000CBE73846FFF736FF0028D9D0BDF80E306C
:10E5900004331844ADF80E00E6E705B0BDE8F08F8F
:10E5A0001236002098E7010814360020437803F063
:10E5B0001F021F2A0FD00278C3F3401342EA03233D
:10E5C00040F2FF12934206D000680138C31C94BF8A
:10E5D0000020012070470120704700002DE9F34121
:10E5E000224FDFF8908006460D4604247B88A34224
:10E5F00037D904230DEB03012246384601F038FADF
:10E600009DF80510737881EA0302D20618D196F8B6
:10E6100000C09DF80400C3F34013C1F340124CEA5C
:10E62000032340EA022293420AD13268019B5340FD
:10E6300013EA080F04D12C80012002B0BDE8F0815C
:10E6400001A8FFF7B3FF20B1094B2C801C800020EC
:10E65000F3E701F01F00FFF7CDFE031D1C44A4B239
:10E66000C4E74FF6FF732B80F1E700BF0E360020A2
:10E670000036002000C0FFFF70B50C462046114652
:10E6800015461E460CF06CFB831CAB420AD85F2279
:10E69000225422180330A84206F1580656709CBF37
:10E6A0000022E25470BD00002DE9F74FDDE90D5462
:10E6B00007468A46164609689DF830809B462246E2
:10E6C0009DF83C30009328460CF036FB4FF00009D3
:10E6D0009BF800105FFA89F29142019212D921460B
:10E6E00028460CF03DFBC0B28442019A07D90BEBDF
:10E6F00082025168221A096828440CF01DFB09F1B6
:10E700000109E5E7E6B1214628460CF029FBC3B232
:10E710009C4204D93168E21AE8180CF00DFB009B0A
:10E7200013B9B8F1000F13D0F37B052B10D143467A
:10E7300022462946384603B0BDE8F04FFFF79CBF9C
:10E74000009B13B9B8F1000F02D09AF81030ECE733
:10E7500003B0BDE8F08F0000F0B58BB007AC1F46EA
:10E760000023C4E9013307930DF11303CDE90043FE
:10E77000154606AB05AA0646FFF7EEFD014610B9A1
:10E7800028700BB0F0BD9DF84030069A0195CDE998
:10E7900002739DF81330009330462346FFF784FF41
:10E7A000EFE700002DE9F04F984689B014234B4362
:10E7B000DFF828A1039204460E4604934FF00009A7
:10E7C0005FFA89F52B0108EB0515059395F80FB055
:10E7D000BBF1000F7FD0BBF1060F58F803702AD1B0
:10E7E0003846FCF7ABFC3946024620460CF06EFA80
:10E7F000002869D12846FFF7A9FB0746002863D007
:10E80000039B079307AA29463046FFF7D9FB002848
:10E810005AD0059B58F80300FCF790FC129B00931C
:10E82000079A3B4631462044FFF7BCFF00284BD0F7
:10E8300009B0BDE8F08F394620460CF02DFA88B9B2
:10E84000DAF80000049B07A91844FFF7ADFB002885
:10E850003AD0129B83F800B06868079B1844039B6A
:10E860001844E5E7BBF1050F2ED1102138460CF016
:10E8700077FA5FFA80FB5A46394620460CF048FA90
:10E8800010BB14F90B305F2B1ED10BF1010B14F8E8
:10E890000B30583B022B17D8DAF80000049B07A96D
:10E8A0001844FFF781FB78B16868079B129A1844F7
:10E8B000039B18440423137014F90B30592B06D012
:10E8C0005A2B06D0582BB3D009F1010978E7043050
:10E8D000AEE70830ACE75846AAE700BF1436002080
:10E8E0002DE9F04F8BB0DFF8C8B00291044617460F
:10E8F00000252E4B1B881FFA85FA534552D9142246
:10E9000053465343DBF8002002EB0309D35899F830
:10E910001080B8F1060F33D11021184603930CF084
:10E920001FFA039B5FFA80F84246194620460CF016
:10E93000EFF90646002833D14846FFF70FFB0346A0
:10E9400070B3029A009204EB080032465146FFF77A
:10E9500029FF804620B37FB10DF11303009306AA6F
:10E9600007AB05A9CDE9076605960996FFF79AFC5E
:10E97000069B0BB19B893B8040460BB0BDE8F08FF6
:10E98000194620460CF088F950B9029B07A983F874
:10E9900000804846FFF708FB20B1DDF81C80EBE75C
:10E9A0000135A6E74FF00008E6E700BF1236002069
:10E9B00014360020F0B5304D87B040F2A512029019
:10E9C0008DF80C1006460C4601A8291DFEF7F2FB37
:10E9D000052204A9286803F091FC074601A8FEF768
:10E9E00005FC052F06D1049BB34203D19DF81430DA
:10E9F000A3423ED0214E224F4FF4B072314601A8BF
:10EA0000FEF7D8FB286803F09DFB042821D928686D
:10EA1000052202A903F00CFC431F5C425C4101A8E3
:10EA2000FEF7E4FB2CBB3C68E36A93F89C3093B997
:10EA3000A06A036801211B699847A06A03684FF424
:10EA4000FA719B689847A06A036800211B69984780
:10EA5000D2E70024E3E7A06A03681B6C984700280C
:10EA6000E6D001F0D1F940F2FA424FF4801101F002
:10EA7000B7F907B0F0BD00BFD8350020DC35002065
:10EA8000382500202DE9F341154E164FC92406F113
:10EA90000408013CA4B2FCB140F24B12414601A86B
:10EAA000FEF788FB306803F033FB054601A8FEF74C
:10EAB0009DFB042D10D93D68A86A03680A211B69D3
:10EAC0009847A86A03680A215B689847A86A0368A0
:10EAD00000211B699847DCE702B0BDE8F08100BF68
:10EAE000D83500203825002000B58BB00023CDE9B3
:10EAF0000733049309930DF10D03009305AA07ABA7
:10EB000004A9FFF7CFFB10B3059B23B3DB7BC289BE
:10EB10008DF8182003F01F03C2F300221B0243EA02
:10EB20004233049A43EA82339DF818200DF10E0116
:10EB3000134306A80693FFF751FD40B19DF8193025
:10EB400003F01F03052B03D09DF80D3003B1002007
:10EB50000BB05DF804FB037CD9E70000F0B5144F5F
:10EB60003B8889B006460D46FBB10DF10B0300242E
:10EB7000009304AA05AB03A9CDE9054403940794C7
:10EB8000FFF790FB88B10B4B38881B68A2B290420C
:10EB90000BD91A46013411688E4203F10C03F5D1EA
:10EBA000137A2B70012009B0F0BD0020FBE700BFF5
:10EBB00008360020FC35002013B50DF1070104468E
:10EBC000FFF7CCFF10B92046FFF78EFF02B010BD53
:10EBD0000138032816D8DFE800F002080E13FDEE16
:10EBE000C07A17EE903A0B707047BDEEC00A10EE77
:10EBF000103A0B807047BDEEC00A81ED000A7047E5
:10EC000081ED000A7047000037B5036803F0004348
:10EC100003600A4B1B880C4613B9002003B030BDBB
:10EC2000074D01A92868FFF7BFF90028F5D014B1F6
:10EC30002B681B7C23700198F0E700BF1236002080
:10EC4000143600202DE9F04F8FB09B469DF87030B0
:10EC50000B93142343439DF860901A9D0A93074633
:10EC600088460892002307939DF81CA008EB0A161B
:10EC7000F47B002C00F0BC80B089FFF739F9002844
:10EC800000F0B380062C2FD13046FFF75FF9044621
:10EC9000002800F0AA80199B0D930DAA3146384632
:10ECA000FFF78EF9002800F0A0804B4652465946E7
:10ECB0004046FFF711F91D9A05920B9A04921B9A90
:10ECC000CDE902520D9A019209F10602D2B2034631
:10ECD00000922146089A3846FFF7B4FF002800F05A
:10ECE00084800FB0BDE8F08F089B1B780993002B40
:10ECF0003CD02B8867F308032B8052464B4659467D
:10ED00004046FFF7E9F83B4B03EA40302B6823F01D
:10ED1000FF4323F4FF0323F4FC4318431B9B2860A9
:10ED200003B11C70344B18680A9B0DA91844FFF7F7
:10ED30003BF9002859D00D9A73681344199A981812
:10ED40000B9A002ACDD02D4A1278002AC9D0F27B26
:10ED5000012AC6D1B2895207C3D5199A9B56002BF6
:10ED6000BFD1EB7843F08003EB70BAE74B465246D5
:10ED700059464046FFF7B0F82B68C3F35133984229
:10ED800033D1089A0123137095F90330002B06DA6A
:10ED9000EB78099A62F3C713EB701046A1E7052CD4
:10EDA00023D16B78C3F34302022A1ED8013262F3E7
:10EDB00044036B701B9B13B11B9A042313700E4BFF
:10EDC00018680A9B0DA91844FFF7EEF868B170683F
:10EDD0000D9C95F801B0199B2044CBF3430B1844CC
:10EDE0000BF1FF3B00EB8B007BE7079B01333AE71E
:10EDF000204676E700E0FF7F143600200C23002039
:10EE00002DE9F04F8BB0DFF8EC90048807920022D8
:10EE10008DF82720B9F800201F46C4F308039A4252
:10EE200005460E461C4662D9DFF8CC801BB2D8F8E6
:10EE3000001003EB83039A0001EB83031B7C052B7B
:10EE400018D14378C3F34301022915D8013161F386
:10EE5000440343700EB104233370D8F8001068786F
:10EE60000A44C0F34300431E506800EB83000BB01C
:10EE7000BDE8F08F062B04D001340123A4B28DF835
:10EE800027304FF0140B4FF0000AB9F80030A342BE
:10EE90002DD9D8F800200BFB04229089FFF728F821
:10EEA000B8B1117C062917D11046FFF757F8014673
:10EEB00078B1079B0597CDE90363CDE901A5CDF8AE
:10EEC00000A000230DF127022046FFF7BBFE00281B
:10EED000CDD10134A4B2D8E72B68C4F3080403F001
:10EEE000004323432B6006B131705068BFE7002018
:10EEF000BDE700BF123600201436002073B505466A
:10EF00000C461646334601220DF107012846FFF74D
:10EF100077FF28B19DF80730042BF3D804B1237094
:10EF200002B070BDF8B514460746002220460E46D2
:10EF3000FFF76AFE002540B1BD4206D000223146EF
:10EF40002046FFF7DBFF0135F5E7F8BD013903295E
:10EF50000BD8DFE801F00204060800F011BD00F054
:10EF600047BD00F065BD00F0E1BC9FED010A7047B0
:10EF70000000C07FB4EE400AF1EE10FA10B504466E
:10EF80000CD69FED327AF0EEC07AF4EE477AF1EECD
:10EF900010FA03DC042902D180ED000A10BD032918
:10EFA00019D1B5EEC00A9FED2A7ADFED2A7A9FEDDE
:10EFB0002A1ADFED2A0AF1EE10FA58BFF0EE477A6E
:10EFC00030EE270A40F6C900FEF7F8FEBDEEC00A93
:10EFD00084ED000AE2E702291AD1B5EEC00A9FEDDE
:10EFE0001C7ADFED1C7A9FED1E1ADFED1E0AF1EE92
:10EFF00010FA58BFF0EE477A30EE270A40F6CE00FE
:10F00000FEF7DCFEBDEEC00A10EE103A2380C5E725
:10F010000129C3D1B5EEC00A9FED0D7ADFED0D7A5F
:10F020009FED111ADFED110AF1EE10FA58BFF0EE64
:10F03000477A30EE270A40F6D300FEF7BFFEFDEE1A
:10F04000C07A17EE903A2370A8E700BFFFFF7F7FDA
:10F050000AD7233C0AD723BC0000004F000000CF92
:10F0600000FEFF46000000C70000FE42000000C393
:10F070002DE9F3411D4690F90030232B0F469046B1
:10F080004FF000042CD01749019401AA0CF01AFD8E
:10F09000064618B9002002B0BDE8F081FCF74EF832
:10F0A0001028F7D80F4901AA20460CF00BFD0028C4
:10F0B000F0D021460CF082FC0A4988ED000A01AA32
:10F0C0003E6020460CF0FEFC30B10749FCF72CF8FE
:10F0D00010B901202870DEE700232B700120DAE749
:10F0E0002046D8E7ACE70108B3E701082DE9F04373
:10F0F0004FF000089DB005460E461746A2F8008066
:10F10000002E35DDB2B200239CB2A24203F1010908
:10F1100002D9EB5C0A2B29D1632C28BF6324224639
:10F12000294603A80BF038F91CAB1C44A6EB0906D2
:10F1300004F8648C9DF90C30232B4D44E0D0002B57
:10F14000DED00DF1020302AA01A903A8FFF790FF88
:10F150000028D5D0019800220DF10301FFF7C0FB74
:10F160000028CDD03B8801333B80C9E74B46CBE735
:10F1700001201DB0BDE8F0832DE9F04FDFF82881B4
:10F180000546D8F800009FB00E4608B1FDF7B0FE66
:10F19000434FDFF818A1DFF8189100240DF10A029F
:10F1A00031462846C8F800403C80AAF80040A9F83B
:10F1B0000040ADF80A40FFF799FF00286DD0BDF878
:10F1C0000A300C205843FDF78DFEC8F8000010B936
:10F1D000344802F09BFEBDF80A303B80A346BDF8E0
:10F1E0000A30A34257D9002E55DDB1B2002297B2A2
:10F1F000B94202F1010302D9AA5C0A2A49D1632F5C
:10F2000028BF63273A46294605A801930BF0C4F8A6
:10F210001EAB1F44019B07F864BCF61A1D449DF900
:10F220001430232BDBD0002BD9D002AB04AA03A9C6
:10F2300005A8FFF71DFF0028D1D0039800220DF18B
:10F240000901FFF74DFB07460028C8D00C2303FB3C
:10F2500004F2D8F800309850D8F800301344049ADB
:10F260005A609DF808201A7222B1B9F800300133B3
:10F27000A9F8003001343846A4B2FFF735FC002865
:10F28000ADD19DF809109DED040A3846FFF772FED6
:10F29000A5E71A46ABE7AAF800301FB0BDE8F08F2B
:10F2A0000A360020C0E70108FC350020083600209F
:10F2B000F835002002460248418A1430FFF75CBF4F
:10F2C00000E80108024B5B8A0BB1FFF7F3BF704700
:10F2D00000E8010830B5002085B0FFF7F3FF214BAF
:10F2E0001A7872B901221A701F4B204A1B680292C9
:10F2F000986A1F4A0368039204AA12E906009B6AEF
:10F3000098471C4D04246B88A34229D90423224624
:10F310006946284600F0ACFB6846FFF747F918B18C
:10F32000154B1C8005B030BD009801A9FEF7DAFE30
:10F3300060B19DF8010000F01F00FFF75BF8221D8F
:10F340000346019992B2284600F092FB9DF8010015
:10F3500000F01F00FFF74EF804300444A4B2D2E7D7
:10F360000020DFE70C36002038250020BB350020C8
:10F370009DF800080E3600200036002070B50E4BB8
:10F380001E880E4B1B68002294B2A64209D91C4667
:10F3900001322568854203F10C03F5D194ED010A91
:10F3A00070BD8B891B0649BF8B6891ED020AC01A9C
:10F3B00090ED000AF4E700BF08360020FC3500207D
:10F3C0002DE9F04105460F464FF000085FFA88F33B
:10F3D00007EB0311CC7BDCB1042C0BD84E682E4418
:10F3E0003046FFF7CBFF31462046FFF7F1FB08F12F
:10F3F0000108EBE7052CFAD14C682C442046FFF7B6
:10F40000BDFF84ED000A84ED010A84ED020AEEE7F7
:10F41000BDE8F08170B50E4B1E880E4B1B680022B4
:10F4200094B2A64209D91C4601322568854203F1EF
:10F430000C03F5D194ED010A70BD8B891B0649BF01
:10F440008B6891ED020AC01A90ED000AF4E700BF44
:10F4500008360020FC3500202DE9F0418AB0002359
:10F46000CDE90733039309930DF10903009304AA2F
:10F4700007AB03A90446FEF715FF054620B9002691
:10F4800030460AB0BDE8F081049B002B3AD0DB7B0C
:10F49000EA898DF8142003F01F03C2F300221B0237
:10F4A00043EA4233039A43EA82339DF814200DF174
:10F4B0000A01134305A80593FFF790F8064658BBC9
:10F4C00006A92846FEF770FD0028D9D09DF81570D2
:10F4D0000499DDF8188007F01F07B9B19DF81C30BA
:10F4E00093B1089A012B556802D0099B5B681D44B3
:10F4F0002046FFF743FF4968414429443846FFF757
:10F5000067FBBDE7037CC3E73546F1E729462046A4
:10F51000FFF780FF4146F1E79DF815009DF809309F
:10F5200000F01F02052A0FD0002BA8D100F01F0009
:10F53000FEF760FFBDF80A200432034692B221466E
:10F54000044800F095FA9BE7002BEFD0A4EB83046E
:10F55000ECE700BF0E3600202DE9F04385B0FEF742
:10F5600005FD134E134F00254FF014083288ABB23F
:10F570009A4219D91C463B6808FB043494F8109051
:10F58000B9F1040F0ED803A92046FEF70DFD48B1CE
:10F59000039801902146FFF73DFF01980146484638
:10F5A000FFF716FB0135E1E705B0BDE8F08300BFCA
:10F5B00012360020143600202DE9F347DFF88C9036
:10F5C0001F4940F678226846FDF7F4FDB9F800704F
:10F5D0002FB11C4B1A881C4B1B889A4228D0194EFD
:10F5E000194D05244FF00008B9F800701FB132889A
:10F5F0002B889A421CD0013C14F0FF0418D0002242
:10F60000114601A83788CDF80480FFF7FDFA4FF0C6
:10F61000000A1FFA8AF30AF1010A28B100221146F2
:10F6200001A8FFF76BFCF4E7A9F800302F80DBE7B7
:10F630006846FDF7DBFD384602B0BDE8F08700BF45
:10F64000BC350020F63500200636002002360020AA
:10F65000024A138801331380704700BFF63500203B
:10F660002DE9F0412DED028B90B00023CDE9083358
:10F6700005930A930DF1110300930E4608AB06AAF9
:10F6800005A90446FEF70EFE0546D8B10699F1B16C
:10F69000CA7BEB898DF81C3002F01F02C3F30020F7
:10F6A0001302059A9DF8117043EA403343EA82330E
:10F6B0009DF81C201A43C3F30423052B079200F086
:10F6C000868037B110B0BDEC028BBDE8F081027CC2
:10F6D000DFE7012B05D121B18B895B0701D5FFF74E
:10F6E000B7FF274677E0BDF812204FF6FF739A4226
:10F6F0000AD14C4B83F800804B4B4C491B689869EE
:10F7000003681B689847DDE79DF81D1001F01F0195
:10F71000042925D99DF81D00BDF81220444900F0A8
:10F720001F00FEF767FE4988131808338B424AD240
:10F730000432104480B2FEF7A5FB9DF81D0000F0D6
:10F740001F00FEF757FEBDF812100431024689B2C1
:10F750003846FEF78FFBBDF81210042207A85EE0C2
:10F760002046FFF7F3FB0699F0EE408A71B1204680
:10F77000FFF704FEB0EE408AF0EE400AB0EE680AF1
:10F78000FEF70CFB38B1002EC4D19BE7294620467A
:10F79000FFF740FEEEE7002EBCD19DF81D3003F0D0
:10F7A0001F03032BB6D09FED230A38EEC88AF0EE74
:10F7B000E88A68EE808AB0EEC88AB4EEE88AF1EE94
:10F7C00010FAA7D57EE7174B01221A7094E7002F95
:10F7D00087D0A4EB870711234FF00108CDE9023849
:10F7E0000BAB01939DF81130009329462046069AF1
:10F7F00008ABFEF759FF0DF1120107A8FEF7EEFE68
:10F8000000283FF470AF9DF81D0000F01F00FEF7C8
:10F81000F1FDBDF812100431024689B23846FEF7F8
:10F8200029FB4FE7F435002038250020E8E70108E0
:10F830000E36002017B7D1387FB5164D2E1D40F279
:10F840007F12314601A8FDF7B5FC286802F060FC84
:10F85000042812D92868052202A902F06BFD431F73
:10F860005C425C4101A8FDF7C1FC44B19DF80C105D
:10F8700002980122FFF7F4FEE1E70024F2E7064BCD
:10F880001B68986A03685B6B984708B1FFF794FEA2
:10F8900004B070BDD835002038250020FFF7CCBF5C
:10F8A00010B50446FDF720FB204610BD38B51148C1
:10F8B000114D01F021FD114A11490E480AF042FD97
:10F8C0002846002340F8043B01F016FD1420FDF704
:10F8D00003FB044610B19B2102F0B8FB0949074A1B
:10F8E00005482C600AF02EFDBDE83840064800218E
:10F8F00000F0B6B8BC350020D83500201C3F0020F1
:10F9000059DE00085DDE00080E360020D1ED007AD9
:10F9100090ED007AF4EE477AF1EE10FA04D0C0EDE3
:10F92000007A0121FFF746B87047000090ED000A09
:10F930007047000091F9001090F900309FED097AAE
:10F9400001705B1A07EE903AF8EEE77AF0EEE77A8C
:10F95000F4EEC77AF1EE10FA4CBF01210021FFF757
:10F9600029B800BF0000003491F9002090F9001080
:10F97000914203D002700121FFF71CB870470000CC
:10F9800090F9003000EE103AB8EEC00A704700005F
:10F9900038B504460D46FFF70FF910B9B5F9003038
:10F9A000238038BDB1F90010B0F900309FED097A1D
:10F9B00001805B1A07EE903AF8EEE77AF0EEE77A0C
:10F9C000F4EEC77AF1EE10FA4CBF01210021FEF7E8
:10F9D000F1BF00BF00000034B1F90020B0F9001001
:10F9E000914203D002800121FEF7E4BF704700007E
:10F9F000B0F9003000EE103AB8EEC00A70470000CF
:10FA000038B504460D46FFF7D7F808B92B682360D0
:10FA100038BD00000B680360704700000A68016889
:10FA20008A4203D002600121FEF7C4BF7047000084
:10FA300090ED000AB8EEC00A7047000008B5064B0A
:10FA40001B68586903685B68984720B9BDE808409F
:10FA5000024801F0C7BC08BD3825002014EA01089F
:10FA6000017011B10023438070474FF44873FAE7E7
:10FA700070B51C460378A3B9B2F5487F11D212FACB
:10FA800084F3B3F5487F094B1B685869C8BFC2F5BA
:10FA900048750368D4BFA5B2ADB29E682B46B04787
:10FAA000641BB4FA84F0400970BD00BF3825002003
:10FAB00070B51C460378A3B9B1F5487F11D211FA8D
:10FAC00084F3B3F5487F094B1B685869C8BFC1F57B
:10FAD00048750368D4BFA5B2ADB2DE682B46B04707
:10FAE000641BB4FA84F0400970BD00BF38250020C3
:10FAF00010B5044B044918600446FFF761FC20462A
:10FB000010BD00BF1836002088EA010890F82330A5
:10FB100063B9012380F82330054800684FF400736F
:10FB2000006C80224FF4E131FDF7E6BB704700BF67
:10FB300038250020002850DD6F2846D01BDC132814
:10FB400045D00EDC431E082B11D8082B33D8DFE834
:10FB500003F0410532363232323239004FF416604A
:10FB60007047392839D064283AD026283AD04FF443
:10FB70007A7358437047B0F5FA7F36D010DCB0F591
:10FB8000807F34D006DC732834D0E628EFD14FF4E0
:10FB900061307047B0F5E67FE9D14FF4E12070475E
:10FBA00040F2DC53984228D0B0F5FA6F27D040F2EB
:10FBB0009933984225D0B0F5FA6FD8DD70474FF4ED
:10FBC000965070474FF4165070470F4870474FF4E7
:10FBD000964070474FF4966070474FF4614070470D
:10FBE0000A4870474FF416407047094870474FF471
:10FBF0007A3070474FF4E130704706487047064846
:10FC000070474FF46120D9E7FCB10100A0860100E4
:10FC100020A1070060E3160080841E000068FFF743
:10FC200089BF00000E4B70B51D68CBB2092B0C4686
:10FC300012D8103355F8232000EBC1031168104689
:10FC40004E6B9988B04750B9A869064903682246A7
:10FC50001B68BDE87040184700231B68FFDE70BDBD
:10FC60003825002034EA01082DE9FF41FF238046B2
:10FC700003A921308DF80C30FFF776FE4046FFF7E0
:10FC800045FF564B1B68019308F1080401267327B2
:10FC9000019A06F1100352F82350E6717DB3B1B218
:10FCA0004046FFF7BFFF94F906300133332B00F2D3
:10FCB0008C80DFE803F0241A1A1A2C3335353D47BF
:10FCC0008A338A528A8A245A8A8A698A8A4C8A7D25
:10FCD0008A8A8A8A8A248A8A8A8A8A8A8A8A8A8AEA
:10FCE0008A8A1A8A8A8A8A8A8A242046FFF796FF95
:10FCF0004FF48073014680222846FDF7FDFA013655
:10FD0000042E04F10804C3D104B0BDE8F081092336
:10FD100003A920460393FFF77DFEF0E73923F7E7B9
:10FD20002046FFF77BFF102301464FF48072E3E784
:10FD300003A920460397FFF76DFE80231A464FF470
:10FD4000E131D9E703A920460397FFF763FE204678
:10FD5000FFF764FF80230146CDE7092303A9A01D17
:10FD60008DF80C30FFF7E6FDC9E703A9204603979D
:10FD7000FFF750FE2046FFF751FF1E2301461A46AB
:10FD80002846FDF7B9FA0DE02046FFF747FF80232C
:10FD900001461A462846FDF7AFFA2B680121DB6CB5
:10FDA000284698472B680021DB6B28469847A6E732
:10FDB00003A920460397FFF723FE2046FFF72EFFF7
:10FDC000102301464FF40072DAE72046FFF726FFC2
:10FDD00001462846FDF79AFA91E700BF3825002032
:10FDE00010B5036802811943436801600133436021
:10FDF000044B1B68DC6AA162D96A40688885DB6AAB
:10FE0000DA8510BD38250020004870471C360020D8
:10FE100008B50449FBF788F90028034818BF0020FB
:10FE200008BD00BFE8EA0108D02202082DE9F04130
:10FE30008846FFF7EDFF054608B9002409E086680B
:10FE4000701C09F061FE04460028F6D026B9C8F8F7
:10FE500000602046BDE8F0814FF4A16009F054FE37
:10FE6000064618B9204609F083FEE6E7002211464F
:10FE700000F040F92B6933606A68F46113447360E1
:10FE8000AB68B361304600F045F90746304609F0EB
:10FE90006FFE002FE6D1AA682146384602F0E2FB49
:10FEA000EB689842DED1AB68C8F80030D1E70000BB
:10FEB00009F05EBEF0B50D46164689B0202200213D
:10FEC00004460AF077FA2A467019824207D012F8DF
:10FED000011B34F81130013324F81130F5E72146C5
:10FEE000002321F802396A4604F11E0031F8027F2E
:10FEF00022F8023B81423B44F8D10023B3420ED0AA
:10FF0000E95C51B108AA02EB410131F8202C501CE8
:10FF1000103221F8200C24F812300133EEE709B03A
:10FF2000F0BD000010B5D0E900329342044603D280
:10FF30005A1C0260187810BD83683BB190F82920E4
:10FF400022B99847031E01DBD8B2F4E7012384F8F5
:10FF500029300020EFE7000010B503695A1E04465F
:10FF6000026123B9FFF7DEFF0723E0602361E06849
:10FF70004308E36000F0010010BD00002DE9F041EE
:10FF80000746164661B1012505FA01F800244545EA
:10FF900007D23846FFF7E0FF00B12C446D00F6E7CA
:10FFA0000C463019BDE8F0812DE9F8430023804666
:10FFB0000E468F1C01F120091D4640465C00FFF7EC
:10FFC000CBFF4F4504440FD037F8023B5A19E31AD0
:10FFD00008D52544B5F5907F06D2103536F81500C2
:10FFE000BDE8F8831546E8E76FF00200F8E7000087
:10FFF0002DE9F04F0E46D3B00521904640F2011294
:020000040801F1
:100000000446FFF7BBFF0122052105462046FFF706
:10001000B5FF0422114607462046FFF7AFFF132223
:100020008246002102A80AF0C5F9DFF8C4B04FF0FB
:100030000009D1450BD0002203212046FFF79EFF87
:100040001BF8013B02AA09F10109D054F1E7132280
:1000500002A93046FFF72EFF05EB07094FF0000A13
:10006000CA4538D231462046FFF79EFF00280ADBFA
:10007000112829D012282BD010281ED1BAF1000F38
:1000800004D16FF0020053B0BDE8F08F02AB5344CF
:10009000032213F8013C022120460193FFF76EFF73
:1000A0000AEB000BCB450246EBD8019B194602AB8D
:1000B00003EB0A000AF07EF904E002AB0AF1010B3F
:1000C00003F80A00DA46CBE7032211460023E3E7F0
:1000D0000B220721FAE72A4602A93046FFF7EAFE7B
:1000E00002AB40463A465919FFF7E4FE0020CAE742
:1000F0004023020810B500234FF0FF34C0E901335C
:10010000C0E90F1280F8293003610363C4624364BD
:10011000436310BD2DE9F0479F4DA04EA04F04460C
:10012000E36A013340F094802046FFF715FF002278
:10013000206302212046FFF721FF0128E0627BD1E6
:100140000023A4F84830A4F84A30A4F84C30A4F8AE
:100150004E30A4F85030A4F85230A4F8543018238C
:10016000A4F856309823A4F858307023A4F85A30D5
:1001700004F168024FF4807322F8023B01339BB212
:10018000B3F58C7FF8D104F19802002322F8023BEA
:100190000133902BFAD14FF48C72A4F8B82140F2BD
:1001A0001912A4F8BA214FF48D72A4F8BC2140F2C0
:1001B0001B12A4F8BE214FF48E72A4F8C02140F2A5
:1001C0001D12A4F8C2214FF48F72A4F8C42140F28A
:1001D0001F12A4F8C62104F5E47222F8023B013391
:1001E0009BB2B3F5807FF8D100232022A4F8B2227D
:1001F000A4F8A832A4F8AA32A4F8AC32A4F8AE321B
:10020000A4F8B03204F5327222F8023B0133202BFD
:10021000FAD1636B002B40F08A8004F1480120463C
:10022000FFF7C2FE94F82930BBB9FF2859DCE36917
:100230005A1CE261C0B240E0022809D104F52A72DA
:1002400004F148012046FFF7D3FE002840F09E80CD
:10025000E36A2BB1013B012BDBD96FF0020095E083
:10026000D4F834A0BAF1000F1CD12046FFF75AFE93
:1002700081462046FFF756FE09EB00292046FFF78E
:1002800051FE80462046FFF74DFE08EB002383F425
:100290007F4383F0FF039945DFD109F101006063DB
:1002A000C4F810A0636B013B6363002B69D0204648
:1002B000FFF738FEE3695A1CE2611870E26B4AB13D
:1002C000636C591C6164D054D4E910329A4201D154
:1002D00000236364A0690138A06100287FF420AF87
:1002E00054E0B0F5807F4CD06FF48073184435F83B
:1002F0001020315C2046FFF741FE04F52A7160634F
:100300002046FFF751FE002840DB264B37F810202F
:10031000195C2046FFF732FEE36B002B29D0226CDC
:10032000904235D8636C181A48BF8018A063E16BFF
:10033000E369A26BF9B1581CE0618A5C1A70E36B47
:100340005BB1626CA16B501C6064595C9954D4E938
:1003500010329A4204BF00236364A36B226C013302
:100360009342A36301D10023A363636B013B6363E7
:10037000B0E74042DAE79A5C1A70E3690133E3615F
:10038000F3E7236B002B3FF4CFAE0120BDE8F087ED
:100390006FF00400FAE700BFE422020820230208FD
:1003A000542302089023020810B4064B064A1B6827
:1003B0000649986903681C68537E127EA4465DF85E
:1003C000044B60473825002000A20008B023020833
:1003D00010B41346026814680022A4465DF8044B6A
:1003E0006047000000F5805090F8810470470000DD
:1003F00000F5805090F87A047047000000F5A55091
:100400007047000000F5805090F9800470470000AC
:1004100050207047302383F3118800F58052D2F8C2
:10042000C434D2F8C0041844D2F8BC341844D2F80A
:10043000A4341844D2F8B4341844D2F8B034184470
:10044000002383F31188704700F58050C0F87C14B6
:10045000012070472DE9FF47054600F580500C4606
:1004600090F87A14BDF830A099B1D0F8A0140131F9
:10047000C0F8A01421688E0006D4217B08290BD96E
:10048000667B0EB10F2907D9D0F8A4340133C0F828
:10049000A4344FF0FF30A4E0302181F31188696D5E
:1004A000D1F8C46016F4001813D0D0F8A8140131A4
:1004B000C0F8A814D0F8AC14002940F09580CDF80D
:1004C00000A021462846FCF79FFD002383F31188F6
:1004D00087E0D1F8C4702668E96CC7F301474FF094
:1004E0004809002E19FB0719B4BF46F08046B60430
:1004F000C9F800602168490044BF46F00056C9F8B9
:100500000060267B390641EA0641C9F8041094F8D8
:100510000DC07E01BCF1000F27D041F44011C9F895
:100520000410D0F8D8140131C0F8D814A91901F575
:100530008451087D40F020000875207BCDE902231E
:10054000FCF7DAFDDDE90223033080105FFA88F161
:10055000814208F101080FDA04EB810C09EB8101FB
:10056000DCF804C0C1F808C0F0E7A91901F584510E
:10057000087D6CF34510DFE7696D0120B840C1F8D4
:10058000CC00A91901F58351C1E90623A7F17C012B
:10059000C9B2204605EB411104F10C0C50F804EBF4
:1005A00041F804EB6045F9D1008808802E4441F2FF
:1005B0009001775006F580560AF0030196F89400F2
:1005C00041F0100120F01F00014386F89410002133
:1005D00081F31188CDF800A021462846FCF714FDD0
:1005E000012004B0BDE8F08700206EE738B5426D09
:1005F000936923F001039361044601F0B1FC0546C1
:10060000636D9B69DB0706D501F0AAFC431BFA2B3F
:10061000F6D9002004E004F58054012084F87A041F
:1006200038BD000030B52DED028B0446A1B00D465B
:10063000302383F3118804F58054022007F072FE02
:10064000D4F8DC341C93D4F8D8341B93D4F8E034B9
:100650001A93D4F8D4341993D4F8D0341893D4F826
:10066000C4341793D4F8C0341693D4F8BC3415931B
:10067000D4F8B8341493D4F8B4341393D4F8B03411
:100680001293D4F8AC341193D4F8A8341093D4F85E
:10069000A4340F93D4F8A0340E93B4F88A349FEDA9
:1006A000248A244AB0FBF2F207EE903AF8EEE77A99
:1006B0001F9267EE887A17EE900AF9F717FFCDE9D7
:1006C0000C0194F890340A9394F88F34099394F8B9
:1006D0008E340893B4F88C340793D4F89834069386
:1006E000B4F8823407EE903AF8EEE77A67EE887A4B
:1006F00017EE900AF9F7FAFECDE9040194F8883470
:10070000039394F88734029394F886340193B4F8F1
:1007100084340093D4F894341F9A0749284601F092
:1007200061FC002383F3118821B0BDEC028B30BD46
:10073000CDCCCC3D40420F00C023020813B500F5DC
:1007400080540191E06E01F0FDFC1F280AD9019947
:10075000E06E202201F06CFDA0F1200358425841C8
:1007600002B010BD0020FBE708B5302383F31188E9
:1007700000F58050C06E01F0B9FC002383F31188AE
:1007800008BD0000002202608281426082607047E2
:1007900010B500220023C0E9002300230446038192
:1007A0000C30FFF7EFFF204610BD00002DE9F047A9
:1007B0009A4688B0074688469146302383F31188CD
:1007C00007F580546846FFF7E3FFE06E01F0A0FCF8
:1007D0001F282DD9E06E2022694601F0ABFD2028AC
:1007E00026D194F87A341BB303AD444605AB2E46AC
:1007F00003CE9E4220606160354604F10804F6D1C4
:1008000030682060B388A380DDE90023C9E90023B4
:10081000BDF80830AAF80030002383F3118853464E
:100820004A464146384608B0BDE8F047FCF794BB5D
:10083000002080F3118808B0BDE8F0872DE9F84F5B
:100840002E4B054640F8043B88462E4600F054FDEA
:100850001822002105F11C0009F0ACFD284B46F8D8
:10086000583B05F582543746183438462037FFF791
:100870008FFFA742F9D105F580544FF48053A66548
:100880000026C4E91736E766012305F5845705F508
:10089000A459666684F8683084F87030183709F116
:1008A00018094FF0000A4FF0000B47E908ABA7F119
:1008B0001800FFF767FF203747F8286C4F45F4D141
:1008C00084F88084A4F88264A4F88464A4F886641C
:1008D00084F88864A4F88A64A4F88C64A4F88E640C
:1008E00084F89064B8F1000F02D0064801F00EFBC6
:1008F000054B6B652846BDE8F88F00BFECE60108A4
:10090000F4250208D82502080064004010B5044B05
:10091000197804464A1C1A70FFF790FF204610BD54
:100920002D3600202DE9F84315460C4600295CD0F1
:10093000022007F0F7FC2E49B0FBF4F78C428CBF85
:100940000A2111214B1EB7FBF1F601FB1671DAB239
:1009500021B1022B1946F5D8002032E0731EB3F501
:10096000806FF9D2C2EBC20808F103014FEAE10E31
:10097000C1F3C701A2EB010C0EF101094FF47A7328
:100980005FFA8CF70EFB033E59FA8CFCBEFBFCFCB5
:10099000BCF5617F17DC1FFA8CF34A1C57FA82F210
:1009A0007243B0FBF2F08442D6D14A1E0F2AD3D84C
:1009B0007A1E072AD0D801202B806E802871697199
:1009C000AF71BDE8F88308F1FF314FEAE10CC1F3E4
:1009D000C701521A0CF1010ED7B20CFB03335EFAB9
:1009E00082F2B3FBF2F39BB2D7E70846E9E700BF18
:1009F0003F420F0030B50D4B0D4D05201C786C4368
:100A00008C420ED15978518099785171D978917171
:100A1000197911715B7903EB83035B00138001206B
:100A200030BD013803F10603E8D1F9E7402602089A
:100A300040420F000B4B10B54FF454720446002196
:100A4000184609F0B7FC084B236440336364D8337D
:100A5000A364F033E364636DE0630022C3F8C02055
:100A600010BD00BF00A4004070A400402DE9F04F6D
:100A700000F580551F4695F88034012B89B0044657
:100A80008946904604D90026304609B0BDE8F08F6B
:100A90009E4A52F8231041B942F8230000F0FAFEB2
:100AA00095F8803400EB8300C4639948C4F834900F
:100AB000017884F8387099B9302383F31188954B05
:100AC0009A6D42F000729A659A6B42F000729A63D6
:100AD0009A6B22F000729A630123037081F31188EC
:100AE00095F879647EB9302383F3118803211520AA
:100AF00007F03AFD0321162007F036FD012385F8A3
:100B0000793486F31188302383F31188626D9369F9
:100B100023F01003936101F023FA8246636D9E690E
:100B200016F0080609D001F01BFAA0EB0A03FA2B15
:100B3000F4D9002686F31188A6E79A6942F00102EB
:100B40009A6101F00DFA8246636D9A69D00706D466
:100B500001F006FAA0EB0A03FA2BF5D9E9E79A6946
:100B600042F002029A61636D4FF0000AC3F854A08C
:100B70008AF31188E86E01F0B9FA04F5835B0BF192
:100B8000180B20220021684609F014FC02A8FFF788
:100B9000F9FDCDF818A06A460BEB06030DF1180E0F
:100BA0009446BCE80300F44518605960624603F1BE
:100BB0000803F5D1DCF80000186020369CF804200A
:100BC0001A71B6F5806FDCD1002304F5A45285F8C4
:100BD000783485F87B34023249462046FFF7A2FE7E
:100BE000064690B9626D936923F00103936101F0A9
:100BF000B7F90546636D9B69D9077FF544AF01F0EE
:100C0000AFF9431BFA2BF5D93DE795F88634C5F8C3
:100C10009494591E95F88734626D013B1B0243EA98
:100C2000416395F8881401390B43B5F884140139F0
:100C300043EA0143D361B8F1000F36D004F5A45262
:100C40000A3241462046FFF7D5FE90B9626D93699E
:100C500023F00103936101F083F90546636D9B69FD
:100C6000DA077FF510AF01F07BF9431BFA2BF5D9BA
:100C700009E795F88F24C5F89884511E95F89024BB
:100C8000636D013A120142EA012295F88E1401398E
:100C90000A43B5F88C14013942EA014242F40002D9
:100CA000DA60636D4FF420629A642046FFF7C2FE5B
:100CB000002385F88134636D6FF040421A65636DDF
:100CC000154A5A65636D44229A65636D0722C3F81D
:100CD000DC20636D03229742DA653FF4D5AE626D86
:100CE000936923F00103936101F03AF90746636DBC
:100CF0009B69DB0705D501F033F9C31BFA2BF6D945
:100D0000C1E6012385F87A34BEE600BF283600200C
:100D10002C360020001002409B0008002DE9F04F07
:100D200000F5A6578BB00446904699464FF0000B4D
:100D300041F2900A1037636DD3F8D43023FA0BF3E5
:100D4000DD0752D504EB4B1151444FEA4B120B799E
:100D500018074AD404F58056D6F8AC340133C6F8E7
:100D6000AC3447E902890B79990648BFD6F8DC34E0
:100D700004EB020148BF0133514448BFC6F8DC34DC
:100D80000B7943F008030B71DB0723D596F87B340E
:100D900003B302A80192FFF7FBFC019A04F5845506
:100DA000154405AB05F1080C286869681A4603C2AA
:100DB000083565451346F7D128681060AA889A80DF
:100DC0000123ADF810302368CDE902899B6C02A99C
:100DD00020469847D6F8D034D6F87C040133C6F8BC
:100DE000D03410B103681B6998470BF1010BBBF1BC
:100DF000200FA0D10BB0BDE8F08F00002DE9F04F1F
:100E00008DB004460F4601F0ADF882468946002FAA
:100E100056D1636DD3F89020920141BF04F5805103
:100E2000D1F8C0240132C1F8C024D3F890201607AD
:100E300003D100200DB0BDE8F08FD3F89050666C60
:100E4000C5F30125482303FB0566E8464046FFF746
:100E500099FC326851004ABF22F06043C2F38A43D2
:100E600043F00043920048BF43F08043009373680F
:100E700013F400131FBF04F5805201238DF80D30C9
:100E8000D2F8E0340EBF8DF80D300133C2F8E034F3
:100E9000F38803F00F038DF80C304FF0000B9DF832
:100EA0000C00FCF729F95FFA8BF3984220D9F2186D
:100EB0000CA90B44127A03F82C2C0BF1010BEEE772
:100EC000012FB6D1636DD3F89820950141BF04F589
:100ED0008051D1F8C0240132C1F8C024D3F8982041
:100EE0001007A6D0D3F89850A66CC5F30125A9E742
:100EF000EFB9636DC3F8945004A8FFF749FC98E874
:100F00000F0007AD07C52B800023ADF8183023680C
:100F10002046CDE904A99B6C04A9984704F58054A8
:100F200058B1D4F8B8340133C4F8B83482E7012F8B
:100F300004BF636DC3F89C50DEE7D4F8BC340133C2
:100F4000C4F8BC34012075E72DE9F04105460F4691
:100F500000F58054012639462846FFF74FFF10B1AF
:100F600084F87B64F7E7D4F8D034D4F87C040133F8
:100F7000C4F8D03420B10368BDE8F0411B691847BC
:100F8000BDE8F081F0B5436D1A6C12F47F0F2BD0E1
:100F900000F580541B6CC4F8D43441F29005002352
:100FA00047194FF0010C00EB43122A445E011179FE
:100FB00011F0020F15D0490713D4B959466DD6F870
:100FC000C8E00CFA01F111EA0E0F0AD0C6F8D010F1
:100FD000117941F004011171D4F8B4240132C4F83C
:100FE000B4240133202BDED1F0BD000010B5254C18
:100FF000254B226802B338B31A6D12060ED5802233
:101000001A6500F0AFFF50EA01020B4602D001382A
:1010100061F1000302462068FFF780FE1A4A136D53
:101020001B032AD523684FF4002103F58053116573
:10103000012283F8812420E001221A6508221A6522
:101040004FF480621A6510BD196DC80702D4196D7E
:10105000890705D50321196510460021FFF774FFA4
:10106000094B1A6D100702D41A6DD10605D5182246
:101070001A6520680121FFF767FF2068BDE810406E
:10108000FFF780BF283600200064004008B53023F9
:1010900083F31188FFF776FF002383F3118808BDDF
:1010A000436DD3F8C40080F40010C0F34050704783
:1010B00008B5302383F3118800F58050C06E01F02D
:1010C00027F8002383F3118843090CBF0120002077
:1010D00008BD000000F5805393F8812462B1416D92
:1010E0008A6922F001028A61D3F8C4240132C3F86C
:1010F000C424002283F88124704700002DE9F743BF
:10110000302181F3118800F583511831002541F217
:10111000900E4FF0010800F5805C00EB451474441C
:10112000267977071CD4F6061AD5D0F854908E6924
:10113000D9F8C87008FA06F63E4211D04F680197F8
:101140000F689742019F9F410AD2C9F8D060267963
:1011500046F004062671DCF8B0440134CCF8B04403
:101160000135202D01F12001D7D1002383F311880F
:1011700003B0BDE8F0830000F8B51E4600231370ED
:101180000F4605461446FFF793FF80F001003870C4
:101190001EB12846FFF784FF2070F8BD2DE9F04FFF
:1011A00085B09946DDE90EA30D46029313780193AD
:1011B00091F800B08046164600F0D4FE2B78044625
:1011C0000F4613B93378002B41D022463B464046A8
:1011D000FFF794FFFFF75AFFFFF77CFF4B463246BD
:1011E0002946FFF7C9FF2B7833B1BBF1000F03D0BD
:1011F000012005B0BDE8F08F337813B1019B002BBF
:10120000F6D108F580530393029B544577EB030313
:101210001DD2039BD3F87C04C8B10368AAEB040178
:101220001B6898474B46324629464046FFF7A4FFC5
:101230002B7813B1BBF1000FDAD1337813B1019BD6
:10124000002BD5D100F08EFE04460F46DCE70020CF
:10125000CFE7000008B50020FFF7C8FEBDE8084052
:1012600005F02CBD08B50120FFF7C0FEBDE8084021
:1012700005F024BD036800211B68184708B5043039
:1012800007F040FE012008BD043007F031BE000029
:101290002DE9F84306460D4621B9043007F006FE55
:1012A000012424E003685B6898470028F8D100F027
:1012B00059FE104B8846D3F800904FF47A710746D8
:1012C0004D43D9F828000368C8219B6898473368C4
:1012D00030465B68984704460028E1D100F042FEA2
:1012E000C01B61EB0801A84271F10003E9D320465D
:1012F000BDE8F8833825002010B5044B044640F8BB
:10130000043B07F091FD204610BD00BF682602088F
:10131000034BC068DB68C31A58425841704700BF8E
:10132000886F00200CB430B585B008AC0A46074978
:1013300054F8043B0D6800940146E86A0394FCF7F6
:1013400057F805B0BDE8304002B07047382500209E
:1013500013B5054C0093246813460A460146E06A1B
:10136000FCF746F802B010BD382500202DE9F34106
:10137000134601920E460A46002107460846FFF72B
:10138000E7FF041E019B05DC4FF0FF34204602B04E
:10139000BDE8F08104F1010801214046019308F005
:1013A000E3FB05460028EFD0019B32464146FFF79C
:1013B000CFFF3D60EAE700000EB403B503AA52F880
:1013C000041B0192FFF7D2FF02B05DF804EB03B0FB
:1013D000704700000A460146014805F0BDBC00BF49
:1013E000006B00200FB407B5054B04A91B6851F82A
:1013F000040B0191984703B05DF804EB04B070470B
:10140000102300207047000013B50468009224697F
:101410000B46A04702B010BD704700000020704787
:101420000020704713B56C4684E8060000F11403F1
:1014300094E8030083E8050002B010BD0020704767
:1014400013B56C4684E8060000F10C0394E8030031
:1014500083E8050002B010BD0023C0E903337047E4
:1014600082B002AB03E9060002B07047704700008B
:10147000002070477047000013B50468009224698B
:101480000B46A04702B010BD0020704700207047F7
:1014900070470000002070470020704782B002A90A
:1014A00001E90C0002B0704770470000002070474F
:1014B000704700007047000001207047012070470E
:1014C000012070472830704782B002A9002001E94E
:1014D0000C0002B070470000704700007047000029
:1014E0007047000070470000084608F0D7B90000B8
:1014F000084608F09DBA000073B51E460C46154616
:10150000011D102201A8FBF755FE32462946204650
:1015100008F00EFA044601A8FBF768FE204602B068
:1015200070BD000013B50D220C46011D01A8FBF78C
:1015300041FE204608F0C4F9044601A8FBF756FE18
:10154000204602B010BD000008F0A6B9084608F019
:101550009FB90000084608F093B9000010B5064B8B
:10156000044640F8843B00F083FD04F1700000F075
:101570007FFD204610BD00BF402E020808B5302078
:10158000FBF7AAFC70B10023C0E90333C0E90533BF
:101590000371037A022262F302030372024B0360B7
:1015A000024B836208BD00BF10270208F42902081D
:1015B00010B4BDF8044001945DF8044B00F0B8BBD2
:1015C00010B4BDF8044001945DF8044B00F05EBB1C
:1015D00000F074BB00F0A2BB10B5044B03600446DE
:1015E000406A08B1FBF784FC204610BD942602082F
:1015F00010B50446FFF7F0FF2046FBF775FC2046C8
:1016000010BD000010B51C4B0360002190B00446D3
:101610000171102200F54A7008F0CCFE04F54E70FE
:10162000FFF76AFE122008F033F9144B0A94CDE953
:101630000B34134BCDE90D34124B0F9310A9024616
:1016400011E9030005AB83E80300DDE90C0103ABFE
:1016500083E80300DDE90A0101AB83E803000A4BDC
:10166000009304F10801234604F5597001F010F8C5
:10167000204610B010BD00BF50280208C115010857
:10168000D1150108D5150108B11501081B4A1C49DF
:101690001C4B10B502611C4A42611C4A8261026403
:1016A0001B4A42641B4A82641B4AC161C2641B49D3
:1016B0001B4A016202651B491B4A416242651B4984
:1016C0001B4A0360816282651A4B1B491B4A4360B7
:1016D000C162C2651A4B1B491B4A83600163002328
:1016E0001A4902661A4AC360044641634266C363EC
:1016F00000F00AFC174B2360204610BD6C3E002012
:1017000030360020EC260208E8390020F0370020AF
:1017100058390020683900207839002038360020F8
:10172000883900201C370020983900208C3D00208B
:10173000A8390020843D002048370020B839002017
:10174000883D002014230020C83900209436002052
:10175000D8390020B027020808B5302383F3118858
:10176000074B1B689A68996B8A4201D0824200D26B
:101770009860986307F0F6FC002383F3118808BD96
:10178000903600207FB51422002101A81C46334E5C
:10179000334D08F00FFE69464FF461433148009322
:1017A00007F040F9304BF2681A60B4202C6007F063
:1017B00039FE03F0EFFF08F015FB2C4B1C684FF4CB
:1017C000E131206CFBF7A2FD206903681B68984794
:1017D000A06A03681B6898470A20FFF7BDFF08F05E
:1017E00017FC40B12248132108F022FC20494C226A
:1017F000881808F0D1FD1F4B286801229A730368EE
:101800001B6898471C4B1B6813B11B6ADB0701D58B
:1018100008F0C8FBE06A03685B68984738B1FEF7D8
:10182000F3FA4FF497724FF40061FEF7D9FA1148BA
:1018300002F0F4F9A06A0F4C03681B6B9847F36839
:101840000E4ADA61B42007F0EDFD286803685B6892
:101850009847204602F0E2F9F7E700BF886F0020C2
:10186000B0360020006B0020903600203825002084
:101870004C3700208C3D0020203F002080260208AD
:10188000014B1868704700BF903600200048704731
:10189000B436002000487047B436002038B53F4DBC
:1018A0003F4C0021284602F093FD3E49224628463F
:1018B00008F048FD3C483D4D00F0CEFE3C4800F0AD
:1018C000CBFE3C4800F0C8FE3B4800F0C5FE3B485C
:1018D00000F0C2FE3A4800F0BFFE3A4800F0BCFEFD
:1018E000394800F0B9FE394800F0B6FE384801F03A
:1018F000C9FC384B384A1A602846384B40F8983BA8
:10190000FFF7FAFC2846364D3649224608F01AFD04
:101910002846FFF777FE224633492846334D08F024
:1019200011FD334804F0FEF82846324B40F8043BE2
:101930002422002108F03EFD05F13400FFF7DCFC15
:101940004FF0FF332C49EB642246284608F0FAFC9E
:101950002A4B2B482B4D30221A714FF47A72DA80C1
:101960004FF4FA621A81284A1A6002F0FBF8274BFA
:10197000002283F89C202846254A1A60254B40F80F
:10198000043BFFF7B9FC22462846234908F0DAFC5D
:10199000BDE838402148FFF779BE00BFF03700208E
:1019A0001C3F00205D150108583900206C3E0020C6
:1019B00068390020783900208839002098390020C3
:1019C000A8390020B8390020C8390020D8390020B3
:1019D000843D0020883D002074270208102B020857
:1019E000E8390020D9140108DD1401083836002038
:1019F00030360020002C0208E11401081C370020BA
:101A00008C3D00209436002014290208483700201D
:101A1000643002088C270208E5140108B43600205F
:101A200070470000037933B108304FF44873086001
:101A300013600120704718467047000000F5597088
:101A400001F03EB810B50446007948B100F088FABC
:101A5000D4F86033C01AB0F5FA6F2CBF0020012013
:101A600010BD000008B5FEF7CFF9A2224FF40031F7
:101A7000FEF7B6F9002008BDF8B50646EAB1CC0875
:101A800001390A44C2F3CC050127A54215D3632CC2
:101A90000ED8630906EB830304F01F0207FA02F174
:101AA000D3F828230A43C3F828230134A4B2ECE76F
:101AB000FFF7D8FF0028ECD1F7E7F8BD122110B5E9
:101AC00013220446A0F858130548FFF78BFC04F5D1
:101AD000597001F03DF810B9024800F017FA10BD36
:101AE000B4270208DA27020810B50179044671B953
:101AF000102200F54A7008F05DFC2046FFF7DEFF7B
:101B0000022121710248BDE81040FFF76BBC10BDF7
:101B1000F8270208B3F5487FF8B507460E46144685
:101B20001D460DD8C3F548739A4209D80834FFF70B
:101B3000DBFF2A4639193046BDE8F84008F02CBCD6
:101B4000F8BD0000B3F5487F2DE9F34105460E4688
:101B500090461C4622D8C3F5487399421ED801F11D
:101B60000807074422463946404608F005FCA8B15C
:101B70002846FFF7B9FFF12205F54E7101A8FBF7E2
:101B800019FB22464146384608F006FC2846A2B218
:101B90003146FFF771FF01A8FBF728FB02B0BDE853
:101BA000F081000037B505460C4601A80121FBF77E
:101BB000E7FAE10089B2082205F5597000F0C2FE8B
:101BC000044601A8FBF7E8FA204603B030BD000048
:101BD0002DE9F74F0379044603B300F54A7300F586
:101BE0004E7853F8042B32B94345FAD100F0B8F9D6
:101BF000C4F8600312E000250123C5F34A1604EB84
:101C0000860605F01F07D6F8282303FA07F71742C0
:101C10001FFA85FA05D10135642DEED103B0BDE878
:101C2000F08FED0008354FF48872414601A8FBF7AC
:101C3000C1FA04EB050B6359C4F85033DBF80430E8
:101C4000C4F8543301A8FBF7D1FA2379022B04F529
:101C50005479E3D151462046FFF7A4FF0028DDD098
:101C60004FF49C72414601A8FBF7A4FA082259469A
:101C7000484608F081FB28B9D6F8283323EA070341
:101C8000C6F8283301A8FBF7B1FAC7E738B51C46F8
:101C9000094BB0F858031B685B6B15461A68014482
:101CA000126818469047BDF810204119204608F0E8
:101CB00073FB012038BD00BF382500202DE9F74314
:101CC000DFF8549006460F4605244FF47A7101A8B8
:101CD000FBF756FAD9F80080B6F85813D8F8340054
:101CE00003683944DB689847054630B101A8FBF723
:101CF00053FA284603B0BDE8F083D8F828000368FB
:101D000001215B689847013C01A8FBF745FA14F0F4
:101D1000FF04DAD1EDE700BF38250020034B1B6834
:101D2000DB6A93F89C0080F00100704738250020A2
:101D30002DE9F04F2DED028B08EE103A2A4BD3F827
:101D400000900446D9F834000F460368B4F85813DD
:101D50001B6885B039449046BDF840B098470525CA
:101D600000EB080A012103A8FBF70AFAD9F83400AE
:101D7000036818EE102A1E6951465B46B0470646B6
:101D800040B103A8FBF708FA304605B0BDEC028B62
:101D9000BDE8F08FD9F82800036801215B689847F7
:101DA000013D03A8FBF7F8F915F0FF05DAD120464D
:101DB000FFF7B4FF0028E7D000F0D2F8D4F85C3386
:101DC00041F28832C31A9342DED9C4F85C0304F5A9
:101DD000597000F0ABFE5B4600904246394603481E
:101DE000FFF700FBD0E700BF3825002018280208C5
:101DF00070B51D46164B1B6813B11B6ADB0725D552
:101E0000144B1E68F46A94F84630C3B9124BA4F818
:101E10004400DB6884F84610E26163B19A6884F894
:101E20004720D96939B194F9483023B9042204F123
:101E3000480000F099F8094B5B68C4E90835F06A7E
:101E40001321BDE87040043008F0ECB870BD00BF4D
:101E5000203F002038250020886F002000ED00E0A2
:101E600000B59BB0EFF309816822684608F094FA48
:101E7000EFF30581074BC9B29A6BD86A986A986AE2
:101E8000986A986A986A9B6A059B7B20FFF7B0FF67
:101E9000FEE700BF00ED00E000B59BB0EFF3098165
:101EA0006822684608F078FAEFF30581064BC9B25C
:101EB0009A6B986A986A986A986A986A9B6A059B6E
:101EC000BF20FFF795FFFEE700ED00E000B59BB0F7
:101ED000EFF309816822684608F05EFAEFF30581A6
:101EE000064BC9B25A6B986A986A986A986A9B6A54
:101EF000059BE320FFF77CFFFEE700BF00ED00E05D
:101F0000FEE70000FEE70000704700000FB483B555
:101F100004AC0F4F54F8048B0E4EFDF775FF4FF4D1
:101F2000A5722021FDF75CFF42F210752146404664
:101F30000194FFF74FFA3846FFF754FA3368986A6E
:101F4000036829465B6898474FF4FA75EEE700BFCF
:101F5000B1E70108382500204FF08043586A7047E8
:101F600007F0A6BE07F088BEF8B50D460746114635
:101F70002846164608F0F4FE864204468CBF421CF2
:101F800002462946384608F007FA2046F8BD000008
:101F900070B5467B05460EBB4468836804EB840439
:101FA000A40804F50074E21A914288BFCC180C4BC7
:101FB00029681B68D86A0368621C1B6D984718B9AA
:101FC00001232B73304670BDAB68C5E90004E21AEB
:101FD0000021184408F0EEF90126F3E70026F1E7A6
:101FE000382500200EB470B5017B85B0044619BBBE
:101FF000D0E901239A421BD0134B1E680AADD4E9E5
:10200000012120680095521A099B03950144F06A4A
:10201000FBF7EEF900280FDBD4E90123D21A824244
:102020000FD8411C2046FFF7B3FF0028E7D103E09B
:10203000FFF7AEFF0028DFD105B0BDE8704003B068
:1020400070471844A060F7E73825002070B50026D7
:102050000446C0E9026601200D4607F085FDB04246
:1020600008BF3546206065602674204670BD0000BC
:1020700010B5037C044613B9006807F079FD2046CB
:1020800010BD000070B5057C04460E46DDB9BFF3F7
:102090005B8FC560BFF35B8FBFF35B8F8560BFF362
:1020A0005B8F43688B420CD0006807F061FD3146BE
:1020B000012007F059FD206010B96560284670BD09
:1020C00066600125FAE70025F8E7000038B5054607
:1020D0000C4644B121462846FFF7D4FF20B904EB53
:1020E0004404A408F5E7204638BD00000023BFF3F0
:1020F0005B8FC360BFF35B8FBFF35B8F8360BFF306
:102100005B8F7047BFF35B8F0068BFF35B8F7047D7
:1021100070B505460C30FFF7F5FF05F108060446DB
:102120003046FFF7EFFFA04206D930466D68FFF753
:10213000E9FF2544281A70BD3046FFF7E3FF201A57
:10214000F9E7000070B50546406898B105F1080050
:10215000FFF7D8FF05F10C0604463046FFF7D2FF23
:102160008442304694BF6D680025FFF7CBFF013CE9
:102170002C44201A70BD000038B50C460546FFF708
:10218000C7FFA04210D305F10800FFF7BBFF0444CE
:102190006868B4FBF0F100FB1144BFF35B8F0120D2
:1021A000AC60BFF35B8F38BD0020FCE72DE9F04148
:1021B000144607460D46FFF7C5FF844228BF044674
:1021C000D4B1B84658F80C6B4046FFF79BFF30443B
:1021D000286040467E68FFF795FF331A9C4203D87B
:1021E0006C600120BDE8F0816B60A41B3B68AB60B4
:1021F0002044E8600220F5E72046F3E738B50C46B6
:102200000546FFF79FFFA04210D305F10C00FFF732
:1022100079FF04446868B4FBF0F100FB1144BFF39C
:102220005B8F0120EC60BFF35B8F38BD0020FCE7C3
:102230002DE9FF41884669460746FFF7B7FF6C4620
:1022400006B204EBC6060025B44209D062682068D5
:1022500008EB050108F0A0F8636808341D44F3E7B3
:1022600029463846FFF7CAFF284604B0BDE8F0818A
:10227000F8B505460C300F46FFF744FF05F1080698
:1022800004463046FFF73EFFA042304688BF6C68E8
:10229000FFF738FF201A386020B130462C68FFF76E
:1022A00031FF2044F8BD000073B5144606460D46C4
:1022B000FFF72EFF844228BF04460190DCB101A93C
:1022C0003046FFF7D5FF019B33B93268C5E90233C9
:1022D000C5E9002401200CE09C4238BF019428602D
:1022E000019868608442F5D93368AB60241AEC60C9
:1022F000022002B070BD2046FBE700002DE9FF413F
:102300000F466946FFF7D0FF6C4600B204EBC005EC
:102310000026AC4209D0D4F8048054F8081BB81940
:10232000424608F039F84644F3E7304604B0BDE8C9
:10233000F081000038B50546FFF7E0FF044601468E
:102340002846FFF719FF204638BD00002DE9F74F5A
:1023500010EE103A009210EE102A072928BF07212C
:10236000C3F316044FEAD37812024FEAD353074659
:102370000E4603F0FE0340F1A6800133DBB2FF2BD3
:1023800032D044F40004DA0859495A4811F902904D
:10239000594951F8225003F00703A4FB0554C3F137
:1023A0000F021133B2F1200104FA03F325FA02F50A
:1023B00058BF44FA01F145EA03054FF0000B58BF3E
:1023C0000D43144145F6F321CDF804B04FF0300A27
:1023D0002A1A64EB0103002B0DDB0AF1010A4FFA04
:1023E0008AFA15461C46F3E714B948F00408C8E712
:1023F00048F00808C5E700230A22F8F717FC019BFC
:10240000D3B9BAF1300F06D109F1FF394FFA89F982
:102410002A462346E5E7009BF3B1009A09F1010340
:102420005BB2013A012BACBFD218013202F0FF03BC
:102430009E42009328BF1E460BF10103BAF1390FEB
:10244000DAB257FA83FC0ADC0123964207F802A0AD
:10245000019319D99346B9E70136F6B2ECE7A2EB3E
:102460000B0039213844CDF800C007F0A3FFDDF898
:1024700000C0634630201946013B0A78013252B24F
:102480003A2A13D00A700CE00A22A0FB0206400888
:1024900040EAC670281A02FB016164EB6104002C5B
:1024A000E7DA87F800800FFA89F01DE0BB4208D117
:1024B000312309F101090B704FFA89F948F010082E
:1024C000EFE75870D7E7002B7FF45BAF002C7FF469
:1024D0005AAF384648F00208721C00F8018BD2B29D
:1024E000302107F067FF204603B0BDE8F08F00BF42
:1024F000EC28020800407A106C280208704700009F
:1025000070470000002070477047000070470000CF
:102510007047000003689B6B184700000368DB6B83
:102520001847000070470000002070477047000007
:10253000002070479FED010A704700BF0000C842AD
:10254000002070470020704700207047704700004F
:10255000002070470020704700207047704700003F
:10256000704700007047000000230B600120704797
:10257000002070470020704770470000704700003F
:10258000704700007047000070470000704700006F
:10259000002070477047000000207047704700001F
:1025A00070470000002070470020704700207047EF
:1025B000704700000020704770470000704700001F
:1025C000704700007047000070470000704700002F
:1025D00032207047704700000F299CBF00EB41007C
:1025E000428170470F299ABF00EB410040894FF4A8
:1025F00061707047102A0B4628BF102200F10A01B3
:102600005200184607F0C8BE03790BB100220271D0
:102610001846704703685B681847000003791BB9C8
:10262000012303711846704700207047704700006F
:1026300010B50446FAF758FC204610BD704700005C
:10264000704700000020704700207047012070474D
:102650001046704700207047014B0360704700BF71
:10266000142A020830B5094D0A4491420DD011F8E0
:10267000013B5840082340F30004013B2C4013F079
:10268000FF0384EA5000F6D1EFE730BD2083B8EDB8
:1026900082B010B5044602A8C4E9001240F8043F15
:1026A00003C804F1080383E80300DDE9050104F130
:1026B000100383E80300DDE9070104F1180383E850
:1026C0000300DDE9090104F1200383E8030020464B
:1026D000BDE8104002B0704710B50A4492B2914272
:1026E00008D004684B1C615C9BB209B1002010BD8E
:1026F0001946F4E70120FAE703680F3332D1836803
:10270000591C0FD1036901332CD14268164B9A42F0
:1027100028D1C368013325D1436901330CBF01209F
:10272000042070470E331DD103695A1C0BD1436836
:102730000D4A934216D1C2689A4213D143690133BC
:1027400010D1022070470D330CD14268064B9A42DB
:1027500008D1C368934205D14069984214BF042050
:10276000032070470420704762B5861510B4BDF889
:1027700004400194D0E90004A4465DF8044B60478E
:102780002DE9F043054685B088464FF0180900F161
:10279000100602276B68023B4B4546D9009703ABF6
:1027A0004A4641463046FFF7E1FF40B19DF80C3004
:1027B00003F00303012B09D0032B02D09BB10020AF
:1027C00001E0C5F82C9005B0BDE8F0839DF80D3010
:1027D0005B09013303EB430409EB4404023407347F
:1027E00024F00709D6E7BDF80C309DF80D20C3F39F
:1027F0008A03520903EB430301325B0002EB4202FE
:102800009BB2540003EB4202B2F5487FD7DC2A6842
:1028100000941344414609F102023046FFF7A6FF37
:102820000028CCD002344C44D9E7C5F82C900120C4
:10283000C9E7000010B4BDF804400194D0E90004D9
:10284000A4465DF8044B60472DE9F047026B8AB05F
:1028500004466AB990F82850039285F001051827BC
:10286000009704AB29461030FFF780FF039A08B9A0
:1028700000203FE0059E214B9E4203D0012384F8B7
:102880003430F5E704A80392FFF736FF0128039AD6
:10289000F4D16FF00C0304F108086FF00E0A6FF02A
:1028A0000D09089394F82810009704AB404607964A
:1028B0000996CDF810A0CDF81890FFF7BBFF0028BF
:1028C000D6D04FF0FF3309930893039A009704ABD7
:1028D0002946404605960796CDF810A0CDF81890E9
:1028E000FFF7A8FF0028C3D040F22E43C4E90B73C2
:1028F00084F828500AB0BDE8F08700BF62B586159D
:1029000070B5044688B0D0E906030D4616469847D0
:10291000A0B19EB10A4B03934FF0FF336FF00E024C
:1029200005930793049306931823029200930022C1
:1029300002AB294604F10800FFF77CFF08B070BD28
:1029400062B586152DE9F04390F8343085B0044621
:102950000E461746002B3FD14FF001094FF00608F5
:10296000002F5CD06368E26A9A1A236B08339A429C
:1029700036D3B6FBF8F59DF8083069F301038DF8FE
:102980000830BDF80820C5F30A0363F38C02ADF8E4
:102990000820C2F307226FF347128DF8092003EBDA
:1029A0004303226802EB430152F81330CDF80A309A
:1029B0008B88ADF80E309DF80830E26A94F8281044
:1029C0006FF301038DF808300823009304F1080029
:1029D0006B44FFF72FFF98B9002005B0BDE8F083E6
:1029E0002046FFF731FF0028C3D1D4E908039847F8
:1029F0000028F1D0204600F04DF80028B9D1EBE7CF
:102A0000E36A0833E36208FB1563C3F10603DBB234
:102A1000BB42E2DC1E44FF1AB6B2BFB2A0E70120FF
:102A2000DBE7000037B505464FF44874062C224614
:102A3000C4F54871A8BF062289B292B22846CDE9F2
:102A40000012FFF749FEDDE9001220B1063C231D0C
:102A5000ECD1012004E02846FFF774FF0028F5D1EF
:102A600003B030BD002310B580F834300363044652
:102A7000FFF7D8FF60B194F828100122514020469A
:102A8000FFF73EFF20B12046BDE81040FFF7DCBE57
:102A9000002010BD38B590F83550044645B1FDF71B
:102AA000B3F991224FF40011FDF79AF9002038BDD7
:102AB000012380F83530FFF7D5FF84F83550F6E76D
:102AC00070B50025182688B080F8345080F828505A
:102AD000C6622A4629460446FFF712FF10B90020B5
:102AE00008B070BD94F82820013A18BF01220121D6
:102AF0002046FFF705FF0028F1D00B4B03936FF042
:102B00000E02059302924FF0FF336FF00D02079310
:102B10000492069394F82810009602AB2A4604F11A
:102B20000800FFF787FEDBE762B5861510B504469F
:102B3000D0E90803984740B12046FFF7C1FF20B114
:102B40002046BDE81040FFF76DBF002010BD00001B
:102B50002DE9F04F804693B005464FF4487258F87F
:102B6000100BDFF818B1002107F024FC06AF002697
:102B7000B9464FF0180ACDF800A03B460022314676
:102B80004046FFF7F3FD044630B90024204613B059
:102B9000BDE8F08F0126EEE77B6803933846FFF728
:102BA000ABFD0138C0B2022802D8039B5B4504D0BC
:102BB0002846FFF785FF0446E8E71837002EE9D0DE
:102BC0004846FFF799FD07468DF814000CA8FFF75B
:102BD00093FD874280468DF8150003D1012FE7D180
:102BE000002608E0032FFBD0032804D0022FF7D0E3
:102BF000831E5E425E4112AB334413F8349CA9F14C
:102C00000203012B05D831462846FFF7B9FD0028FD
:102C1000CED086F0010112AB0B4413F8343C023BDA
:102C2000012B04D82846FFF7ABFD0028C0D00023B5
:102C3000B9F1030F85F834302B6315D0032F06D17B
:102C4000012200212846FFF75BFE00289DD0B8F145
:102C5000030F06D1012211462846FFF751FE002836
:102C600093D000232B6391E786F0010685F8286056
:102C70002846FFF7D7FE0028E0D199E762B5861510
:102C800090ED120A7047000090ED130A70470000A3
:102C9000B0F8540070470000B0F8560070470000CC
:102CA00090ED040A7047000010B52DED028B04462C
:102CB00082B000F12001782201A8FAF77BFA237D87
:102CC00053B994ED028A01A8FAF790FAB0EE480AD7
:102CD00002B0BDEC028B10BD07EE903A94ED067A7F
:102CE000D4ED076AF8EEE77A002387EE278AA3611E
:102CF000E3610023237586EEA77A84ED028A84EDD2
:102D0000037AE0E7F7B506460F4640F2063200F1D7
:102D1000980101A8FAF74EFA0025331D53F8042B49
:102D20009AB93820FAF7D8F8044628B10D4B036059
:102D300087802030FEF7E0FA06EB85056C6001A87D
:102D4000FAF754FA204603B0F0BD0135102DE5D155
:102D5000054B06491B68986903681B68984700245F
:102D6000EDE700BFF02A020838250020AC2A02084F
:102D7000FF2937B504460D461CD0B0F904308B420C
:102D800015D0672901D00E2914D1EB2204F12001BE
:102D900001A8FAF70FFA00230022A580A361E361DE
:102DA00022752361A360E36001A8FAF71FFA0120EE
:102DB00003B030BD0020FBE738B50C4B834214D183
:102DC0000B4B0C4D1C681021204607F049F804F10C
:102DD00010012A6834F8020B13688C420344136014
:102DE000F7D1054A13680833136038BD9069002095
:102DF0002C3F0020243F0020283F002070B51C4BB2
:102E00001C4E1B680446D86A036800229B6C102184
:102E10009847306040B3042006F076FE164B1860E9
:102E200010B304F158050021144805F0D5FB4022E9
:102E30000021284607F0BEFA012384F85830A4F890
:102E40005A300F4BE3654FF4005363664FF4E04193
:102E50004FF46073C4E921133268084829460823F7
:102E6000BDE8704005F0C6BB0648FFF74FF800BF4D
:102E7000382500202C3F0020243F002090690020AE
:102E8000B92D0108C42A0208FFF7B8BFB0F9043011
:102E9000DFED047A9FED040A0E2B08BFB0EE670A3F
:102EA000704700BF3333533A6740533A08B52DEDAE
:102EB000028BFFF7EBFF03681B68B0EE408A984770
:102EC00028EE000ABDEC028B08BD000010B50368B7
:102ED0000446DB6898472046FFF7D8FFD4ED037A15
:102EE00020EE270A10BD000008B52DED028BFFF77C
:102EF000CDFF03685B68B0EE408A984728EE000A71
:102F0000BDEC028B08BD000010B52DED028B82B028
:102F1000044600F12001FB2201A8B0EE408AF0EE49
:102F2000608AFAF747F9F0EE087AF4EEE78AF1EEF4
:102F300010FA5CBFB1EE040A28EE000A237DD4ED3E
:102F4000077A94ED067A84ED048A58BFC0EE286AA9
:102F500003F10103DBB223754CBF38EE270A36EECE
:102F6000A70A38EE077AFE2B84ED067A84ED070A6D
:102F70000BD1F6EE007A27EE277A20EE270A7F2380
:102F800084ED067A84ED070A237501A8FAF72EF975
:102F900002B0BDEC028B10BD30B5302383F3118835
:102FA00069B9094C0948236805681B68B3FBF5F348
:102FB000136023681960016081F3118830BD00231C
:102FC00083F31188FAE700BF243F0020283F002048
:102FD0002DE9F84F2DED028BB1FA81F46B466409AF
:102FE000A3EBC40300AF9D46EB465A4605469FED52
:102FF0001C8ADFED1C8AFFF7CFFF00290CBF4FF0C2
:103000000E094FF0FF094FF00008A04522D22E1DF7
:1030100005F1440A4FF0010856F8040B70B1B0F9FD
:10302000043099450DD1B9F1FF0F07D0DBED007ADF
:10303000D5ED120AB8EE670AFFF766FF5645EBD1E9
:10304000E3E7672BFAD195ED140AF0EE680A80EEFB
:10305000080AF1E7BD46BDEC028BBDE8F88F00BF62
:103060006740533A00000000B0F854305BB133F0D1
:10307000200308D0084B1B68DB6A93F89C30002BB8
:103080000CBF00232023B0F85620A0F854301A4378
:10309000A0F85620704700BF3825002010B5044620
:1030A000FEF75AFF636C42F20F72C31A934208D9BB
:1030B00060642046FFF7D8FF0021BDE81040FFF70D
:1030C00087BF10BD80F82D107047000080F82C10CD
:1030D0007047000001207047806A0430704700008C
:1030E00080F83410704700000020704701207047BE
:1030F00008B503685B689847002008BD03685B68F3
:10310000184700007047000070470000704700003B
:103110001FB502AC84E80C00009094E80C00806AB3
:1031200002F07CFD04B010BD806A02F0CFBD00004B
:1031300010B50446006B06F01BFD606A034B23606C
:1031400008B1F9F7D5FE204610BD00BF942602084D
:1031500010B50446FFF7ECFF2046F9F7C5FE204600
:1031600010BD000070B5044688B0503005F05CFE1C
:10317000104B0494CDE9053414200F4B0793F9F755
:10318000ABFE054690B108AA12E9030094F8483056
:103190000A4E06EB031601AB83E80300059B009380
:1031A0007279049BB179284602F002FBE56108B010
:1031B00070BD00BF0531010809310108702B0208FC
:1031C000194B03EB00102DE9F041027980680321CF
:1031D00002F0AEFC044628B306F006FE24F00F060B
:1031E000012204F00F0402FA04F407462146304697
:1031F00004F044FB0D4BD3F8008014257369634041
:103200007361D8F8280003680A219B68013D98473C
:1032100015F0FF05F2D13A4621463046BDE8F041AF
:1032200004F02CBBBDE8F081702B0208382500208B
:10323000124B37B503EB001002210279104802F05F
:1032400077FC0446B8B106F0CFFD0121054624F015
:103250000F0004F00F04A1400022CDE9000104F0AA
:103260000DFB0098019903692A4623FA04F404F03F
:10327000010404F003FB204603B030BD702B0208AC
:103280000704004838B5084D084B03600446002386
:10329000284685F84830FFF765FF054BEB64054B82
:1032A000EB63204638BD00BF303F0020882B02086A
:1032B000A08601008C5F506070B51E46204B0360F5
:1032C0000D46204B80F82D200021C0E90311C0E9F4
:1032D00005110171642105FB01338362022380F82B
:1032E0002C309DF8103080F83530059B8363EB005F
:1032F000044643F0010303724272134612492A4600
:103300003030FEF759F8A26AD36CB34215D90F4B8F
:103310009E429EBF0E49D163A26A0E4998BFD364F4
:103320000D4B1B689869A36ADA6C03681E684FF43A
:103330007A73B2FBF3F32A46B047204670BD00BF54
:10334000A02B0208303F0020282B0208A086010095
:103350003E2E8130342B02083825002030B585B050
:10336000CDE902320D4689B93C20F9F7B5FD044696
:1033700048B1099901919DF820100091DDE90232D0
:103380002946FFF799FF204605B030BD0024FAE733
:103390002DE9F04F89B05E4D0693836ADDF84880D1
:1033A00093F8483007911B0104461646E8581FFA67
:1033B00088F905F085F9A06ACDF8009006ABB2B2A5
:1033C00007A902F099FC074650B9A36A93F8483060
:1033D0001B01E85805F078F9384609B0BDE8F08FD0
:1033E00006EB0803DFF830B104934FF0000AA16A3E
:1033F000484ACB6CB2FBF3F3049AA06B53434FF4EF
:103400007A72B3FBF2F35B000133834238BF0346A9
:10341000C869059302F046FBA16A91F848000001D3
:103420003C31285805F000F9302181F31188DBF890
:103430000010C86A416B01314163002181F311889A
:10344000059B94F82D104FF47A72A3FB0232A26A06
:1034500092F848000001002E33D10093069A2858B4
:10346000434605F017F9A26A059092F84820120128
:10347000A85805F0E7F8A26A0121D06902F0F2F934
:10348000A06A059B90F8482011016958896811F0DD
:10349000800F20D0FCF7B8FC40F293124FF40021CB
:1034A000FCF79EFCDDE90621A06A4B4602F04AFCCF
:1034B000A36A93F848301B010027E85805F004F987
:1034C0008AE7CDE90183069B0093079A2858334683
:1034D00005F0C6F8C7E72BB9DDE906214B4602F037
:1034E00031FC72E7013308D11046FFF7A1FE20B985
:1034F000A36A93F84800FFF763FE94F82C200AF1C2
:10350000010A5FFA8AF39A42BFF471AFCAE700BFBB
:10351000702B020800127A0038250020F0B504460E
:10352000806A85B00430CDE902210A9F1E46FDF76E
:10353000EFFEDDE90221054660B91C4BA2681B685D
:103540001B49986903681E6894F82D30B0472846D7
:1035500005B0F0BDA36A94F83550186CA5B140F4DD
:103560008010186494F83450E5B181B9002EEED083
:10357000002FECD000220A9733461146204605B0B2
:10358000BDE8F040FFF704BF20F48010E9E7002A0F
:10359000ECD0002300932046FFF7FAFE0028E5D187
:1035A0000546D4E70A973346E8E700BF38250020F0
:1035B000482B020808B5B021044802F019FBBDE809
:1035C0000840034A0349002006F0BCBE303F0020FB
:1035D0001C3F00200D31010870470000002070479B
:1035E000B0F94C0070470000B0F94E007047000081
:1035F000012380F85430704780F855107047000060
:1036000090F8543013B190F8300070471846704766
:1036100037B590F8543004460D46ABB190F83030D1
:10362000122BA8BF122399420EDA00F13401612255
:1036300001A804EB4504F9F7BDFD01A8A488F9F73A
:10364000D5FD204603B030BD0024FAE737B590F829
:1036500054500446A5B100F134014A2201A8F9F7FB
:10366000A9FDD4E90A51226D0023994208BF954271
:10367000C4E90A2301A814BF01250025F9F7B6FD06
:10368000284603B030BD000073B590F8544005469D
:103690000E468CB1122A28BF122200F134011446C2
:1036A00001A87122F9F786FD6200291D304606F057
:1036B00073FE01A8F9F79AFD204602B070BD000024
:1036C00070470000407B70470161704710B5074BA1
:1036D000074ADB680446DA61A37B33B923684FF4F9
:1036E0007A719B6820469847F6E710BD886F0020E6
:1036F000282C020838B50D4B0D4ADB680446DA6108
:103700002368A27B9B6862B10A4D236820469B68B0
:103710004FF47A7198472B68586903681B6998477A
:10372000F3E742F2107120469847E9E7886F0020DE
:10373000EF2702083825002013B504460121C830C0
:1037400005F01CFD04F1D400012105F017FD1F4B0D
:103750000094B7224FF4BE611D4805F0EDFD1D4BEE
:10376000C4F8C4000094B5224FF4FE611A4805F075
:10377000E3FD1A4BC4F8B0000094B5224FF47C71FD
:10378000174805F0D9FD174BC4F8B4000094B122D6
:103790004FF4BE61144805F0CFFD144BC4F8B800D7
:1037A00000943A224FF41F61114805F0C5FD114BFA
:1037B000C4F8BC0000943B224FF4BE610E4805F0F3
:1037C000BBFDC4F8C00002B010BD00BFC539010880
:1037D000884900203D3D0108485F0020CD360108A2
:1037E00068550020553A0108784F0020D13D010866
:1037F000983F0020F53601085859002070B5437DE8
:1038000004460D464BB903681B6C984728B1B62097
:10381000FDF7A2FF40F20113A38223682946204648
:103820009B68BDE87040184708B5FEF729F8034BC0
:10383000DB681B1A5842584108BD00BF886F002042
:103840002DE9F04704460D46FEF78CFBDFF8689043
:1038500006460F46FEF786FB801B4FF0000361EB28
:1038600007014FF47A72F7F731FAA84271F10003B9
:1038700020D223684FF47A719B6820469847A3882A
:10388000AB42E7D8236820461B6C98470028E1D05C
:10389000D9F80080D8F82C30FC2293F94CA083F89A
:1038A0004C2023682046DB6C9847D8F82C3083F8EE
:1038B0004CA0CFE7BDE8F0873825002008B53022BE
:1038C00082F311888368002B01DC05F07DFC05F094
:1038D00049FC002383F3118808BD0000F7B50446B6
:1038E00000F1C8066D46304685E8060005F062FC2A
:1038F00094F86430DDE90007224604EBC30C62450E
:103900000DD0516A814208D1916AB94205D1304641
:1039100003B0BDE8F040FFF7D1BF0832EFE7072B57
:103920000AD895E8030004EBC3022432013382E88D
:10393000030084F86430EAE7034B04491B68986984
:1039400003681B689847E2E738250020302C0208FE
:1039500008B50E4B1B68586A0368DB6C0C46984729
:103960000B4B0C48002C08BF184606F02DFA72B617
:10397000BFF34F8F0849094BCA6802F4E062134352
:10398000CB60BFF34F8F00BFFDE700BF382500209D
:10399000020007B0010007B000ED00E00400FA05E6
:1039A00010B5836904461BB9BDE8104006F054B851
:1039B000FEF7D6FAA369C01AE3699842F4D8012049
:1039C00010BD0000F8B51F4B1F4ADB680446DA61E2
:1039D0002368657B5B681DB9642120469847F7E73B
:1039E0001A4B1B6813B11D6A05F00105184F2368B7
:1039F00064215B68204698473E6825B1F06A132130
:103A0000043006F00FFB002006F07CF8FEF7A8FA61
:103A1000D4F8AC30C01AB0F5FA7F0DD32368204635
:103A20005B69984740B9FCF7EFF9F36A4FF400413E
:103A3000B3F84220FCF7D4F9F0690368DB6B9847D0
:103A4000D5E700BF886F0020482C0208203F0020E7
:103A50003825002038B50D4B0D4ADB680446DA6185
:103A60002368A27B9B685AB10A4D236820469B6855
:103A70004FF47A7198472B68186AFFF721FEF4E734
:103A800044F6206120469847EAE700BF886F00208F
:103A9000502C02083825002008B5437B13B1034899
:103AA000FEF734FA0123437308BD00BF582C020807
:103AB00005F0D6BB084605F0DDBB000029B10A2998
:103AC00038BF0A21084605F0C5BC704710B5036829
:103AD0001B6C0446984740B1637D33B10023637586
:103AE000B420BDE81040FDF737BE10BDF7B5044661
:103AF00000F1D4066D46304685E8060005F05AFB15
:103B000094F8A830DDE90007224604EBC30C6245B7
:103B10000DD0916E814208D1D16EB94205D13046A7
:103B200003B0BDE8F040FFF7C9BE0832EFE7072B4E
:103B30000BD895E8030003F10D0204EBC202013338
:103B400082E8030084F8A830E9E7044B04491B68C5
:103B5000986903681B689847E1E700BF3825002093
:103B6000982C020810B5084B0446402240F8243B2C
:103B7000002106F01FFC4022002104F1680006F03D
:103B800019FC204610BD00BFC42C020810B50B4C18
:103B90001046002314F813208A4209D104EB430392
:103BA000FF225B7802211844FAF736F9C0B210BD43
:103BB00001330E2BEED13A20F9E700BF182D020891
:103BC000F0B585B0074602AD082085E806001E4620
:103BD00005F09AFF0446D8B195E803009DF930201E
:103BE00084E803009DF82C103846FFF7CFFF0A9DAC
:103BF000094B009405F2F7150246314625F00700FF
:103C000005F0E0FF054628B9204605F0B1FF28463B
:103C100005B0F0BD0120FBE7253E010810B50446C4
:103C200006F0D4F9FEF79CF9C4F8AC0010BD000012
:103C300070B503681B6C04460D46984738B12046A2
:103C4000FFF7ECFF4DB9236A13B90023A36170BDE0
:103C5000013B2362002BFAD1F7E7FEF781F9A36954
:103C600043B1E269C11A8A4204D913441B1A9D4226
:103C700038BF1D46236AC4E9060501332362236861
:103C800020469B69BDE870401847000010B51148F8
:103C900006F0F0F83F2807D8FCF7B6F84FF6FF72A9
:103CA0004FF40001FCF79CF805F062F9044678B186
:103CB000006A06F0DFF83F2806D8FCF7A5F8228F47
:103CC0004FF40001FCF78CF8204605F061F9EDE7B0
:103CD00010BD00BF00010020D0E90003184700001C
:103CE000F8B590F86530044603F0FF051BBB0123CF
:103CF00000F1C80680F86530304605F05BFA3046C2
:103D000094F86470FFF7DAFD04F12406AF4207DD92
:103D1000736813B13046FFF7DFFF01350836F5E76A
:103D2000236903B19847044B1B681869FFF7B6F97C
:103D3000002384F86530F8BD3825002010B5104BFD
:103D4000104ADB680446DA612368A27B9B6822B9CB
:103D50004FF47A7120469847F6E723684FF47A715A
:103D60009B68204698472046FFF7BAFF2368204605
:103D70005B6998470028F0D02046FFF74FFFECE73B
:103D8000886F0020B02C0208F8B590F8A9300446DE
:103D900003F0FF05DBB9012300F1D40680F8A93058
:103DA000304605F007FA304694F8A870FFF786FD14
:103DB00004F16806AF4207DD736813B13046FFF7C0
:103DC0008BFF01350836F5E7002384F8A930F8BDEC
:103DD00070B5124B124ADB680446DA612368A27B95
:103DE0009B6822B94FF47A7120469847F6E700267F
:103DF00023684FF47A719B68204698472046FFF766
:103E0000C3FFFEF7ADF8831BB3F57A7F0546EFD904
:103E10002046FFF73BFF2E46EAE700BF886F0020F1
:103E2000B82C020810B50446FFF756FF2046BDE83F
:103E3000104005F09DBE000090F809017047000099
:103E400003695B7923B9406B0A23B0FBF3F0704739
:103E50004FF4483070470000406B7047037D03B15A
:103E6000437D18467047000090F8ED20034602F0AD
:103E7000FF0012B193F8EC00C0B270470020704709
:103E800000207047F8B590F80831476B1F330C4697
:103E900000EBC30150F833504E6877B103695B798A
:103EA0005BB903685B6998472044054BB3FBF7F3A4
:103EB0005843281A054666F1000628463146F8BDE3
:103EC00080969800C089704708B58430FEF720F9C5
:103ED000003818BF012008BD90F8EC303BB1054B0D
:103EE000026DDB689A4202D17030FEF711B90020F2
:103EF000704700BF886F002013B540F27F22044650
:103F000000F1D4016846F9F755F94FF4207204F135
:103F1000BC0101A8F9F74EF9002384F8EC3084F8CD
:103F2000ED3023695A7912B9186804F089FD00212F
:103F300004F17000FEF7A6F8002104F18400FEF7FA
:103F4000A1F801A8F9F752F96846F9F74FF902B05C
:103F500010BD000008B580F84C11806A082104F0FB
:103F600011FF012008BD000090F8ED20034602F08B
:103F7000FF001AB103F18400FEF7E4B870470000B7
:103F80002DE9F843174604460D46FDF7E9FFDFF833
:103F90005C90064600EB0708236820465B6998475B
:103FA000A84218D24FF4806004F0C0FED9F80C305B
:103FB000A4F858506365FDF7D3FF821BBA420AD2BA
:103FC000A8EB00034FF47A71A3FB01134FF4806058
:103FD00004F0F8FEE0E7236820465B6998478542D5
:103FE0008CBF00200120BDE8F88300BF886F00204F
:103FF00010B53023044683F311880B0707D5FBF770
:1040000003FF40F232324FF00061FBF7E9FED4F8D3
:10401000B8305A68136823F00F031360D4F8B8302F
:10402000197C1A680E238B405360FDF795FF02211F
:10403000C4F80C01A06A04F08FFE002383F31188FA
:1040400010BD000070B503695A790446002A78D182
:104050001D68036A002B08BF0021036880F809115E
:10406000DB6A984700286CD094F80931032B68D894
:10407000DFE803F002322F68206A88B1012600F0E1
:104080000F01324606FA01F120F00F0003F0F6FBB3
:10409000236A23F00F0203F00F039E40B6B256834B
:1040A000012384F80A31302383F311886B6D9A68F9
:1040B00012F4407F42D01A6822F001021A606A6D41
:1040C000936823F4407393606A6D136843F00103AF
:1040D00033E00023C4E94333206A012600F00F01D6
:1040E000324606FA01F120F00F0003F0C7FB236A05
:1040F00023F00F0203F00F0306FA03F39BB253837E
:1041000084F80A61302383F311886B6D9A6802F496
:104110004072B2F5007F11D01A6822F001021A60D5
:104120006A6D936843F4007393606A6D936823F437
:10413000807393606A6D136833431360002383F3C5
:10414000118870BD236993F82920FF2A1BD0206AAB
:10415000D20100F00F030121994042F0020220F049
:104160000F0003F08BFB302383F311886B6D9A688B
:104170005204E3D41A6822F001021A606A6D93684F
:1041800043F480439FE723682046DB6BBDE8704023
:104190000021184710B50446C06940B100F00F0374
:1041A00001210022994020F00F0003F067FBA06975
:1041B00050B100F00F030121BDE8104000229940EA
:1041C00020F00F0003F05ABB10BD000038B50369A2
:1041D0005A7904460D46002A38D10173186804F054
:1041E0002FFC012D33D0022D35D02DB9E36B23F0F8
:1041F000805323F4B053E363236904F13801186852
:1042000004F010FC94F8643133B12369186804F5A4
:10421000A871043004F070FD002D14BF01230023A9
:1042200084F8643109D0236918684FF400622023B0
:1042300004F5A871043004F04BFD237D33B12369EC
:104240001B685A6D136823F02003136038BDE36BBD
:1042500043F4B053CFE7E36B23F4007343F4A0536C
:10426000C9E70000037DA3B1D0F8B4305A681368E1
:1042700023F00F031360D0F8B430197C1A680E23B2
:104280008B405360D0F8B4305A68136823F00103B0
:104290001360704738B503695A7904460D46D2B9A0
:1042A000186804F0CDFB012DD4F8283114D0022D6C
:1042B00017D0D4F828312364236904F13801186831
:1042C00004F0B0FB237D33B123691B685A6D13687A
:1042D00023F02003136038BD23F40053C4F82831C1
:1042E000E7E743F40053F9E703695B791BB9806A98
:1042F000042104F047BD7047F7B590F8ED3004464F
:104300000E46174603F0FF05BBB100F19C014FF4C8
:10431000427201A8F8F74EFF3A46314604F1840094
:10432000FDF786FF94F84C3105461BB1A06A0421C5
:1043300004F028FD01A8F8F759FF284603B0F0BDA6
:1043400070B590F8093105460C46D3B9406AB8B14A
:10435000012600F00F0106FA01F120F00F003246AD
:1043600003F08CFA6D6A05F00F0184EA060001F192
:10437000100398408C4025F00F050443AC61304693
:1043800070BD0020FCE7000070B590F809310546CB
:104390000C46D3B9006AB8B1012600F00F0106FA45
:1043A00001F120F00F00324603F068FA2D6A05F0A3
:1043B0000F0184EA060001F1100398408C4025F0BB
:1043C0000F050443AC61304670BD0020FCE70000DF
:1043D000164B10B50360164B80F832102C2201FBEF
:1043E000023303614FF4614304464363002170309C
:1043F000FDF72CFE002104F18400FDF727FE04F1F7
:104400009C00FCF779FF04F1BC00FCF775FF04F198
:10441000D400FCF771FF002394F8322084F80931AE
:10442000044B43F82240204610BD00BF402E020836
:10443000B42D02083867002013B5094C23686BB906
:1044400000930849084B3C224FF49E6005F0BAFBEC
:104450002060236813B90548FDF758FD02B010BD70
:1044600064670020342D0208155101083C2D020814
:1044700030B5836A85B004462BBB144B22691B6898
:104480005579D86A13790093114A124B04F12C0123
:10449000002D08BF134606220391F8F7C9FF94F8D0
:1044A0004C3103990094002B18BFB5220A4B08BF6A
:1044B0003C224FF44C7005F085FBA062A36A13B94F
:1044C0000648FDF723FD05B030BD00BF38250020AC
:1044D000632D02085C2D0208295001086B2D02088B
:1044E00038B5D0F8B8500446EDB9302383F31188BD
:1044F00000690D4A407B23460C2103F029F8C4F8DB
:10450000B80085F31188D4F8B8305A6823691B685D
:104510005B6D283393602369D4F8B8001969BDE84E
:10452000384003F099B938BDF13F0108FFF7D8BF13
:1045300010B590F85C3083F0010380F85C3090F89F
:104540005C3018330446402150F8230005F088FC05
:1045500094F85C30D4F8B4201833526854F82330FF
:10456000D360D4F8B4305B6840225A60D4F8B430D9
:104570005B688A221A60D4F8B4305A68136843F032
:104580000103136010BD00002DE9F04104468AB01C
:1045900090461F460E4689B957EA02030ED190F89D
:1045A000ED305BB190F8EC3043B1034BDB68036551
:1045B0000AB0BDE8F08100BF886F0020FFF73CFF24
:1045C00023691A68002AF3D05B794FF4C870B6FBF0
:1045D000F0F0B0F5007F38BF4FF40070002B0CBF37
:1045E0004FF400734FF4806385B29F4238BF1F467B
:1045F0004FF49472454504F1D40104A838BF4546F0
:10460000F8F7D8FD636F9D4207D0002384F8EC30A3
:10461000294604F17000FDF759FD636F1B09C4F8CA
:104620009830C6B1636BB34200F04B819B4B1B6863
:104630009B696663A34200F0448104F1700528463B
:10464000FDF766FDD4F820311844C4F8200128464F
:10465000FDF74CFD012694F83031E3B9E389D90523
:1046600019D4226E52B923699B793BB18B4B1B68DD
:10467000D86A036840219B6C98472066626E52B9E5
:1046800023699B793BB1854B1B68D86A036840213D
:104690009B6C98476066A36E73B923691B7B5BB103
:1046A000E28912F4007207D17C4B1B68D86A036858
:1046B00040219B6C9847A06694F83031002B00F0A5
:1046C00002810023A382B4F86C20636BB2F57A7F79
:1046D00004D9B3F5E12F0DD800226275B3F5E13F9F
:1046E00008D823691A7B2AB1587B01F081F808B1F8
:1046F00000236375E289D4F8243112054CBF23F0FE
:10470000005343F00053C4F8243140F2671204F11F
:10471000BC0105A8F8F74EFDD4F888309F4207D0B9
:10472000002384F8ED30394604F18400FDF7CEFC17
:104730001EB104F18400FDF7D9FC23695B79002BDD
:1047400040F08E80636B002B00F08A8094F8EE605E
:1047500094F8EE30F6B203F0FF0503BB237DDBB126
:10476000302383F3118820694D4AC07923460C21F8
:1047700002F0EEFEC4F8B40085F31188D4F8B4302A
:104780005A6823691B685B6D243393602369D4F8EE
:10479000B400996803F060F8012384F8EE30637D7B
:1047A0000BB3D4F8F030F3B93E4B0694CDE907349F
:1047B00014203D4B0993F8F78FFB054678B10AAA00
:1047C00012E9030023695F7B01AB83E80300079BC9
:1047D0000093FF22069B3946284600F0E9FFC4F803
:1047E000F05005B96575636BA363217DD4F828315A
:1047F000D4F824212364D4F82C31E263636429B112
:1048000042F0100243F04003E2636364637D1BB136
:10481000636C43F080036364244BC4E9123423695E
:1048200004F13801186804F0FDF8237DC3B1236951
:104830001B685A6D136823F02003136086B9D4F8FF
:10484000B4305A68136823F00F031360D4F8B430FF
:10485000197C1A680E238B4053602046FFF768FED0
:10486000D4F8883013B1012384F8ED30636F13B1AD
:10487000012384F8EC300E4BDB6823652046FFF7FC
:10488000F7FD236894F80911DB6B2046984794F8EC
:1048900032307BB994F8ED300CE000BF38250020B1
:1048A000C54D01082D45010801490108654201086F
:1048B000886F002005A8F8F799FC04A8F8F796FC83
:1048C00076E60026C7E6226E1AB1636E003B18BF7B
:1048D00001232375A36E003B18BF01236375F2E625
:1048E00010B53023044683F31188D0F8B80002F0E5
:1048F000ABFE0023C4F8B83083F3118810BD00006C
:10490000FFF7EEBF2DE9F74FD0F8F03004460E4622
:104910004BB346B394F809112046F8F70FFD50B198
:10492000636A43B123F00F0203F00F03126922FA06
:1049300003F3DB0717D404F19C0840F255324146DB
:1049400001A8F8F737FC04F18407402E3246A16E27
:1049500028BF40223846FDF7D1FC85B281462DB9EB
:1049600001A8F8F743FC03B0BDE8F08F3846FDF727
:10497000CFFB864228BF064601A8F8F737FCD4F8DB
:10498000F00001F08FF8022004F0D0F9D4F8F00024
:10499000C37C002B00F0A680636BB3F5E12F0FD82A
:1049A000B4F86C10033189B2B1F57A7FA4F86C10B9
:1049B00006D90021617503B0BDE8F04F00F052BF89
:1049C000FA214E4A4B43B3FBF2F31FFA89F201334B
:1049D0009A4200D99DB24FF0300B8BF31188D4F876
:1049E000B83059680B6823F00F030B60D4F8B83067
:1049F000197C18684FF00E0A0AFA01F14160A06EA6
:104A0000294605F02FFAD4F8B810A06E49683C4B3F
:104A1000C860D4F8B81049684D60D4F8B810496837
:104A20009A200860D4F8B8104868016841F0010184
:104A30000160A91C606B5943324BB1FBF0F1324865
:104A400001F5FA71994288BF0146002080F3118870
:104A5000022004F0B7F9814610BB8BF31188D4F81B
:104A6000B8205068026822F00F020260D4F8B82023
:104A70001068127C0AFA02F34360D4F8B8305B681D
:104A80005B689D4237D9ED1AADB21DB1FDF764FAEE
:104A9000C4F80C01022004F03FF9002383F31188CD
:104AA000D4F8F000C9F3400100F0DCFE002D3FF423
:104AB0005AAF40F2B132414601A8F8F77BFB2946D4
:104AC0003846FDF759FBD4F814312B44C4F814319F
:104AD000D4F818312B44C4F8183101A8761BF8F724
:104AE00085FB16E7B4F86C30002B3FF474AF013B44
:104AF000A4F86C306FE74D46CCE700BF40420F0092
:104B0000809698009F860100A086010013B5D0F81A
:104B100048310446BBB900F59A7004F011F9182326
:104B2000C4F8483123691868019003F089FF636C69
:104B3000019823F0080304F13801636402B0BDE872
:104B4000104003F06FBF02B010BD00002DE9F04728
:104B5000044686B00D4640F2CA3200F19C0101A81D
:104B6000F8F728FB94F8303123B1012D02D9204603
:104B7000FFF7CCFF04F184092A4602A94846FDF755
:104B800093FB4FF00008824602AD4746C2451FDD49
:104B900022695379D3B910680268D669D5E9001241
:104BA000B047061E14DB05D0FDF7D6F93744C4F82C
:104BB0000C01BFB2083531464846FDF7DDFA55F81D
:104BC000043C9E4204D108F10108DFE70026F1E72A
:104BD000D4F814313B44C4F81431D4F818313B44B0
:104BE000C4F8183101A8F8F701FB06B0BDE8F0875A
:104BF00070B504468430FDF78BFA0146B8B1637D89
:104C00002046ABB1FFF77EFE94F80931022B0ED19E
:104C1000D4F810511DB9FDF79FF9C4E94405637D2F
:104C20004BB1D4F80C31D3B1012384F8093170BDF4
:104C3000FFF78CFFE8E723691B689A6BE38913F49D
:104C4000006FD4F81431C2F500700CBF0C2108219C
:104C5000984204D2A3F5007313448B42E4D8FDF7C5
:104C60007BF9D4F81031C01A0B4B9842DFD90B4BAB
:104C700022691B680A4998690A4BD21A0A4B92109A
:104C80005A430368D2B21B68984723682046DB6BFF
:104C9000BDE870400021184720A1070038250020FA
:104CA0008C2D0208B42D0208A38B2EBA10B5036A0E
:104CB0000446E3B190F80911F8F740FBB8B104F1EC
:104CC0007000FDF73FFA94F80A21D4F8983080B2CA
:104CD00072B198420BD2226A002384F80A3122F082
:104CE0000F01012302F00F0293409BB20B8310BD12
:104CF00010339842FBD9226A012322F00F0102F0FF
:104D00000F0284F80A3193409BB24B83EFE7000017
:104D100070B5124B026DDB689A42044619D190F8C7
:104D2000EC3003F0FF0593B100F170063046FDF75B
:104D3000EFF9D4F820311844C4F820013046FDF7CB
:104D4000D5F994F80A3133B92046FFF7AFFF28466A
:104D500070BD0025FBE71D46F9E700BF886F002006
:104D600038B50D4B0546DB68006D984210D195F8BB
:104D7000EC306BB105F17000FDF7DCFA044628B1A8
:104D800095F80A3113B92846FFF790FF204601E055
:104D90004FF0FF3038BD00BF886F002038B590F865
:104DA00008510446FDF7DEF885F0010504EBC50562
:104DB000C5E93E0194F8083183F0010384F8083115
:104DC00038BD000070B5037D0446002B4AD0D0F8F2
:104DD000B4305B685D6890F85C601A6822F00F027E
:104DE0001A60D0F8B430197C1A680E23C5F140055A
:104DF0008B40ADB25360F6B2FFF79AFBADB11836F7
:104E00002A4654F8261004F17000FDF711FAD4F880
:104E10001C31D4F820212B4415442D1AC4F81C3120
:104E2000C4F820512046FFF7B9FF636D93B104F138
:104E30007000FDF76DF9B4F8583098420AD330236A
:104E400083F311884FF48061606D03F085FF0023C8
:104E500083F3118894F80A3123B12046BDE87040ED
:104E6000FFF724BF70BD00002DE9FF4700F1700877
:104E700004464046FDF766F9694602464046FDF79E
:104E800095F96E468146002704F5A87AB9450ADDF2
:104E90002269537953B910680268156AD6E900127D
:104EA000A847051E03DA04B0BDE8F087002594F892
:104EB00064313BB1504603F043FF10F0200F18BFA0
:104EC0004FF0FF35D4F848315BB929464046FDF72D
:104ED00095F9D4F81C312B44C4F81C312046FFF757
:104EE0005DFF7368AB4206F10806DCD80137CDE7F9
:104EF00030B590F8ED3085B00446002B51D0D0F895
:104F0000483100F1BC050BB340F2D742294603A853
:104F1000F8F750F904F59A7003F012FFD4F848310D
:104F200023EA0000C4F8480168B9236918680190B1
:104F300003F086FD636C019843F00803636404F199
:104F4000380103F06FFD03A8F8F750F994F83031F9
:104F5000DBB140F2F54204F1D40103A8F8F72AF9D5
:104F60002046FFF781FF636D63B104F17000FDF728
:104F7000CFF8B4F85830984204D3606D4FF4806194
:104F800003F000FF03A8F8F731F940F2FD4229468B
:104F900003A8F8F70FF92046FFF72AFE03A8F8F751
:104FA00025F905B030BD0000F8B51E4D0446A36AD2
:104FB0003BB92B68986A03684FF47A719B689847ED
:104FC000F5E700264FF47A7141F20C0003F0FAFE87
:104FD0000546FCF7C1FF831BB3F57A7F2ABF06465F
:104FE0000027012729070AD594F84C31C3B1236D56
:104FF000986B0130B52828BFB52004F013FA94F857
:10500000ED30002BDED06A0706D42FB9D4F8483132
:10501000002BD7D0EB04D5D52046FFF769FFD1E7A9
:105020003C20EAE73825002008B5FFF7BDFF000067
:1050300037B590F8EC30044603B390F83031EBB953
:1050400000F1D4014FF48B6201A8F8F7B3F8237D87
:10505000B3B92046FFF708FF636D63B104F1700038
:10506000FDF756F8B4F85830984204D3606D4FF409
:10507000806103F087FE01A8F8F7B8F803B030BDEF
:10508000D4F8B430002BE7D0302383F31188D4F860
:10509000B4305B681A68D20734D45D68C5F1400546
:1050A00015F0FF051DD094F85C3018332A4654F8EB
:1050B000231004F17000FDF7BBF8D4F81C31D4F8CC
:1050C00020212B4415442D1AC4F81C31C4F820515A
:1050D0002046FFF763FE94F80A3113B12046FFF72C
:1050E000E5FDD4F8B4305A68136823F00F03136059
:1050F000D4F8B430197C1A680E238B4053602046D4
:10510000FFF716FA002383F31188237D002BA3D128
:105110009FE70000104B70B5104C1D68A86A22680C
:1051200003689B681AB94FF47A719847F6E7A86A42
:105130000B4E03684FF47A719B6898470B2456F81E
:10514000040B20B190F8EC300BB1FFF771FF013C7C
:1051500014F0FF04F3D1EAE738250020646700204B
:105160003867002038B50446C8060D4604D5E06906
:1051700010B1022104F064FE690604D5A06910B1E3
:10518000022104F05DFEAA0604D5E06910B10121F8
:1051900004F056FE2B0606D5A06920B1BDE83840C4
:1051A000012104F04DBE38BD2DE9F74F03690D46CE
:1051B0005979044629B1B5FA85F0400903B0BDE834
:1051C000F08FC581D3F800809869D8F854205668CC
:1051D0009768126802F001091A7900F0A9FC2369A6
:1051E000E0611A795869012100F0A2FC2369A061ED
:1051F0001A79D869042100F09BFC236920621A798E
:10520000186A042100F094FC23686062DB6B94F858
:10521000091120469847D4E906A015F0080B1EBFD7
:1052200052468246104615F00403019303D0AB07A3
:1052300018BF45F00305E907D4F8282161D542F4E9
:10524000803246F48036C4F8282110B1022104F0DF
:10525000F7FDAB07D4F828215DD542F4003246F4BF
:105260000036C4F82821BAF1000F03D002215046BD
:1052700004F0E6FDD4F82831BBF1000F56D046F417
:10528000004643F40043019AC4F82831D4F82C3185
:10529000002A50D043F00803C4F82C3194F8303180
:1052A00047F0080763B9236918684FF48052182340
:1052B00004F59A71043003F00BFD012384F83031BA
:1052C000237D73B1D4F8B4305BB15A68136823F00E
:1052D0000F031360D4F8B430197C1A680E238B4086
:1052E00053600023A38229462046FFF73BFFD8F8EE
:1052F00054305A68B24225D19A68BA4222D101206C
:105300005CE722F4803226F48036C4F82821002895
:105310009FD001219BE722F4003226F40036C4F826
:105320002821BAF1000FA5D00121A0E726F40046FC
:1053300023F40043A7E723F0080327F00807C4F885
:105340002C31D0E7B9F1000F03D01A6822F0010226
:105350001A60D8F854305E60D8F854309F60B9F1C4
:10536000000FCCD0D8F85420136843F00103136029
:10537000C5E7000000487047D82E0208002070479B
:10538000014B0020197070476867002070470000CB
:10539000002070477047000004F0EEBB084609B1DA
:1053A00004F0E6BB7047000008B5134612780C2ADB
:1053B000A8BF0C2208461A70024904F0EDFF012034
:1053C00008BD00BF9075FF1F1046194604F09ABC37
:1053D00004F0AABC2DE9F34742F6F8216846F7F736
:1053E000CFFE534801A9FAF721FD524B05461C6830
:1053F00068B9A0694E4A03684F491B68984703245F
:105400006846F7F7C9FE204602B0BDE8F087019B69
:10541000606B1F3323F01F030193036800211B6897
:105420009847019A01460746284604F0A5FFA3695C
:105430001A68126838B91846404990472846FAF762
:1054400037FD0124DCE73E49184690470026B14667
:10545000019B4B4523D9606B03685FFA86F85B6854
:1054600041469847824620B92846FAF721FD022492
:10547000C6E7A06A03684FF47A711B699847606BAE
:1054800003684146DB689847013630B9A0692D4969
:1054900003681B6842469847E6E7D144D8E7A0690D
:1054A000234A036828491E68DFF8A8903B46B047A6
:1054B000606B036801215B6998474FF00108A06A9F
:1054C00003684FF47A711B699847606B03682A463A
:1054D0001E69019B3946B0470646A0690368D6B9E4
:1054E0004246D3F800A049460A23D047A06A036881
:1054F00064215B6808F101089847B8F10B0FDED111
:10550000606B036831465B699847A0690F4903687F
:105510000A221B68BFE71B680D499847606B036848
:1055200000215B6998472846FAF7C2FC002467E728
:10553000E8EA010838250020F02E0208032F0208AF
:105540001A2F0208232F0208342F0208702F020896
:10555000662F0208472F02082DE9F04F254B9DB01A
:1055600093F890200F9293F89120109293F8922044
:10557000119293F89320129293F8952093F89470D7
:10558000139293F89620149293F89720159293F81B
:1055900098B093F899A093F89A9093F89B8016ABE3
:1055A0000C46054614491722184605F0C5FB139A08
:1055B0000792149A0692159A05920F9A0492109ADD
:1055C0000392119A0292129A0C4B0897CDE90002AD
:1055D0000026CDE90989322221462846CDE90BABC8
:1055E0008DF86F60F7F724FF012084F831601DB05B
:1055F000BDE8F08F0075FF1F69E50108902F0208D4
:1056000004F006BD2DE9F0471B4A1C4CDFF87480FE
:10561000DFF874A0DFF8749086B010460F4604F0EF
:1056200029FC154A1649A41A034600943846FCF78B
:10563000D9FC03F09DFC0446D4B1256AE269A36B52
:1056400005924545284614BF661BAAEB080604933D
:1056500004F010FCDDE90432CDE901064946384684
:105660000095FCF7BFFC204603F092FC0446E3E7FC
:1056700006B0BDE8F08700BF000100200007002051
:10568000C82F02080007002000230020FB2F02087B
:10569000084600F0F9B800002DE9F04188B00D4649
:1056A00004A805A904F0ACFA1549DFF858800646AD
:1056B0002846FCF797FC00242746E0B286421CD916
:1056C000CDE9067710B1049B03EB441007AA06A9A5
:1056D00003F0D4FA05990C2262438818D0E901300E
:1056E000029007980190069800908A589B0A4146BC
:1056F0002846FCF777FC0134DFE708B0BDE8F0810D
:10570000203002082B30020808460AB904F000BA1B
:10571000012A01D104F024BA022AF7D0012004F0B2
:1057200023BA000070B50C4615462AB9084604F0A5
:105730001FFA2E46304670BD104619B9BDE87040BC
:1057400004F0E2B904F0E0F906460028F2D054F87B
:10575000042CAA4228BF2A46214604F01DFE2046FA
:1057600004F006FAE6E7000070B50C461546002680
:10577000AE4204D2F8F758FBA0530236F8E7EB0725
:1057800004D5F8F751FB2C4404F8010C012070BD3E
:10579000F7F718BE38B5054D00242846013403F04C
:1057A00043FB102C05F12005F7D138BD70670020B0
:1057B00082B010B5914203934FF00003C0E900336B
:1057C000C0E9023304460174427484BF0274417418
:1057D000DDE9030184E80300DDE9050104F10803C4
:1057E00083E803002046BDE8104002B07047000087
:1057F0000F289DBF4FF4004323FA00F000F0010092
:10580000002070470F2838B50AD8074B03EB401526
:105810002846AC6803F04AFB14B1AB689C4201D146
:10582000002038BD0120FCE7706700200F2938B543
:105830000446154610D8094800EB411003F062FBFE
:1058400055B1074B1B683BB1227C02EB420203EBD4
:1058500082039A6801329A6038BD00BF70670020E9
:105860006C67002013B5002304460A468374019137
:10587000417CFFF7DBFF019A217C204602B0BDE8A6
:105880001040FFF7D3BF00002DE9F04F354E2DED4E
:10589000028B33688BB007461BB9CC20F7F722FB8D
:1058A000306031499FED318ADFF8C4803846FCF71B
:1058B00099FB00254FF00C09326809FB05F4EBB2A7
:1058C000115902EB040C31B9DCF8041019B9DCF8F9
:1058D000081000293DD0111991ED007A52F804E02A
:1058E000DCF80400DCF8081007910EEB0001013130
:1058F00007EE901AB8EE477AF8EE677A27EE087A44
:10590000DCF804A052F804B0C7EE277A0722B3FBF4
:10591000F2F2C2EBC20CA3EB0C0301330132DBB297
:10592000D2B20993089217EE900AF4F7DFFD079BB5
:105930000093CDE90401DDE90823CDE901AB41463F
:105940003846FCF74FFB336800221A513368234472
:105950005A600135102DAFD10BB0BDEC028BBDE804
:10596000F08F00BF6C670020E43002080000C842DE
:10597000EB300208D0E900031847000038B50446B0
:10598000007C0F280FD8454D05EB4013D96951B164
:10599000A14208D018461430FFF7ECFF237C05EB3A
:1059A00043150023EB61607C0F280FD83B4D05EBBE
:1059B0004013D96951B1A14208D018461430FFF7FD
:1059C000D9FF637C05EB43150023EB61237C0F2B90
:1059D00004D8324A02EB4312D26942B1627C0F2AE8
:1059E00048D82E4901EB4212D269002A53D12146F0
:1059F0002046FFF7BFFF237C0F2B0BD8274AD4E9A3
:105A0000020102EB4313143383E80300237C02EB0F
:105A10004312D461637C0F2B0BD8204AD4E90201D6
:105A200002EB4313143383E80300637C02EB43125D
:105A3000D4611B480268D2B1237C0F2B09D8E57CC6
:105A400003EB4303990002EB8303E5B153580133A1
:105A50005350637C0F2B0AD80268E07C03EB4303AE
:105A6000990002EB830390B1535801335350012343
:105A7000A37438BD102B01D0102ADAD1214620465C
:105A8000FFF778FFD5E75A6801325A60E1E75A68B4
:105A900001325A60EBE7102BEFE700BF7067002080
:105AA0006C67002038B50446007CFFF7ABFE054666
:105AB000607CFFF7A7FE002D08BF0546E574204671
:105AC000BDE83840FFF75ABF044B11220021013ACC
:105AD000C3E9051103F12003F9D170477067002075
:105AE00070470000704700007047000000207047BA
:105AF000704700000020704782B002A9002001E931
:105B00000C0002B070470000002070470079704719
:105B10000020704700207047002070477047000049
:105B200001207047014B0360704700BF2831020815
:105B3000704700002DE9F7432C4E0546071DFCF782
:105B400011FA2C6A80468946FCB1D4E904239045B9
:105B500079EB030317D3D4E90412884579EB0203E8
:105B600006D3E3685B1842F10002C4E90432F2E7AD
:105B70004522394601A8F7F71DFBD4E901039847F0
:105B800001A8F7F733FB2468DEE7FCF7EBF92A6A94
:105B9000234692B154EA0308D2E904EC03D0A645A7
:105BA0007CEB030807D2704571EB0C0804460B46EA
:105BB0003CBF744663461268EBE7844273EB010214
:105BC0004CF250320AD3241A63EB0103944273F16E
:105BD000000303D2642C224638BF64223368986ADB
:105BE000036891B29B689847A9E700BF3825002059
:105BF00038B504460D460430FBF77EFB04F1340053
:105C000084F8245000220A2104F03EF904F13800FF
:105C100000220A2104F038F9204638BD2DE9FF4161
:105C200002AF87E80C0090F82C30DDF8288005469C
:105C30000E464BBB012380F82C30C0F83080072083
:105C400003F062FF0446A0B398F8083003F007029F
:105C5000012A10D0022A14D0184B95F82420009560
:105C600021464FF4BE6003F0ADFFA86260B914484E
:105C70002146FCF74BF9134ADB080721FBF752FBDF
:105C8000EAE7114ADB08F8E71820F7F725F9044698
:105C900078B1031D97E8030083E80300E660FCF792
:105CA00061F9301841F10001C4E904012B6A236055
:105CB0002C62204604B0BDE8F08100BF355B0108CE
:105CC000783102086C3102087231020838B5094B8C
:105CD0001446DB68826A9A420D4609D1CC60FCF713
:105CE00041F9201841F10001C5E90401012038BD46
:105CF0000020FCE7886F0020F8B51E461B680546AB
:105D00000C4617461BB9236863B9012408E0BDF8A7
:105D10001820806B314604F0CFF80028F3D100241E
:105D20002046F8BD2146686B3A4604F0FFF8044669
:105D30000028EAD13368002BF1D0A86B04F02EF9CB
:105D4000EEE7000038B50D46114604461A4611B17B
:105D5000806B04F0DDF82DB1606B2946BDE838405A
:105D600004F014B938BD00002DE9F041456A15B9B9
:105D70004162BDE8F0818B6823F06047C3F38A4637
:105D80004FEAD37EC3F3807816EA230638BF3E4637
:105D9000AC462B469A68BEEBD27F22F060440AD014
:105DA000002A18DAA40CB44217D19D420FD10D601D
:105DB000DEE71346EEE7A74207D102F08044C2F3C4
:105DC000807242450BD054B1EFE708D2EDE7CCF832
:105DD00000100B60CDE7B44201D0B442E5D81A6898
:105DE0009C46002AE5D11960C3E700002DE9F04781
:105DF000089D01F007044FEAD508224405F0070585
:105E000000EBD1004FF47F49944201D1BDE8F08707
:105E100004F0070705F0070A57453E4638BF5646C7
:105E2000C6F10806111B8E4228BF0E46E10808EB9A
:105E3000D50E415C13F80EC0B94029FA06F721FAD5
:105E40000AF1FFB28CEA010147FA0AF739408CEAFD
:105E5000010C03F80EC034443544D5E780EA012034
:105E6000082341F2210201B24000002980B203F16F
:105E7000FF33B8BF504013F0FF03F4D17047000068
:105E800038B50C468D18A54200D138BD14F8011B59
:105E9000FFF7E4FFF7E7000042684AB11368436088
:105EA0004389818901339BB29942438138BF838101
:105EB0001046704770B588B0202204460D466846EB
:105EC000002104F077FA20460495FFF7E5FF02462B
:105ED00058B16B46054608AE1C4603CCB442286058
:105EE0006960234605F10805F6D1104608B070BD7B
:105EF000082817D909280CD00A280CD00B280CD058
:105F00000C280CD00D280CD00E2814BF40203020B7
:105F100070470C20704710207047142070471820DD
:105F20007047202070470000082817D90C280CD98A
:105F300010280CD914280CD918280CD920280CD9D1
:105F400030288CBF0F200E207047092070470A2090
:105F500070470B2070470C2070470D2070470000E1
:105F60002DE9F843078C072F04461ED9D0E9029883
:105F700000254FF6FF73C5F12006A5F1200029FA90
:105F800005F108FA06F628FA00F031430143C9B2D8
:105F90001846FFF763FF0835402D0346EBD1E16952
:105FA0003A46BDE8F843FFF76BBF4FF6FF70BDE818
:105FB000F883000010B54B6823B9CA8A63F309025D
:105FC000CA8210BD04691A681C600361C38A013B60
:105FD000C3824A60EFE700002DE9F84F1D46CB8AE7
:105FE0000F46C3F309010D29814692460B4630D076
:105FF0000020AAB207F11A049EB20C2E1FFA80F8F4
:106000000FD8904503F1010306D3FB8A0A4462F3DB
:106010000903FB8201201AE01AF80060E6540130FF
:10602000EAE79045F1D2A1F10D0B24237C68BBFB7C
:10603000F3F203FB12BB1FFA8BF6002C46D1484645
:10604000FFF72AFF044638B978606FF00200BDE818
:10605000F88F4FF00008E6E7002606607860ADB2E2
:106060004FF0000B454510D90AEB0803221D13F829
:10607000011B9155B1B208F1010823291FFA88F8D4
:106080002CD0454506F10106F1D8FB8AC3F309027D
:10609000154465F30903BCE7013292B21C4623683C
:1060A000002BF9D1A5F10D030B442421B3FBF1F32F
:1060B00001339BB29A42D2D2BBF1000FCFD14846F6
:1060C000FFF7EAFE20B9C4F800B0BEE70122E6E718
:1060D000C0F800B05E4620600446C0E74545D4D90C
:1060E0004846FFF7D9FE08B92060AEE7C0F800B017
:1060F000002620600446B5E72DE9F04F2DED028B18
:106100001C4683B05B69019207468846002B00F06D
:10611000B280238C2BB1E269002A00F0AC80072BFF
:106120003AD807F10C00FFF7B7FE054638B96FF013
:106130000206304603B0BDEC028BBDE8F08F28228A
:10614000002104F037F9228CE16905F1180004F010
:1061500023F9208C013080B2FFF7E6FEFFF7C8FE7E
:10616000013880B22084013085F820006369228CD8
:106170001B782A4403F01F0363F03F0348F00041FB
:106180001376A960D4E90A232946C5E904233846D1
:10619000FFF7EAFD0126CCE702339BB20722C18A52
:1061A0000633B3FBF2F3828A521A9BB292B2934245
:1061B000BDD800F10C034FF0000908EE103A4FF083
:1061C000800ACB464E4618EE100AFFF765FE0546DC
:1061D0000028ACD02822002104F0ECF8BBF1000F1D
:1061E0003CD1019B2B83022205F1180E1FFA82FC81
:1061F0000CF10100BCF1060F218C80B201D88B4557
:106200002ED3FFF791FEFFF773FE62691278013813
:1062100002F01F028B4508BF4FF0400A42EA4912C4
:1062200015FA80F14AEA020A013048F0004281F88A
:1062300018A0AA6085F82000D4E90A01C5E9040184
:1062400029463846FFF790FD228C01365A4536B272
:1062500089F001094FF0000AB5D16AE70022C3E7CF
:10626000E1690BF1010311F80B100EF802101FFA8F
:1062700083FB0132BAE76FF001065AE7F8B515461D
:106280000E463022002104461F4604F093F8B5F56F
:10629000201F069B636038BF2822079BA76028BF8A
:1062A0004FF6FF72A36238BFB5FBF2F2E66197B218
:1062B00004F1100000239A4206D800230360A7824D
:1062C000E3822383E360F8BD06600133304628365D
:1062D000F1E7000003781BB94BB2002BC8BF017077
:1062E0007047000000787047F8B50C46C96907464A
:1062F00011B9238C002B37D1257E1F2D34D8387847
:1063000028BB228C072A2CD8268A36F003032BD1EF
:106310004FF6FF70FFF7B4FD20F00100310240049A
:1063200041EA0561400C41EA40254FF6FF722346E1
:1063300029463846FFF7E0FE002807DD626913783A
:106340000133DBB21F2B88BF00231370F8BD218AF5
:106350002D0645EA012505432046FFF701FE0246CA
:10636000E5E76FF00300F1E76FF00100EEE70000F2
:106370002DE9F041D36905460C4616460BB9138C3E
:106380005BBB377E1F2F28D895F80080B8F1000F2F
:1063900026D03046FFF7E4FD3378210241EAC331CD
:1063A00041EA0801338A41EA076141EA03410246B2
:1063B000334641F080012846FFF79EFE00280ADDA3
:1063C0003378012B07D1726913780133DBB21F2BAD
:1063D00088BF00231370BDE8F0816FF00100FAE779
:1063E0006FF00300F7E70000406A00B10830704723
:1063F000436A1A68426202691A600361C38A013BF8
:10640000C38270472DE9F041D0F820802A4E14460F
:106410001D464146002721B9416A0B4661BBBDE8D4
:10642000F081D1E90232E31A65EB02029E4277EB7A
:1064300002031ED2036A8B420DD1FFF7BBFD036A34
:106440001B68036203690B60C38A0161016A013B37
:10645000C3828846DFE7FFF7ADFD0B68C8F8003060
:1064600003690B60C38A0161013BC382D8F8001045
:10647000D1E788460968CEE7D1E90476A742AE4164
:106480000A680BD2466A8E420BD1036942620B60E6
:10649000C38A0161416A013BC3820A460B46114629
:1064A000BCE71A6002690A60C28A0161013AC282CD
:1064B0001A681946F2E700BF80841E002DE9F04FEC
:1064C0008BB00D46DDF8509014469B468046002860
:1064D00000F01B81B9F1000F00F01781531E3F2B14
:1064E00000F21381012A03D1BBF1000F40F00D81AE
:1064F0000023CDE90833B8F81430B5EBC30F4FEAE9
:10650000C30703D300200BB0BDE8F08F2B199F42C7
:10651000D8F80C303ABF7F1BFFB227461BB9D8F81A
:106520001030002B7CD0672D4ED8C5F16806B742DD
:106530004FF000032CBFF6B23E4600932946D8F830
:10654000080008AB3246FFF751FCA7EB060A3544BA
:106550005FFA8AFAB8F8143003F100530D3BDB0000
:106560000493D8F80C3003936821039B13B1BAF15C
:10657000000F2CD1D8F8100040B1BAF1000F05D0AF
:10658000009608AB5246691AFFF730FC38B2002F6C
:10659000B8D066070AD00AAB03EBD401624211F807
:1065A000083C02F00702134101F8083C082C3ED9D0
:1065B000102C40F2B780202C40F2B980BBF1000FC4
:1065C00000F09E80082336E0BA460026C2E7049B0E
:1065D000B3F5907F28BF4FF4907306930B44AB4202
:1065E000059314D95A1B03980096924534BF52461E
:1065F000D2B2691A08AB04300792FFF7F7FB079A8B
:106600001644AAEB020A1544F6B25FFA8AFA049B12
:10661000069A05999B1A0493039B1B680393A4E7AE
:106620000093D8F8080008AB3A462946ACE7BBF11E
:10663000000F13D00123B4EBC30F6CD0082C12D879
:106640009DF82030621E23FA02F2D50706D54FF0DE
:10665000FF3202FA04F423438DF820309DF82030F5
:1066600089F800304FE7102C12D8BDF82030621E98
:1066700023FA02F2D10706D54FF0FF3202FA04F4F2
:106680002343ADF82030BDF82030A9F800303AE7B8
:10669000202C0FD80899631E21FA03F3DA0705D5D9
:1066A0004FF0FF3202FA04F40C430894089BC9F837
:1066B000003028E7402C2BD0DDE90865611EC4F1CD
:1066C0002102A4F1210326FA01F105FA02F225FACA
:1066D00003F311431943CB0712D50122A4F1200380
:1066E000C4F1200102FA03F322FA01F1A24052425E
:1066F00043EA010363EB430332432B43CDE9082311
:10670000DDE90823C9E90023FDE66FF00100FAE6A0
:106710006FF00800F7E6082CA0D9102CB3D9202C74
:10672000EED8C3E7BBF1000FADD0022383E7BBF186
:10673000000FBBD004237EE730B5012A144638BFD2
:106740000124402C85B028BF40240025012ACDE932
:10675000025518D81B788DF8083063070AD004ABAF
:1067600003EBD405624215F8083C02F0070293409F
:1067700005F8083C009103462246002102A8FFF7D5
:1067800035FB05B030BD082AE4D9102A03D81B8890
:10679000ADF80830E1E7202A8DBFD3E900231B685C
:1067A0000293CDE90223D8E710B5CB681BB98B6003
:1067B0000B618B8210BD04691A681C600361C38A77
:1067C000013BC382CA60F0E703460A8B4869186040
:1067D0009A8018467047000003064CBFC0F3C030D3
:1067E0000220704708B50246FFF7F6FF022806D1DF
:1067F0005306C2F30F2001D100F0030008BDC2F31D
:106800000740FBE72DE9F04F93B0CDE903230A6879
:1068100004461046FFF7E0FF022814BFC2F3062625
:106820000026002A0D46824680F2FD8112F0C04902
:1068300040F0F981097E002900F0F581022803D09B
:106840002378B34240F0F281C2F30463069310460A
:1068500002F07F030593FFF7C5FF059B29444FEA2C
:10686000834848EA0A4848EA4668CE7B002300226B
:10687000CDE90823F309834648EA0008029367D06C
:10688000059B009302466768534608A92046B8470F
:10689000002800F0CE81276A4FB9414604F10C0070
:1068A000FFF708FB074690B96FF0020054E03B6920
:1068B00098450DD03F68002FF9D1414604F10C00F6
:1068C000FFF7F8FA07460028EED0236A3B602762FC
:1068D00097F817C006F01F08CCF3840CACEB080047
:1068E0001FFA80FE0028B8BF0EF12000A8EB0C03B1
:1068F0001FFA83FED7E90221B8BF00B2002B07932D
:10690000BEBF0EF120031BB2079352EA010338D039
:10691000039BDFF828E39A1A049B4FF0000C63EB0B
:10692000010196457CEB01032BD36B7E97F81AE0AF
:10693000734519D1029B002B79D0012821DC78689E
:10694000F8B9DFF8F4C2944570EB010316D337E0D1
:10695000276A27B96FF00C0013B0BDE8F08F3B69D0
:106960009845B5D03F68F4E7B34890427CEB01030B
:1069700001D30020F0E7029B002BFAD0079B0F2BDE
:1069800017DCFA7DB30002F0030203F07C0313432B
:10699000FB7539462046FFF70DFB6B7EBB76029BED
:1069A0003BB9FB7DC3F38402013262F38603FB75BE
:1069B000D0E76A7EBB7E9A42DBD1029B002B36D0A9
:1069C000B309022B33D0039BBB60049BFB601422F2
:1069D00000210DA803F0EEFC039B0A93049B0B938C
:1069E00005F110030C932B7EADF83EB0013BDBB2FA
:1069F000ADF83C30069B8DF84230059B8DF8433056
:106A000094F82C308DF840A083F001038DF84430C9
:106A10008DF84180A3680AA920469847FB7DC3F3FF
:106A20008403013303F01F039B02FB82A1E7FB7D7C
:106A3000C6F34012B2EBD31F40F00281C3F38403CC
:106A4000434540F00081029A2B7EB609002A53D0BC
:106A500016F0010663D1032B40F2F880039BBB6064
:106A6000049BFB60FB8A66F30903FB822B7E05F126
:106A70001206033BDBB23246394604F10C00FFF745
:106A8000ABFA00280CDA39462046FFF793FAFB7D73
:106A9000C3F38403013303F01F039B02FB8203E76C
:106AA000DDE908842B8A3B834FF6FF73C9F1200090
:106AB000A9F1200228FA09F104FA00F0014324FAAE
:106AC00002F211431846C9B2FFF7C8F909F10809E3
:106AD000B9F1400F0346E9D1B8822A7E033AD2B217
:106AE0003146FFF7CDF9FB7DB882DA43C2F3C0121D
:106AF00062F3C713FB753CE78EB905F11006013B45
:106B0000DBB23246394604F10C00FFF765FA002883
:106B1000B9DB2A7EB88A013AD2B23146E1E7F98A76
:106B2000C1F30901013B0C29DAB25DD805F110006F
:106B3000002307F11B069A4208D910F801CB06F88A
:106B400001C0013101330D29DBB2F4D103990A915F
:106B500004990B91934207F11B010C9138BF10333C
:106B600079680D9134BF55FA83F300230E93FB8AA5
:106B7000ADF83EB0C3F309031A44069B8DF84230CA
:106B8000059B8DF8433094F82C30ADF83C2083F011
:106B900001038DF8443000238DF840A08DF841802A
:106BA0007B602A7EB88A013A05F11001FFF768F987
:106BB0003B8BB882834203D1A3680AA92046984739
:106BC00020460AA9FFF7F0FDFB7DBA8AC3F38403D0
:106BD000013303F01F039B02FB823B8B9A420CBFE5
:106BE00000206FF01000B7E67B68002BAED00D20C0
:106BF00001E0243033461E68002EFAD1091A081D20
:106C000005F11006184401EB090CBCF1230F5FFAE3
:106C100089F39BD89A4299D916F8013B00F8013BB9
:106C200009F10109EFE76FF0090095E66FF00A003E
:106C300092E66FF00B008FE640420F0080841E004A
:106C40006FF00D0088E66FF00E0085E66FF00F0024
:106C500082E600BFEFF3098305494A6B22F0010287
:106C60004A63683383F30988002383F311887047EC
:106C700000EF00E0302080F3118862B60C4B0D4A23
:106C8000D96821F4E0610904090C0A43DA60D3F8F9
:106C9000FC20094942F08072C3F8FC200A6842F0E7
:106CA00001020A602022DA7783F82200704700BFD1
:106CB00000ED00E00003FA05001000E010B53023FD
:106CC00083F311880E4B5B6813F4006314D0F1EE6C
:106CD000103AEFF30984683C4FF08073E361094B8D
:106CE000DB6B236684F3098802F012FA10B1064BBD
:106CF000A36110BD054BFBE783F31188F9E700BFE3
:106D000000ED00E000EF00E01FB1000822B1000834
:106D1000F0B500F10B04002B14BF1D460D462346B1
:106D2000B1FBF2F702FB171101F13006392EC8BF93
:106D300001F1370603F8016D2E4696423946B5FB40
:106D4000F2F5EDD2421EE11A13F8015B02F8015F81
:106D5000A342F9D10844F0BD2DE9F04F2DED048B8D
:106D600006468BB0904600270C4614F8013B002BDA
:106D70003FD0252B06D032681946D268304690475E
:106D80000137C3E14B782D2B06BF8C1C0123002358
:106D9000029323782B2B04BF01344FF0010B94F89E
:106DA00000A018BF4FF0000BBAF1300F0CBF013438
:106DB0004FF0200A23782A2B21D158F8043B019365
:106DC000023414F8013C2E2B48D123788BB12A2BA6
:106DD00026D0611C4FF000090A20A3F13002D2B284
:106DE000092A0C4620D811F8013B00FB0929002B89
:106DF000F3D138460BB0BDEC048BBDE8F08F002317
:106E000001930A2114F8013B002BF2D0A3F13002C8
:106E1000D2B2092AD7D8019B01FB03230193F1E7E2
:106E200058F8049B6378023403F0DF024C2A18D12F
:106E30002378002BDDD0782B04F1010420D8622BBD
:106E400000F27081582B1BD84E2B00F29F81442BEF
:106E500000F09680492B00F0938011E04FF000097C
:106E6000E2E7A3F14102782BD2B209D8622B0BD80A
:106E7000582B05D84E2B3BD8442B7CD0492B7AD0AD
:106E80008DF81030454656E0A3F163001528F7D879
:106E900001A555F820F000BF296F0108776F0108A0
:106EA000816E010815700108816E0108816E01086C
:106EB000776F0108816E0108816E0108816E0108FB
:106EC000816E0108816E0108D7700108C97101083F
:106ED000816E0108816E0108416F0108816E010811
:106EE000C5710108816E0108816E0108C971010830
:106EF000A3F14F02092AC3D801A050F822F000BF25
:106F0000D7700108C9710108816E0108816E0108FE
:106F1000816E0108816E0108C5710108816E01084A
:106F2000816E0108C971010845464FF0200A55F8E5
:106F3000043B8DF810300DF110080DF1110030E018
:106F40004546A24B55F8048BB8F1000F08BF984690
:106F500047F6FF73B9F1000F08BF9946C144434695
:106F6000184613F8012B1AB1A9EB0302002AF7DA2D
:106F70004FF0200A15E04546192A55F8041B02D89F
:106F8000454655F8041B00293BDA2D238DF81030B7
:106F900049420DF1110000230A22FFF7B9FE0DF15D
:106FA0001008019B0299A0EB0809A3EB090222EA51
:106FB000E273002940F0AC80002AC3F1000B1EDD13
:106FC00098F800102D2901D02B290DD1BAF1300FDE
:106FD0000AD132680193D26830469047019B01374D
:106FE00009F1FF3908F1010832680193D26851466E
:106FF000304690471BF1010B019BF5D11F444B46D6
:1070000078E0BBF1000F03D02B238DF81030C0E7E0
:1070100004A8C0E708F1070525F00705F5E8020117
:10702000F3F7B4FD08EE100AB5EEC08AF1EE10FADF
:1070300047D52D238DF81030B1EE488A0DF1110897
:1070400018EE100AF3F752FA09F1FF33092B28BFA3
:107050004FF0090909F1FF395D4BFDEEC87A53F88D
:107060002930039341EC190B0A2217EE901A0023E2
:107070004046FFF74DFE83462E2317EE900A0BF88D
:10708000013BF3F721FA02460B4651EC190BF3F7DB
:10709000CDF8804603988946F3F706FA02460B4678
:1070A00040464946F3F77AFA4FF00A08039BB3FBD0
:1070B000F8F30393F3F722FD039B0146424658463B
:1070C0006BE7BBF1000F03D02B238DF81030B5E731
:1070D0000DF11008B4E708224546002355F8041BBB
:1070E00004A85AE7326818F8011BD26801933046A9
:1070F0009047019B013BF5D5B9F1000FA8BF4F4464
:10710000D846B8F1000F05D15F44A84621462BE6CA
:107110009B4674E733685146DB683046984708F170
:10712000FF38EEE7A3F16302152A3FF6A9AE01A1ED
:1071300051F822F0296F0108816F0108816E010862
:1071400015700108816E0108816E0108816F0108C8
:10715000816E0108816E0108816E0108816E01084F
